:020000040000FA
:10C000003DB8F39600C000002000000074C200009C
:10C01000000000000104000000000000000000001B
:10C02000DEADC0DEDEADC0DEDEADC0DEDEADC0DE6C
:10C03000DEADC0DEDEADC0DEDEADC0DEDEADC0DE5C
:10C04000DEADC0DEDEADC0DEDEADC0DEDEADC0DE4C
:10C05000DEADC0DEDEADC0DEDEADC0DEDEADC0DE3C
:10C4000000000120791E01008D1B0100051C0100A8
:10C41000A11B0100B51B0100C91B0100DD1B0100B0
:10C42000000000000000000000000000491C0100A6
:10C43000F11B0100000000005D1C0100711C0100E7
:10C44000000000000000000000000000D51C0100FA
:10C4500000000000E91C01000000000000000000D6
:10C460007127010035280100435F0100D55F0100FD
:10C4700000000000FD1C0100111D0100251D010030
:10C48000391D01004D1D01000000000000000000EA
:10C49000851C0100F12301000000000000000000E5
:10C4A000611D01000000000000000000991C010057
:10C4B000AD1C0100751D0100891D01009D1D0100BD
:10C4C000B11D0100C51D0100D91D0100ED1D0100B8
:10C4D000011E010000000000151E01000000000008
:10C4E000291E010000000000C11C01000000000026
:10C4F0003D1E0100000000000000000000000000E0
:10C500000000000075220100000000000000000093
:10C51000000000000000000000000000000000001B
:10C5200000000000511E010000000000000000009B
:10C5300000000000000000000000000000000000FB
:10C54000651E010000000000000000000000000067
:10C5500000000000000000000000000000000000DB
:10C5600000000000000000000000000000000000CB
:10C5700000000000000000000000000000000000BB
:10C5800000000000000000000000000000000000AB
:10C800003E3D3D484558494E464F3D3D3E61707066
:10C810002D626F6F742D6E7266393136302D7365EF
:10C82000632076312E342E3020545A3220284A7517
:10C830006E20323520323032302031363A33303AC1
:10C840003437293C3D3D484558494E464F3D3D3CD7
:10C8500000DEADBEEFDEADBEEFDEADBEEFDEADBEE7
:10C86000EFDEADBEEFDEADBEEFDEADBEEFDEADBEE8
:10C87000EFDEADBEEFDEADBEEFDEADBEEFDEADBED8
:10C88000EFDEADBEEFDEADBEEFDEADBEEFDEADBEC8
:10C89000EFDEADBEEFDEADBEEFDEADBEEFDEADBEB8
:10FBF000EFDEADBEEFDEADBEEFDEADBEEFDEADAA39
:10FC00007FE97FE901F080BE7FE97FE905F066BF0B
:10FC10007FE97FE901F0C8BA7FE97FE901F054BAD2
:10FC20007FE97FE901F022BB7FE97FE905F00BBFA7
:10FC30007FE97FE901F0FABB7FE97FE906F00AB8C6
:10FC40007FE97FE906F04CB87FE97FE901F0AABEC1
:10FC50007FE97FE905F0A9BF7FE97FE901F04EBBAD
:10FC6000FFFFFFFFFFFFFFFFFFFFFFFFFFFFFFFFA4
:10FC7000FFFFFFFFFFFFFFFFFFFFFFFFFFFFFFFF94
:10FC8000FFFFFFFFFFFFFFFFFFFFFFFFFFFFFFFF84
:10FC9000FFFFFFFFFFFFFFFFFFFFFFFFFFFFFFFF74
:020000040001F9
:100000002DE9F04F456A97B0044606910B92129382
:10001000DDF8808057EC106BCDE900673DB910200A
:1000200003F0C6FD60620560C560C0E90155636A02
:10003000196851B15A680123204693404A608B6089
:1000400006F011FE636A00221A603B1EB7BF23F060
:100050000043002301220193ACBFC8F80030C8F868
:100060000020AF4BDDF8048033EA080314D142F2DC
:100070000F73129A1360009B23B9C8F31300002872
:1000800000F03E85219BDFF8ACB2002B00F04085EC
:100090000BF1030300F03ABDDDE900670022002305
:1000A0003046394605F0F4FA814668B10123129AC8
:1000B0001360219B002B00F020859A4B219A03F1BD
:1000C000FF3B136000F024BDC8F30A5514AA15A91C
:1000D000204647EC106B06F0D4FF0490002D7AD038
:1000E000C7F31303B246A5F2FF35CDF84C9043F0A9
:1000F0007F5B4BF4401B00228B4B5046594604F06B
:10010000A7FE81A3D3E9002305F05AF880A3D3E921
:10011000002304F09FFE06460F46284604F0E6FF43
:100120007DA3D3E9002305F04BF802460B46304689
:10013000394604F08FFE06460F4605F0F1FA00221C
:10014000824600233046394605F0ACFA48B15046A5
:1001500004F0CCFF32463B4605F09AFA08B90AF1A2
:10016000FF3ABAF1160F57D8704901EBCA01DDE921
:100170000023D1E9000105F0B3FA00284ED00AF1BE
:10018000FF3A00230F93149B5D1BB5F1010849BF93
:10019000C5F1010300234FF00008059358BF0593F4
:1001A000BAF1000F3CDB0023D044CDF838A0079310
:1001B000069B092B00F28E80052BC5BF043B002552
:1001C00001250693069B023B032B00F28F80DFE89C
:1001D00003F07D7F3171DDE914531D4405F2324097
:1001E000202813DDC0F14000009B08FA00F805F25A
:1001F000124023FA00F048EA000004F067FF0123F0
:100200008246A1F1F87B013D139374E7C0F1200011
:10021000009B03FA00F0F0E70123B3E70F90B2E789
:10022000059BA3EB0A030593CAF100030793002380
:100230000E93BDE701230A930B9B002B59DD9946D2
:1002400002930022666A7260042202F1140071684F
:10025000984253D9204606F0D2FC636AB9F10E0FDA
:100260003060D3F800B000F2E880002D00F0E580A7
:10027000BAF1000F9DED007B8DED107B76DD0AF06D
:100280000F032A4A4FEA2A1602EBC303F00693ED46
:10029000007B8DED087B67D5254B06F00F06032507
:1002A000D3E90823DDE9100105F0B4F8CDE9000138
:1002B0001F4F4EE001230A930B9B534403F10109A6
:1002C00002934B46012BB8BF0123BAE70023B2E7E4
:1002D0000023F0E7012500230A9506934FF0FF3332
:1002E00000220293994612230B92AAE701230A9354
:1002F000F4E70123029399461A46F5E701315200CB
:100300007160A2E7AFF3008061436F63A787D23FBC
:10031000B3C8608B288AC63FFB799F501344D33FF4
:100320000000F07F2E7F01000000F83FA87301005D
:10033000807301005A7F0100F10708D50135DDE91E
:100340000801D7E9002304F03BFFCDE9080176104E
:100350000837002EF0D1DDE90823DDE9000105F0C2
:1003600059F8CDE900011AE00225A1E700F0A080CC
:10037000CAF100069F4BA04F022506F00F0236116E
:1003800003EBC203DDE91001D3E9002304F018FFF9
:100390000023CDE90001002E7FD1002BE1D10F9B7E
:1003A000002B00F087800022944BDDE90067304687
:1003B000394605F077F900287CD0B9F1000F79D0E3
:1003C000029B002B35DD0AF1FF333946002230460F
:1003D000089301358A4B04F0F3FE029FCDE900013A
:1003E000284604F083FEDDE9002304F0E9FE002244
:1003F000844B04F02FFD0546A1F15076002F5DD10E
:100400000022814BDDE9000104F022FD2A4633463B
:10041000CDE9000105F064F9002840F087822A4602
:1004200006F10043DDE9000105F03CF9002840F049
:100430007B82DDE91023CDE90023159B002BC0F260
:100440004F81BAF10E0F00F34B816A4B03EBCA03E5
:1004500093ED007B0B9B002B8DED027B80F2D8800F
:10046000B9F1000F00F3D48040F05D820022664BAA
:100470004F464E4651EC170B04F0A2FEDDE9002377
:1004800005F024F9002840F0338231230BF10105F7
:100490000AF1010A8BF800302EE2F20705D501358A
:1004A000D7E9002304F08CFE01237610083772E7A9
:1004B000022574E7CDF820A04F4691E74D4B03EBA2
:1004C000C70353E902010A9B002B47D002460B46A3
:1004D00000204E4904F09EFF2A465D46334604F054
:1004E000B7FCCDE90C01DDE9000105F019F906467C
:1004F00004F0FCFD024630360B46DDE9000104F055
:10050000A7FC05F8016BDDE90C23CDE9000105F03E
:10051000C9F8002862D100203849DDE9002304F041
:1005200097FCDDE90C2305F0BDF8002840F0B7800A
:10053000A5EB0B039F427FF77CAF0022304BDDE938
:100540000C0104F03DFE00222D4BCDE90C01DDE94C
:10055000000104F035FECDE90001C4E72A46334628
:100560000BEB07055E4604F02BFECDE90C01DDE93F
:10057000000105F0D5F8074604F0B8FD0246303713
:100580000B46DDE9000104F063FC06F8017BAE4296
:100590004FF00002CDE9000125D11C4BDDE90C0133
:1005A00004F058FC02460B46DDE9000105F098F81E
:1005B000002874D100201549DDE90C2304F048FC23
:1005C00002460B46DDE9000105F06CF800283FF417
:1005D00030AF15F8013C6A1E302B02D0DDF820A0A8
:1005E0004BE01546F5E7064B04F0EAFDCDE90001C6
:1005F000BDE700BFA8730100807301000000F03F59
:100600000000244000001C40000014400000E03FB7
:10061000DDE900675D4630463946DDE9022304F036
:10062000F9FE05F07DF8804604F060FDDDE9022367
:1006300004F0C6FD0246304608F130060B46394646
:1006400004F006FC05F8016BA5EB0B0602460B4611
:10065000B14538D104F0FEFB06460F46DDE9022322
:1006600005F03EF8C8B930463946DDE9022305F009
:100670000FF810B118F0010F0FD10499204606F0C1
:10068000F2FA0023129A2B700AF101031360219BE6
:10069000002B00F03D821D603AE2CDF820A015F855
:1006A000012C6B1E392A08D19B450AD1089B0133C6
:1006B000089330238BF800305B461A7801321A70A9
:1006C0008CE71D46EBE700229A4B04F079FD0022EF
:1006D000002306460F4604F0DBFF00289BD0CCE742
:1006E0000A9A002A00F08B80069A012A6EDC139A7F
:1006F000002A67D003F23343079F059D059A012125
:10070000204698441A44059206F04FFB0646002DF9
:100710000CDDB8F1000F09DD45452B46059AA8BF51
:100720004346D21AED1AA8EB03080592079BEBB1DA
:100730000A9B002B67D08FB131463A46204604F021
:10074000BDF9049A01460646204606F037FB049997
:100750000890204606F087FA089B0493079BDA1B53
:1007600004D00499204604F0A9F904900121204600
:1007700006F01BFB0E9B0746002B00F0CD811A46AE
:100780000146204604F09AF9069B0746012B40DCFF
:10079000009B002B39D1019BC3F31303002B36D1EF
:1007A000019B23F000431B0D1B052BB1059B08F19A
:1007B000010801330593012307930E9B002B2AD1D7
:1007C000012030E0149BC3F1360395E7079B09F144
:1007D000FF37BB42B7BF079BDF1B0797FA1ABFBFA4
:1007E0000E9B00279B180E93B9F1000FB3BF059B1A
:1007F0004B46059DA3EB0905B8BF00237EE7079F85
:10080000059D0A9E83E7079AABE70023D4E7009B88
:10081000D2E7002307933B6907EB8303186906F0CF
:1008200076FAC0F12000404410F01F0047D0C0F11C
:100830002003042B3BDDC0F11C00059B0544034451
:1008400080440593059B002B05DD1A46049920463C
:1008500006F049FB0490B8F1000F05DD3946424629
:10086000204606F040FB07460F9B53B339460498D9
:1008700006F08DFB002824DA00230A220499204682
:1008800006F008FA0A9B0AF1FF3A0490002B00F0E8
:100890004A81002331460A22204606F0FBF9029BDA
:1008A0000646002B4EDC069B022B4BDD11E0C9D027
:1008B0001C33059A1A441D4498440592C2E7034626
:1008C000F6E7B9F1000F37DC069B022B34DDCDF8DB
:1008D0000890029B63B939460522204606F0DAF9F2
:1008E00001460746049806F052FB00283FF7CDADBD
:1008F0000B9B5D466FEA030A4FF00009394620461C
:1009000006F0B1F9002E3FF4B8AEB9F1000F05D0F2
:10091000B14503D04946204606F0A5F931462046A8
:1009200006F0A1F9A9E600273E46E1E7DDF820A0A0
:100930003E46AAE5000024400A9BCDF80890002B13
:1009400000F0F880002D05DD31462A46204606F0ED
:10095000CAFA0646079B002B4CD07168204606F069
:100960004EF93269054606F10C0102320C30920054
:1009700005F082FE01222946204606F0B4FA009BCB
:10098000B1460646CDF814B003F00103079339468B
:10099000049806F03CF84946054600F130080498F2
:1009A00006F0F5FA324600903946204606F009FB7B
:1009B000C368024603BB01460890049806F0E7FAB4
:1009C000089A034611462046089306F04CF9089B06
:1009D000A3B9069A92B9079A82B9B8F1390F29D00A
:1009E000009B002B01DD05F13108059B5D1C83F8A0
:1009F000008083E73046C2E70123E3E7009A002A3C
:100A000004DB24D1069A12BB079A02BB002BECDD53
:100A100001220499204606F066FA3946049006F051
:100A2000B6FA002803DCE0D118F0010FDDD0B8F1F0
:100A3000390FD8D1059B059A5D1C3923137015F821
:100A4000013C6A1E392B4ED00133137056E7059ACC
:100A5000002B02F1010506DDB8F1390FEAD008F1EB
:100A60000108059BC3E7A5EB0B03029A05F8018C6F
:100A7000934221D000230A220499204606F00AF965
:100A8000B14504904FF000034FF00A02494620465A
:100A900005D106F0FFF881460646059577E706F092
:100AA000F9F83146814600230A22204606F0F2F882
:100AB0000646F2E74FF0000901220499204606F0AD
:100AC00012FA3946049006F062FA0028B7DC02D127
:100AD00018F0010FB3D115F8013C6A1E302B7FF4DA
:100AE0000DAF1546F7E7934505D131230AF1010A09
:100AF0008BF8003002E71546A1E7DFF864B007E0A5
:100B0000219BDFF860B01BB10BF10803219A136041
:100B1000584617B0BDE8F08F069B012B7FF738AE23
:100B20000E9B07934CE6029B002B03DC069B022BDB
:100B30003FF7CFAE5D463946049805F068FF00F1F7
:100B40003008029A05F8018BA5EB0B039A42B1DD40
:100B500000230A220499204606F09CF80490EAE754
:100B60002D7F0100517F010010B5054C237833B96A
:100B7000044B13B1044800E000BF0123237010BDF3
:100B800028020020000000006C80010008B5034B23
:100B90001BB10349034800E000BF08BD000000008E
:100BA0002C0200206C800100154B002B08BF134B5A
:100BB0009D46A3F5803A00218B460F461348144A00
:100BC000121A05F07DFD0F4B002B00D098470E4BFD
:100BD000002B00D098470020002104000D000D4894
:100BE000002802D00C4800E000BF02F0BDFF20004A
:100BF000290000F09FF902F091FF00BF00000800FB
:100C00000000012000000000000000002002002081
:100C1000D0B90020000000000000000080B483B0C4
:100C200000AF7860034B18460C37BD465DF8047B77
:100C3000704700BF0025845090B587B004AF0023F3
:100C4000FB715E4B01225A6005F0EAF85C4B1B68B1
:100C50005B4A23F0010313605A4B1B68002B2CD016
:100C6000584B1B681C4664086400204621462246F7
:100C700023469FED550ADFED540A9FED531ADFED31
:100C8000521A9FED512ADFED502A9FED4F3ADFEDCA
:100C90004E3A9FED4D4ADFED4C4A9FED4B5ADFED4A
:100CA0004A5A9FED496ADFED486A9FED477ADFEDCA
:100CB000467A05F0A4FC0346FB71444B1B68002BED
:100CC0004CD000230093012301220821404804F066
:100CD0009FFD012303930B2302930A230193072310
:100CE00000930123082245214FF4E13001F04AFD31
:100CF000384802F045FE374802F042FE354802F01F
:100D00003FFE354802F03CFE2E4B1B681946334827
:100D100002F036FE324B1B881946324802F030FE94
:100D2000314B1B781946314802F02AFE304B1B78B4
:100D30001946304802F024FE2F4B1B6819462F48F5
:100D400002F01EFE2E4802F01BFE2E4802F018FE96
:100D50002D4802F015FE2C4802F012FE00233B60E5
:100D600010E00F2004F081FD4FF4FA7005F065F8F3
:100D7000164B1B68002B02D0244802F001FE3B6892
:100D800001333B603B68092BEBDDFB79002B07D07F
:100D90000E4B1B68002B02D01D4802F0F1FDFEE750
:100DA0000A4B1B68002B02D01A4802F0E9FD05F03F
:100DB000DDF800BF0C37BD4690BD00BF00400140CC
:100DC00010E000E0440200200000000038B90020DC
:100DD000003000507074010090740100BC74010078
:100DE0002AED00E0CC74010029ED00E0DC74010084
:100DF00028ED00E0EC7401002CED00E0FC74010033
:100E00000C750100387501005875010078750100F6
:100E100080750100A075010080B483B000AF7860D8
:100E2000034B18460C37BD465DF8047B704700BF86
:100E30000025845080B483B000AF0346FB71054A9F
:100E4000FB79C2F80C3500BF0C37BD465DF8047B5A
:100E5000704700BF0080014080B483B000AF78606D
:100E6000044A7B68C2F8043500BF0C37BD465DF804
:100E7000047B70470080014080B483B000AF03461C
:100E8000FB71084BD3F80825FB79012101FA03F324
:100E900004491343C1F8083500BF0C37BD465DF85F
:100EA000047B70470080014080B483B000AF0346EC
:100EB000FB71064AFB7903F5C073054942F823101C
:100EC00000BF0C37BD465DF8047B704700800140D1
:100ED0003546526E80B500AF0E4802F023FD0E4835
:100EE00002F020FD0D4B0E4A0E490F4802F01AFD8C
:100EF000002005F02DF801464FF05023D3F80034C0
:100F00001A460A4802F00EFD094802F00BFD00BF28
:100F100080BD00BFC0750100C475010018760100D6
:100F20001C760100247601003C7601005476010015
:100F30007076010080B584B004AF04F01EFF0F206E
:100F400004F0DCFC00210F2004F029FD324800F001
:100F50006BFE05F053FA314B0122C3F878250123CB
:100F600003930B2302930A23019307230093012386
:100F7000082245214FF4E13001F004FC284B294AB6
:100F80001A60294B274A1A60FFF7A4FF274802F08E
:100F9000C9FC274802F0C6FCC82226494FF48060ED
:100FA00001F006F92349244802F0BCFCC822234979
:100FB0004FF4484001F0FCF82049214802F0B2FC0F
:100FC000C82220494FF4423001F0F2F81D491E4872
:100FD00002F0A8FC05F022FA01F096FD1B4802F091
:100FE000A1FC01F00FFC00210F2004F099FC01F09E
:100FF00061FC0920FFF71EFF4FF4C030FFF72CFF04
:101000000020FFF739FF0020FFF74EFF4FF441307B
:1010100000F01EF8FEE700BF390C01000040005050
:1010200034B900201928010038B90020C475010026
:101030009076010048020020AC76010010030020E9
:10104000B4760100D8030020BC760100C47601000C
:1010500090B585B000AF78607B681B6883F38888A3
:101060007B6804331B68FB60FB681C4664086400F3
:1010700020462146224623469FED120ADFED110A43
:101080009FED101ADFED0F1A9FED0E2ADFED0D2AEE
:101090009FED0C3ADFED0B3A9FED0A4ADFED094A6E
:1010A0009FED085ADFED075A9FED066ADFED056AEE
:1010B0009FED047ADFED037A05F0A1FA00BF143743
:1010C000BD4690BD0000000080B584B000AF7860E0
:1010D000396012223968786802F08EFCF860FB688B
:1010E000002B26D02F4B0122C3F8002501F09CFDD8
:1010F000034683F00103DBB2002B08D001F08AFD28
:101100000346002B01D001F077FD01F053FD0023D1
:10111000BB6007F108031A463968F86801F08EFDD4
:101120000346002B05D1BB683A689A4201D10123DE
:1011300000E0002318461037BD46BDE880407146E8
:1011400072467346B7EE000AF7EE000AB7EE001AD1
:10115000F7EE001AB7EE002AF7EE002AB7EE003AD3
:10116000F7EE003AB7EE004AF7EE004AB7EE005A43
:10117000F7EE005AB7EE006AF7EE006AB7EE007AB3
:10118000F7EE007A8EF3008C10B4F1EE10CA4FF631
:101190006074C0F6FF740CEA040CE1EE10CA10BCD7
:1011A000F44674470000845080B586B000AF034613
:1011B000B9607A60FB7312227968B86802F01CFC8F
:1011C00078617B69002B15D0FB7B002B10D0FB7B5B
:1011D000032B0DD8FB7B013BC82202FB03F3224A01
:1011E00013447A681946786905F0AFFB012302E0E1
:1011F000002300E0002318461837BD46BDE88040B4
:10120000714672467346B7EE000AF7EE000AB7EE73
:10121000001AF7EE001AB7EE002AF7EE002AB7EE32
:10122000003AF7EE003AB7EE004AF7EE004AB7EEA2
:10123000005AF7EE005AB7EE006AF7EE006AB7EE12
:10124000007AF7EE007A8EF3008C10B4F1EE10CA3B
:101250004FF66074C0F6FF740CEA040CE1EE10CA9D
:1012600010BCF446744700BF4802002080B500AFB0
:1012700001F0D0FC0346002B01D001F0BDFC1E4B59
:101280000022C3F8002500BFBD46BDE8804070467F
:10129000714672467346B7EE000AF7EE000AB7EEE3
:1012A000001AF7EE001AB7EE002AF7EE002AB7EEA2
:1012B000003AF7EE003AB7EE004AF7EE004AB7EE12
:1012C000005AF7EE005AB7EE006AF7EE006AB7EE82
:1012D000007AF7EE007A8EF3008C10B4F1EE10CAAB
:1012E0004FF66074C0F6FF740CEA040CE1EE10CA0D
:1012F00010BCF446744700BF0000845080B582B033
:1013000000AF786012220421786802F075FB034672
:101310007B607B68002B01D1002303E01D4A7B68C2
:101320001360012318460837BD46BDE8804071466A
:1013300072467346B7EE000AF7EE000AB7EE001ADF
:10134000F7EE001AB7EE002AF7EE002AB7EE003AE1
:10135000F7EE003AB7EE004AF7EE004AB7EE005A51
:10136000F7EE005AB7EE006AF7EE006AB7EE007AC1
:10137000F7EE007A8EF3008C10B4F1EE10CA4FF63F
:101380006074C0F6FF740CEA040CE1EE10CA10BCE5
:10139000F44674474402002080B588B000AF7860FE
:1013A00039607A683B681344103BFB617A683B689C
:1013B0001344183BBB61BB697B617B69083B3B61A4
:1013C0003B69083BFB603B691B78012B05D1FB683F
:1013D0001B7803F00703022B01D0012320E0FB69F7
:1013E00010221149184605F038F90346002B01D0A8
:1013F000002315E07B691B78012B01D101230FE04D
:101400007B691B78FF2B0AD10123FB7207F10B01CB
:1014100005230122B86904F061FD034600E00023C2
:1014200018462037BD4680BDE076010080B588B003
:1014300002AF00237B610BE07B69D9B200230093EC
:10144000072301224C4804F0D9FA7B6901337B6100
:101450007B69042BF0DD06233B610BE03B69D9B2CD
:101460000023009307230022434804F0C7FA3B6996
:1014700001333B613B69102BF0DD404B0122C3F887
:1014800084254FF4E0314FF44040FFF785FF0346D9
:10149000002B0AD04FF4B0214FF44030FFF77CFF0F
:1014A0000346002B01D0012300E00023FB71FB79F0
:1014B00003F00103FB71314B0022C3F8842506239E
:1014C000FB600BE0FB68D9B20023009305230022E8
:1014D000294804F093FAFB680133FB60FB68102B8A
:1014E000F0DD0023BB600BE0BB68D9B200230093A2
:1014F00005230122204804F081FABB680133BB6058
:10150000BB68042BF0DDFB7918461837BD46BDE8F3
:101510008040714672467346B7EE000AF7EE000A45
:10152000B7EE001AF7EE001AB7EE002AF7EE002A1F
:10153000B7EE003AF7EE003AB7EE004AF7EE004A8F
:10154000B7EE005AF7EE005AB7EE006AF7EE006AFF
:10155000B7EE007AF7EE007A8EF3008C10B4F1EE5D
:1015600010CA4FF66074C0F6FF740CEA040CE1EE8A
:1015700010CA10BCF446744700300050009003506D
:1015800080B485B000AF4FF43443BB60274BFB60A1
:10159000FB6803F00703002B0CD0FB680733FB60EC
:1015A000FB6823F00703FB60BA68FB68D31A1F4A85
:1015B0001344BB60FB687B601D4A7B6813601C4B57
:1015C00000225A607B68BA681344FB600822FB68FB
:1015D0009B1AFB60FB6823F00703FB60FB68154A5E
:1015E0001360144B1B6800225A60124B1B680022C8
:1015F0001A607B683B603B68FA68D21A3B685A60A5
:101600000C4B1A683B681A603B685B680A4A1360B7
:101610003B685B68094A1360094B4FF000421A604F
:1016200000BF1437BD465DF8047B7047A00400205E
:10163000A0B80020A8B80020B0B80020ACB80020A6
:10164000B4B8002080B485B000AF7860284BFB6050
:1016500002E0FB681B68FB60FB681B687A689A42C3
:10166000F7D8FB68BB60FB685B68BA6813447A68AC
:101670009A4208D1FB685A687B685B681A44FB6829
:101680005A60FB687B607B68BB607B685B68BA689C
:101690001A44FB681B689A4218D1FB681A68154BFC
:1016A0001B689A420DD07B685A68FB681B685B68B0
:1016B0001A447B685A60FB681B681A687B681A606A
:1016C00008E00C4B1A687B681A6003E0FB681A6834
:1016D0007B681A60FA687B689A4202D0FB687A6875
:1016E0001A6000BF1437BD465DF8047B704700BF29
:1016F000A0B80020A8B8002080B586B000AF786000
:101700000023FB60514B1B68002B01D1FFF738FF12
:101710004F4B1A687B681340002B40F086807B6833
:10172000002B19D008227B6813447B607B6803F090
:101730000703002B10D07B6823F0070308337B607E
:101740007B6803F00703002B06D0012383F3108886
:10175000012383F39088FEE77B68002B65D03D4B27
:101760001B687A689A4260D83B4B3B613A4B1B68D6
:101770007B6104E07B693B617B691B687B617B6902
:101780005B687A689A4203D97B691B68002BF1D1A8
:101790002E4B1B687A699A4247D03B691B68082226
:1017A0001344FB607B691A683B691A607B695A685D
:1017B0007B68D21A08235B009A421BD97A697B683E
:1017C0001344BB60BB6803F00703002B06D0012362
:1017D00083F31088012383F39088FEE77B695A68BE
:1017E0007B68D21ABB685A607B697A685A60B868AD
:1017F000FFF728FF174B1A687B695B68D31A154AF5
:101800001360144B1A68154B1B689A4203D2114B94
:101810001B68124A13607B695A680D4B1B681A4398
:101820007B695A607B6900221A60FB6803F007033A
:10183000002B06D0012383F31088012383F39088C3
:10184000FEE7FB6818461837BD4680BDA8B80020E3
:10185000B4B80020ACB80020A0B80020B0B8002078
:1018600080B584B000AF78607B68FB607B68002B3C
:1018700042D008235B42FA681344FB60FB68BB60FC
:10188000BB685A681E4B1B681340002B06D101230E
:1018900083F31088012383F39088FEE7BB681B68FD
:1018A000002B06D0012383F31088012383F3908853
:1018B000FEE7BB685A68124B1B681340002B1BD015
:1018C000BB681B68002B17D1BB685A680C4B1B68A0
:1018D000DB431A40BB685A60012383F39088BB68DE
:1018E0005A68084B1B681344064A1360B868FFF730
:1018F000A9FE002383F3908800BF1037BD4680BD4A
:10190000B4B80020ACB8002080B483B000AFEFF3CF
:1019100005837B607B68002B08D0214B1B689BB242
:101920001F4A43F0BF6343F41033136000BF0C370A
:10193000BD465DF8047B7046714672467346B7EE4D
:10194000000AF7EE000AB7EE001AF7EE001AB7EE3B
:10195000002AF7EE002AB7EE003AF7EE003AB7EEAB
:10196000004AF7EE004AB7EE005AF7EE005AB7EE1B
:10197000006AF7EE006AB7EE007AF7EE007A8EF3AF
:10198000008C10B4F1EE10CA4FF66074C0F6FF740C
:101990000CEA040CE1EE10CA10BCF446744700BF18
:1019A0000CED00E080B483B000AFEFF305837B6003
:1019B0007B68002B11D0254B1B68244A43F44063FD
:1019C0001360234B1B68224A23F000531360204B03
:1019D0001B681F4A43F08063136000BF0C37BD468D
:1019E0005DF8047B7046714672467346B7EE000A96
:1019F000F7EE000AB7EE001AF7EE001AB7EE002A6B
:101A0000F7EE002AB7EE003AF7EE003AB7EE004ADA
:101A1000F7EE004AB7EE005AF7EE005AB7EE006A4A
:101A2000F7EE006AB7EE007AF7EE007A8EF3008CDC
:101A300010B4F1EE10CA4FF66074C0F6FF740CEAF1
:101A4000040CE1EE10CA10BCF44674478CED00E0C3
:101A500034EF00E080B483B000AF7860034B1846E9
:101A60000C37BD465DF8047B704700BF00258450ED
:101A700080B588B004AF7860344B1B68334A23F0DC
:101A800001031360324B1B68002B3AD000230093F4
:101A90000123012208212F4804F095F90123039323
:101AA0000B2302930A2301930723009301230822A7
:101AB00045214FF4E13000F065FE274801F060FF5A
:101AC000254801F05DFF244801F05AFF234B1B8895
:101AD0001946234801F054FF224B1B78194622482F
:101AE00001F04EFF214B1B781946214801F048FFB9
:101AF000204B1B681946204801F042FF786801F02E
:101B00003FFF1E4801F03CFF1D4801F039FF1C4813
:101B100001F036FF0023FB600CE0182004F033F9DD
:101B20004FF4FA7004F089F9164801F029FFFB68B8
:101B30000133FB60FB68092BEFDD134801F020FF48
:101B400004F014FA00BF1037BD4680BD10E000E07D
:101B500038B9002000300050F07601002AED00E096
:101B60001477010029ED00E02477010028ED00E062
:101B7000347701002CED00E0447701005477010038
:101B800074770100947701009C77010080B500AF65
:101B90000248FFF76DFF00BF80BD00BFBC770100AA
:101BA00080B500AF0248FFF763FF00BF80BD00BFF4
:101BB000C877010080B500AF0248FFF759FF00BFAA
:101BC00080BD00BFE477010080B500AF0248FFF799
:101BD0004FFF00BF80BD00BFF877010080B500AFA8
:101BE0000248FFF745FF00BF80BD00BF0C78010031
:101BF00080B500AF0248FFF73BFF00BF80BD00BFCC
:101C00002078010080B500AF054B1B68002B02D087
:101C1000034B1B6898470348FFF72AFF00BF80BDAE
:101C2000B8B800203478010080B483B000AF786089
:101C3000044A7B68136000BF0C37BD465DF8047B27
:101C4000704700BFB8B8002080B500AF0248FFF76A
:101C50000FFF00BF80BD00BF4878010080B500AF16
:101C60000248FFF705FF00BF80BD00BF54780100A8
:101C700080B500AF0248FFF7FBFE00BF80BD00BF8C
:101C80006478010080B500AF0248FFF7F1FE00BFA5
:101C900080BD00BF7478010080B500AF0248FFF737
:101CA000E7FE00BF80BD00BF8478010080B500AFB3
:101CB0000248FFF7DDFE00BF80BD00BF9478010041
:101CC00080B500AF0248FFF7D3FE00BF80BD00BF64
:101CD000A478010080B500AF0248FFF7C9FE00BF3D
:101CE00080BD00BFB478010080B500AF0248FFF7A7
:101CF000BFFE00BF80BD00BFC478010080B500AF4B
:101D00000248FFF7B5FE00BF80BD00BFDC780100D0
:101D100080B500AF0248FFF7ABFE00BF80BD00BF3B
:101D2000F078010080B500AF0248FFF7A1FE00BFC8
:101D300080BD00BF0479010080B500AF0248FFF705
:101D400097FE00BF80BD00BF1879010080B500AFCD
:101D50000248FFF78DFE00BF80BD00BF2C79010057
:101D600080B500AF0248FFF783FE00BF80BD00BF13
:101D70004079010080B500AF0248FFF779FE00BF4F
:101D800080BD00BF5079010080B500AF0248FFF769
:101D90006FFE00BF80BD00BF6079010080B500AF5D
:101DA0000248FFF765FE00BF80BD00BF70790100EB
:101DB00080B500AF0248FFF75BFE00BF80BD00BFEB
:101DC0008079010080B500AF0248FFF751FE00BFE7
:101DD00080BD00BF9079010080B500AF0248FFF7D9
:101DE00047FE00BF80BD00BFA079010080B500AFF5
:101DF0000248FFF73DFE00BF80BD00BFB079010083
:101E000080B500AF0248FFF733FE00BF80BD00BFC2
:101E1000C079010080B500AF0248FFF729FE00BF7E
:101E200080BD00BFD079010080B500AF0248FFF748
:101E30001FFE00BF80BD00BFE079010080B500AF8C
:101E40000248FFF715FE00BF80BD00BFF07901001A
:101E500080B500AF0248FFF70BFE00BF80BD00BF9A
:101E6000007A010080B500AF0248FFF701FE00BF15
:101E700080BD00BF107A01000649074A074B9B1A34
:101E800003DD043BC858D050FBDC00F02BF8FEF714
:101E90008BFE00007880010000000020200200205E
:101EA00080B400AFBFF34F8F054BDB6803F4E062F3
:101EB0000349044B1343CB60BFF34F8F00BFFDE7D3
:101EC00000ED00E00400FA0580B400AF034B044AC3
:101ED0001A6000BFBD465DF8047B7047000000201B
:101EE0000090D00380B582B000AF5E4B1B685D4AA6
:101EF00043F00203136000237B6000237B6011E04A
:101F00004FF47F024FF47F017B68603351F8333028
:101F100019467B686033DB0013445B680B607B68A9
:101F200001337B607B68FF2B08D84FF47F027B680E
:101F3000603352F83330B3F1FF3FE1D100F0B2F833
:101F40000346002B04D100F09BF80346002B3FD042
:101F500000BF454BD3F80034012BFAD1424B01228C
:101F6000C3F8042500BF404BD3F80034012BFAD14D
:101F700000F098F80346002B0BD03C4BDB693B4A42
:101F800023F00103D36100BF374BD3F80034012B9A
:101F9000FAD100F075F80346002B0DD0334B1B6AC5
:101FA00023F0FF03314A43F02003136200BF2E4B9E
:101FB000D3F80034012BFAD12B4B0022C3F80425AF
:101FC00000BF294BD3F80034012BFAD1FFF768FF8B
:101FD00000F07AF80346002B09D04FF0502300227E
:101FE000C3F814214FF050230022C3F8182100F049
:101FF00087F80346002B06D01D4B01221A601D4BAB
:102000000122C3F8782500F091F80346002B06D092
:10201000174B00221A60174B0122C3F8782500F0F5
:102020009BF80346002B02D0134B0C221A60134B73
:10203000D3F88C30114A43F44063C2F88C300F4B14
:10204000D3F888300D4A43F47003C2F88830BFF3E8
:102050004F8FBFF36F8FFFF737FF00BF0837BD46C5
:1020600080BD00BFD0ED00E0009003500080FF0075
:10207000384A005000400050E4AE035000ED00E04C
:1020800080B400AF064B1B6AB3F1FF3F01D10123BF
:1020900000E000231846BD465DF8047B704700BF92
:1020A0000080FF0080B400AF064BDB6903F0010342
:1020B000002B01D0012300E000231846BD465DF847
:1020C000047B70470080FF0080B400AF0A4B1B68A0
:1020D000092B0BD1094B1B68012B01D1012306E011
:1020E000064B1B68022B01D1012300E00023184698
:1020F000BD465DF8047B70473001FF003401FF00EE
:1021000080B400AF074B1B68092B05D1064B1B6839
:10211000012B01D1012300E000231846BD465DF8E4
:10212000047B70473001FF003401FF0080B400AF32
:10213000074B1B68092B05D1064B1B68022B01D1ED
:10214000012300E000231846BD465DF8047B70477C
:102150003001FF003401FF0080B400AF074B1B6863
:10216000092B05D1064B1B68022B01D1012300E08E
:1021700000231846BD465DF8047B70473001FF0020
:102180003401FF000022044B1A601A68824200D317
:1021900070471A680132F7E7BCB8002080B500AF7D
:1021A000024803F05AFE0346184680BD00900350D3
:1021B00080B5BAB000AFF860B9607A6007F1140377
:1021C000C8220021184604F07BFA7A680021B8681A
:1021D00004F076FA07F11403C7221946F86803F0F1
:1021E00057FE07F114032149184604F0C3FBC7F852
:1021F000E400D7F8E430002B01D1002331E0D7F818
:10220000E4300D33C7F8E43007F1140318491846D9
:1022100004F0B0FBC7F8E000D7F8E030002B01D1A4
:1022200000231EE0D7F8E020D7F8E4309A4201D826
:10223000002316E0D7F8E020D7F8E430D31AC7F827
:10224000DC307B68013BD7F8DC209A4201D90023BF
:1022500007E0D7F8DC20D7F8E410B86804F00CFAEF
:1022600001231846E837BD4680BD00BF287A01002B
:10227000387A010080B582B000AF00237B6024E093
:10228000154A7B68403352F82330002B1AD0124A8B
:102290007B684033002142F82310104A7B6852F8D3
:1022A0002330002B0ED00D4A7B6852F823300A49A8
:1022B0007A6802F5A27251F82220120C02F0030291
:1022C000104698477B6801337B607B68072BD7DD1E
:1022D00000BF0837BD4680BD00100340C0B80020D5
:1022E00080B400AFBFF34F8F054BDB6803F4E062AF
:1022F0000349044B1343CB60BFF34F8F00BFFDE78F
:1023000000ED00E00400FA0580B400AF0D4B1B782F
:1023100083F00103DBB2002B0DD04FF05023D3F834
:102320000034094A13604FF050230022C3F8002400
:10233000044B01221A70044B1B681846BD465DF819
:10234000047B7047C8B90020E0B8002080B582B097
:1023500000AF786039603B68002B04D0FFF7D4FFF2
:1023600002463B681A60FFF7CFFF0346042B22D0DA
:10237000042B06D8012B16D0012B12D3022B14D01C
:102380001FE0B3F5803F12D0B3F5803F02D8102B89
:1023900013D016E0B3F1011F11D0B3F5003F08D000
:1023A0000FE00A4B0EE00A4B0CE00A4B0AE00A4B26
:1023B00008E00A4B06E00A4B04E00A4B02E00A4B35
:1023C00000E00A4B18460837BD4680BD487A010038
:1023D0005C7A0100747A0100887A0100987A010021
:1023E000B87A0100E87A0100087B0100307B010027
:1023F00098B500AF4FF48271314803F0CAFD03462F
:10240000002B0DD02F4BD3E900124B1C42F10004DE
:102410002C4AC2E900344FF48271294803F0C9FD07
:102420004FF4A071264803F0B4FD0346002B10D0F2
:102430004FF4A071224803F09DFD4FF4A071204895
:1024400003F0B7FD204B1B68002B02D01E4B1B680E
:1024500098474FF480711A4803F09BFD0346002B08
:1024600004D04FF48071164803F0A3FD4FF4A2711D
:10247000134803F08EFD0346002B04D04FF4A271E5
:102480000F4803F096FD4FF4A4710D4803F081FD51
:102490000346002B04D04FF4A471094803F089FDD2
:1024A0004FF4A671064803F074FD0346002B04D0D8
:1024B0004FF4A671024803F07CFD00BF98BD00BF39
:1024C0000050014020020020E4B8002080B483B016
:1024D00000AF7860034B18460C37BD465DF8047BAF
:1024E000704700BF0025845080B483B000AF78608F
:1024F0007B68B3F5964F1FD0B3F5964F09D8B3F567
:10250000965F1DD0B3F5165F18D0B3F5166F19D0CE
:102510001BE0B3F5614F09D0B3F5E13F03D0B3F54C
:10252000164F06D011E04FF0EB730FE04FF46B0342
:102530000CE04FF41D0309E0074B07E0074B05E0F3
:10254000074B03E04FF41D2300E0002318460C372F
:10255000BD465DF8047B704700A04E000050270088
:1025600000B0130080B582B000AF78607B685B7DFF
:10257000002B05D1074B084A4621084801F0B0FA64
:102580007B681B680022C3F8002500BF0837BD46E2
:1025900080BD00BFE47B0100907C0100F07B010066
:1025A00090B589B002AFF860B96011461A460B4683
:1025B000FB711346BB7100237B61F868FFF7D2FF04
:1025C000BB79082B08D0BB79072B05D0404B414A7B
:1025D0005021414801F084FABB79072B08D1FB79DF
:1025E000452B05D03D4B3B4A54213B4801F078FA3E
:1025F000BB79072B06D1FB79452B03D1FB68012260
:102600009A7502E0FB6800229A75BB79082B06D107
:10261000FB79452B03D17B6943F00E037B6197F86F
:102620002830022B03D17B6943F010037B61FB68E8
:102630001B687A69C3F86C25386B03F0FBFC002338
:10264000019300230093032300220121386B03F040
:10265000C8FCFB681C68B868FFF746FF0346C4F86F
:102660002435FB681B683A6BC3F80C2500230193E3
:1026700000230093032300220021786B03F0B1FCB8
:10268000FB681B687A6BC3F81425FB6803F108022A
:10269000FB681B68C3F83425FB681B680122C3F87C
:1026A0003825FB681B680022C3F81021FB681B68F3
:1026B0000022C3F8442197F82C20FB681A61FB68BC
:1026C0001B680822C3F8002500BF1C37BD4690BD1B
:1026D0003C7C0100A07C0100F07B01005C7C0100DF
:1026E00080B584B000AFF860B9607A60FB685B7D4C
:1026F000002B05D11B4B1C4AE9211C4801F0F0F9C5
:10270000FB689B7D002B06D001237A68B968F868C6
:1027100003F0EFFC23E0BB68B3F5801F05D2002374
:102720007A68B968F86803F0E4FCFB681B68BA686B
:10273000C3F84425FB681B687A68C3F84825FB6822
:102740001B680022C3F82021FB681B6801229A60E5
:1027500000BFFB681B68D3F82031012BF9D110377B
:10276000BD4680BDE47B0100AC7C0100F07B010034
:1027700080B500AF024803F04BFD00BF80BD00BF35
:10278000E8B8002080B586B004AF786008461146EE
:102790001A460346FB700B46BB7013467B703B7FAB
:1027A000002B06D0124B134A1A60114B124A5A6082
:1027B00005E00F4B114A1A600D4B114A5A600C4B41
:1027C00008221A750A4B01225A75B978FA78BB6942
:1027D00003937B6902933B7C01937B7800930B46C8
:1027E00079680348FFF7DCFE00BF0837BD4680BDAF
:1027F000E8B8002000800050002584500080004090
:102800000025844080B500AF0248FFF7ABFE00BF53
:1028100080BD00BFE8B8002080B582B000AF78600E
:102820007968034803F0E2FC00BF0837BD4680BD6D
:10283000E8B8002080B500AF024803F0E9FC00BF13
:1028400080BD00BF00B9002080B483B000AF034654
:10285000FB7197F90730002B22DB154A97F90730F7
:102860005B09A03352F82310FB7903F01F03012208
:102870009A400F4897F907305B090A43A03340F8A4
:1028800023200B4A97F907305B09A03352F8232025
:10289000FB7903F01F0322FA03F303F0010300E0C6
:1028A000002318460C37BD465DF8047B704700BF17
:1028B00000E100E080B588B002AF00237B610BE04F
:1028C0007B69D9B200230093052301228D4803F0D0
:1028D0001EFD7B6901337B617B69042BF0DD0123E5
:1028E0000093012306220021864803F0E0FC012327
:1028F0000093062301220521824803F008FD0623E8
:102900003B610BE03B69D9B2002300930523002211
:102910007C4803F0FCFC3B6901333B613B69102BB5
:10292000F0DD1123FB600BE0FB68D9B201230093BB
:1029300006230022734803F0EAFCFB680133FB60C6
:10294000FB681F2BF0DD0023BB600BE0BB68D9B236
:1029500001230093062301226A4803F0FDFCBB68B3
:102960000133BB60BB68072BF0DD08237B600BE005
:102970007B68D9B20123009306230022614803F04B
:10298000EBFC7B6801337B607B681F2BF0DD012350
:1029900000930023002242215A4803F002FD012344
:1029A00000220021574803F062FC0123009300231A
:1029B00000220521534803F0F4FC00230093002378
:1029C000002208214F4803F0ECFC01230093002370
:1029D000002209214B4803F0E4FC0123009300236B
:1029E00000221B21474803F0DCFC01230093002355
:1029F00000221C21434803F0D4FC01230093002350
:102A000000221D213F4803F0CCFC0123009300234A
:102A100000222A213B4803F0C4FC01230093002339
:102A200000220521374803F0BCFC0123009300235A
:102A300000223121334803F0B4FC0123009300232A
:102A4000002239212F4803F0ACFC0123009300231E
:102A500000223A212B4803F0A4FC01230093002319
:102A600000221521274803F09CFC0123009300233A
:102A700000221421234803F094FC01230093002337
:102A800000220E211F4803F08CFC01230093002339
:102A900000220F211B4803F084FC01230093002334
:102AA00000221021174803F07CFC0123009300232F
:102AB00000221121134803F074FC0123009300232A
:102AC00000220B210F4803F06CFC0123009300232C
:102AD00000220A210B4803F064FC01230093002329
:102AE00000221721074803F05CFC01230093002318
:102AF00000221821034803F054FC00BF1837BD46DC
:102B000080BD00BF0030005080B483B000AF002310
:102B10007B604FF441333B603B6823F0604323F01C
:102B20007F030B497A6813438B604FF444433B6047
:102B30003B6823F0604323F07F0306497A68134320
:102B40008B6000BF0C37BD465DF8047B704700BF4B
:102B500000ED02E000ED00E080B500AF002102488A
:102B600003F096FC00BF80BD0090035080B500AF1D
:102B70000121024803F08CFC00BF80BD009003508F
:102B800080B582B000AF7860396000BF084803F0BC
:102B90006BFC034683F00103DBB2002BF6D17B68AC
:102BA0003A681A60BFF35F8F00BF0837BD4680BD2B
:102BB0000090035010B50C4C236813B10B4B1B68ED
:102BC0006BB900F0CBF838B10138062896BF084B36
:102BD000084853F8200010BD0122044B1A6001235D
:102BE0000020236010BD00BF18B900201CB90020D0
:102BF000B87C0100FE8FFFFF08B500F047F8002306
:102C00000249034A0B601360184608BD18B900203A
:102C10001CB90020034B1868A0F10100B0FA80F045
:102C20004009704718B90020034B1868A0F1010053
:102C3000B0FA80F0400970471CB9002090292DE9B6
:102C4000F0410C460746164617D9002503E03368C5
:102C5000E41A1D440ED0902C2246334628BF902201
:102C60007919002000F09EFC0028F0D0002333608A
:102C7000BDE8F0813560BDE8F0811346BDE8F04164
:102C80000A460146002000F08DBC00BF10B500F0E0
:102C9000A9F800280CBF0024032400F0EDF820461A
:102CA00010BD00BF30B5ADF5157D4FF408720021A1
:102CB0000CA803F005FD002302A819462822019361
:102CC00003F0FEFC02A800F0C5FC18B105200DF5CC
:102CD000157D30BD1C4D4FF0FF31286800F016F90E
:102CE0000446F0B9002000F041F9B0B90CAA02A9DD
:102CF00001A800F049FC0446012000F037F9F0B9C2
:102D0000286800F00BF910B1104800F0F3FC2046E1
:102D1000002CDBD10DF5157D30BD0D4800F0EAFC2F
:102D2000E4E70C4800F0E6FC012CDBD1286800F059
:102D3000F5F80028CAD0054800F0DCFCC6E70648D4
:102D400000F0D8FCDCE700BF14000020EC7C0100A0
:102D5000047D0100D47C0100247D010008B500F051
:102D60003FF818B100F088F8032008BD00F056F8CD
:102D700068B900F0FBF860B9154B1B681B0EF02B0F
:102D800012D000F02FF800F077F8062008BD0420DC
:102D900008BD00F027F800F06FF8FFF783FF002868
:102DA0000CBF0020052008BD0A4A0B4B12689A424E
:102DB00005D000F017F800F05FF8072008BD0120EB
:102DC00000F0D4F80028E4D1044B1860E5E700BF18
:102DD00028198450241A84500000E0200C1A8450D2
:102DE0000020704700207047430503D54FF0FF32A5
:102DF000024B1A60024B1860704700BF08118450E4
:102E0000081A8450014B1860704700BF041A8450A0
:102E100008B100F04FB84FF47500704710B5114875
:102E200000F060F800B110BD0F4800F05BF800281A
:102E3000F9D10E4C204600F055F80028F3D10C4B88
:102E40000C481C6000F04EF801460028EBD100F061
:102E50002DF8044608B1204610BD00F069F8204660
:102E6000FAE700BF10000020040000200C00002042
:102E7000140000200800002008B5084800F03CF8C5
:102E8000074800F039F8074800F036F8064800F027
:102E900033F8BDE8084000F00BB800BF1000002078
:102EA000040000200C0000200800002000207047D3
:102EB000704700BF0246074803681342FCD021B1A7
:102EC000054B06481B680B600360054B00201A6029
:102ED000704700BF001A84500411845008118450B8
:102EE000081A845008B5034B02681B68106898479D
:102EF000002008BD2000002008B5034B02685B6875
:102F000010689847002008BD200000200268024B8E
:102F100010689B68184700BF2000002008B5034BCD
:102F20000268DB6810689847002008BD2000002078
:102F300070B5094C094D2069AB68984718B1084B2A
:102F400008485B6898470021074AEB6811602069D0
:102F5000BDE87040184700BF30000020200000206E
:102F600018000020447D010020B9002070B5144CE9
:102F7000144D0646AB6820699847F0B9124A1368A9
:102F80005EB91BB901201149C1F800050133136076
:102F9000EB6820699847002070BD002BF8D0012B0A
:102FA00008BF0A4903F1FF3308BFC1F800052069D3
:102FB0001360EB6898470020EEE7054870BD00BF3E
:102FC000300000202000002020B9002000008450A4
:102FD000E98FFFFFA8B32DE9F0414C1EB4F5047F43
:102FE0002CD25BB352B34FF0000CC900E6466546E5
:102FF00064464F1E03F1FF380CE0AB4216D08E45FD
:1030000001D10CF1010CA84516D00134BC4205F1E8
:10301000010518D8610950F8211004F01F06F1408D
:103020001F2E18BF01F00101002CE6D10025A84594
:103030008E464FF0010CE8D16245E6D20348BDE868
:10304000F081024870470020BDE8F081370CF100A4
:103050002DE9F04F8FB00D46DDE919418346002977
:1030600057D12969039100211C60189B1960002A1F
:1030700000F02281814A824B11686A6A1B689A4279
:1030800057D10A2955D19BF803300693039904239D
:1030900008467C4A0293A2FB00029208CB0002EB96
:1030A000420204F10800A1EB4202013BDFF8D0919B
:1030B000DFF800A2049000920593189B039C1C600B
:1030C000002C00F0CC800026049F00F013FC0023AD
:1030D0000793069BBBF1000F3AD0002D34D053BBB1
:1030E0005B000693BBF1000F36D0002D34D0E3B166
:1030F00006A9284600F0EEFB002800F07D81624B17
:10310000984212D0009000F0F5FB00980FB0BDE897
:10311000F08F4FF47F01D1F80C0C01300CBF4FF44D
:103120000471D1F80C1C03919DE72B6A73B95648C2
:10313000E8E75648E6E706A9284600F0CBFB68B169
:10314000534B9842DED0069B082BC9D15148D9E792
:10315000082BFBD05B0006934F48D3E7294606981F
:1031600000F09AFB0028EBD1069B082B00F00E81A3
:10317000042B00F03181A3F10203B3FA83F35B095E
:10318000019301231946454A136042F8843C434B9E
:1031900019606B6AC9F80030D9F800206B6A9A424E
:1031A000F5D14FF000084FF0FF30CAF80080FFF76C
:1031B0001BFE3B4A3B4B40461A60FFF723FE0A22A8
:1031C000019839492D4B08601A602A69A8F15538D1
:1031D000A8FB02126B6A120903EB4303DB0303FB38
:1031E00002F3324A9B0913600123CAF800300699A2
:1031F000DBF800200B0243EA016322F07F42134315
:10320000CBF8003007A800F037FB002898D1284BF6
:10321000A8FB04281A681433089253F8102CB6EB54
:10322000980F099253F80C2C0A9253F8082C0B9221
:1032300053F8042C0C921B680D9301D1009B9BB991
:103240003846182208A900F08BFA183C18370136C6
:10325000002C7FF43AAF049B002B40F09A800023AF
:10326000189A1360069B6FE71A46384608A9E41AB5
:1032700000F076FA009B1F44E9E700BF3811845044
:1032800030118450ABAAAAAA310CF100300CF10025
:10329000020CF100320CF100350CF100C411845025
:1032A000FEFFFF0F001184500C118450D811845080
:1032B000141184502C118450BBF1000F3FF44CAF1B
:1032C000002D3FF449AF01230EA941F8203DCBF872
:1032D0000020284600F0FEFA00287FF413AF2946AC
:1032E000069800F0D9FA00287FF40CAF069F082F4B
:1032F00000F0EB80042F00F0EA80A7F10207B7FA94
:1033000087F77F0901221646734B74491A601846E5
:103310000A60943B06606A6A1A6019686A6A914298
:10332000F8D14FF000086E4B4FF0FF30C3F800802B
:10333000FFF75AFD6B4B6C4A40461A60FFF762FD7F
:103340000A226A496A4B0F601A601A992B6901298F
:103350006A6A00F0B1806749A1FB03131B090121D0
:1033600002EB4202D20303FB02F3634A9B091360A0
:103370005B4B19600699DBF800200B0243EA0163FE
:1033800022F07F421343CBF800307FE60323019302
:10339000F7E6039BB3F5047F3FF661AFDDE9047CFC
:1033A000204623466E6904E001200133634514463C
:1033B00015D85A0957F8222003F01F01CA401F29C7
:1033C00018BF02F00102002BEED0A242ECD1013076
:1033D0008642EAD149480BE002230193D1E64FF43B
:1033E0008063DDE90310AA69FFF7F4FD00285DD0D2
:1033F0000023189A1360A3E62946069800F04CFAB9
:1034000000287FF47CAE069C082C51D0042C51D0AF
:10341000A4F10204B4FA84F4640901231E46194697
:103420002D4A136042F8843C2B4B19606B6AC9F833
:103430000030D9F800206B6A9A42F5D100274FF08E
:10344000FF30CAF80070FFF7CFFC264B264A3846FB
:103450001A60FFF7D7FC0A222449254B0C601A603A
:103460002A6924496B6AA1FB021203EB4303120988
:10347000DB0303FB02F3204A9B091360CAF80060D8
:10348000069BDBF800101A0242EA036321F07F4238
:103490001A43130A03F47F03134323F07F43CBF84B
:1034A0000030029B013B02937FF407AE002029E627
:1034B0000324B2E70224B0E74FF47F03D3F80C1CD7
:1034C000013106D0D3F80C3C45E703271AE7022761
:1034D00018E7162343E700BFC411845040118450FD
:1034E0002C11845000118450FEFFFF0F0C118450EA
:1034F00038118450ABAAAAAAD8118450360CF10016
:103500002DE9F0431B4C85B00746DDE90D56884692
:1035100020684FF0FF319146FFF7F8FC28BB0020F0
:10352000FFF724FDE8B90023CDE9005602934A468F
:10353000414638460C9BFFF78BFD05460120FFF7FF
:1035400015FD50B92068FFF7E9FC10B10A4800F0FA
:10355000D1F8284605B0BDE8F083084800F0CAF865
:10356000F0E7074800F0C6F8DDE7064800F0C2F8CB
:10357000D5E700BF14000020EC7C0100247D010091
:10358000047D0100D47C010010B5012486B005AB98
:10359000CDE901240093002204ABFFF759FD06B0EA
:1035A00010BD00BF2DE9F041ADF51A7D0F46059223
:1035B0000021144612A84FF408721E4603F080F84A
:1035C000002308A819462822069303F079F8002F53
:1035D0003CD0002E3AD0002C38D0042106A800F0B0
:1035E000C1F808A8282100F0BDF808A800F032F8BA
:1035F00078B14FF0FF3512A84FF4087100F088F948
:1036000006A8042100F084F928460DF51A7DBDE8CE
:10361000F08112AB0DF11C080390CDE90163024665
:1036200005AB08A9CDF8008006A8FFF769FF0028C0
:10363000DFD13368A342DCD3D8F800100546083147
:103640003846224600F08CF83460D4E74FF0FF355E
:10365000DAE700BF1C2330B583B002A941F8043D6E
:10366000044600F083F80546D8B9019B1C2B1BD1FA
:10367000D4E9003201210033E16118BF01230AB10E
:1036800043F00203A26832B9E268AAB9C4E9083279
:103690003BB90D4D09E0E26843F0040362B9C4E9A7
:1036A0000832284603B030BD084D20461C2100F0EA
:1036B00059F8284603B030BD0022284643F00803DD
:1036C000C4E9083203B030BD0E0CF000370CF00036
:1036D000BFF34F8F0549064BCA6802F4E0621343FB
:1036E000CB60BFF34F8F00BFFDE700BF00ED00E0F0
:1036F0000400FA05014B5B68184700BF1800002062
:10370000704700BF10B5044620B1BFF35F8F0020A3
:10371000206010BD0348FFF7EDFFBFF35F8F00206F
:10372000206010BD887D010010B5044610B1002353
:10373000236010BD0248FFF7DDFF0023236010BDAA
:10374000647D010050B10122D0E8EF3FC0E8E12FD5
:103750000029F9D1012BF7D0BFF35F8F002070470C
:1037600002F095BF0A46002102F0AABF18B111B1BC
:103770000B681C2B01D0012070474FF47F033A4A9D
:10378000D3F8101C91425AD0D3F8102C013256D0E5
:10379000D3F8102C4FF47F030260D3F8141C334A83
:1037A00091425ED0D3F8142C01325AD0D3F8142CA5
:1037B0004FF47F034260D3F8182C12F5947F4DD05C
:1037C000D3F8182C013249D0D3F8182C4FF47F03CA
:1037D0008260D3F81C1C264A91423CD0D3F81C2CA2
:1037E000013238D0D3F81C2C4FF47F03C260D3F8D9
:1037F000002C70322DD0D3F8002C013229D0D3F810
:10380000002C4FF47F030261D3F8042CAF321ED09A
:10381000D3F8042C01321AD0D3F8042C4FF47F03D0
:103820004261D3F8081C134A91420BD0D3F8082CFC
:10383000013207D0D3F8083C83610020704740F67E
:10384000FC02A7E740F23733836100207047512222
:10385000E4E79022D5E742F60412C5E740F6D862C5
:10386000B4E742F2D002A3E7FCF8FFFFD020FFFF4D
:103870000429FFFF37F3FFFF08B501464FF48060CE
:10388000FFF7C6FA00230249024A0B60136008BD25
:10389000C81184502C1184500138072815D8DFE84E
:1038A00000F0100C140814141404CB6800204B62B0
:1038B00070478B6800204B6270474B6800204B625A
:1038C00070470B6800204B6270470148704700BF8B
:1038D000310CF1000B6802E0082B0B6006D8026A7D
:1038E00013424FEA4303F7D0002070470048704767
:1038F000310CF10000230449044A0B604FF480604E
:103900001360FFF771BA00BF2C118450C4118450AA
:1039100030B129B100230144037001308142FBD151
:10392000704700BF0FB480B582B000AF8022002185
:103930000F4802F0C5FE07F114033B603B683A698B
:1039400080210B4800F05AFE78607B687F2B03DDF6
:10395000084B094A10681860084B1B6804489847D0
:1039600000BF0837BD46BDE8804004B0704700BFC7
:103970003CB90020B7B90020A87D010034B900206F
:103980000FB480B5A2B000AF194B1B68002B04D058
:10399000174B1B68B3F1FF3F01D1012300E0002367
:1039A000002B1DD107F19403C7F880303846D7F8B3
:1039B0008030D7F89020802100F020FEC7F88400E6
:1039C000D7F884307F2B06DD3B467B33094A1068ED
:1039D000186012791A71064B1B683A4610469847D0
:1039E00000BF8837BD46BDE8804004B0704700BFC7
:1039F00038B90020B07D0100C3438B426DD332F053
:103A00001F036AD1013902F01403014410B481EAA2
:103A10000004142B0ED8DFE803F0390D0D0D420D14
:103A20000D0D0D0D0D0D0D0D0D0D4B0D0D0D110091
:103A30009B0200D400205DF8044B70471F2C40E827
:103A4000C0F305D941E8C0F11C460B469C42F1D1B8
:103A500022F01402013A0A2AECD801A151F822F00E
:103A6000D53A0100CF3A0100313A0100353A010060
:103A7000353A0100353A0100353A0100C93A0100F2
:103A8000D53A0100C33A0100313A01001F2C40E849
:103A900000F3DDD941E800F11C460B46D6E71F2CA8
:103AA00040E840F3D4D941E840F11C460B46CDE74D
:103AB0001F2C40E880F3CBD941E880F11C460B462F
:103AC000C4E7DC02B7D4B5E75B03B3D5B3E759026B
:103AD000B1D5AFE71A03AED4ACE70020704700BF02
:103AE0001FB51C46094B05461B68D86852B1084BE8
:103AF00000910849CDE901322B46224600F022F818
:103B000002F07EFF044B1A46F2E700BF440000209B
:103B1000D07E0100DD7E01000B7F010008B5074B60
:103B2000044613B1002100E000BF054B1868836A0A
:103B300003B19847204601F069FE00BF0000000075
:103B4000607E01000EB403B503AB0146054853F88F
:103B5000042B0068019300F0DBF802B05DF804EB81
:103B600003B070474400002070B50D4E00250D4C89
:103B7000A41BA410A54209D10B4E00250B4C03F049
:103B8000F1FBA41BA410A54205D170BD56F8253049
:103B900001359847EEE756F8253001359847F2E7AA
:103BA0001402002014020020140200201802002039
:103BB000024B0146186800F051B800BF44000020D5
:103BC00038B50546002945D051F8043C0C1F002BA0
:103BD000B8BFE41803F011F81F4A1368104633B950
:103BE000636014602846BDE8384003F007B8A3427C
:103BF0000CD921686218934202BF1A685B68521898
:103C0000636008BF22600460ECE713465A680AB19B
:103C1000A242FAD919685818A0420BD12068014471
:103C2000581819608242DDD11068526801445A6008
:103C30001960D7E702D90C232B60D3E7206821183D
:103C40008A4202BF116852680918626008BF216089
:103C50005C60C7E738BD00BFBCB9002070B5CD1CA3
:103C6000064625F0030508350C2D38BF0C25002D20
:103C700001DBA94203D90C233360002070BD02F0A0
:103C8000BCFF214A1468214691B9204C23681BB916
:103C9000304600F0A3FC20602946304600F09EFC30
:103CA000431C24D10C233046336002F0A7FFE4E725
:103CB0000B685B1B18D40B2B0FD9CC180B60CD50A5
:103CC000304602F09BFF04F10B00231D20F007009B
:103CD000C31AD3D05A42E250D0E78C424B681ABF85
:103CE00063600C461360EBE70C464968CCE7C41CE4
:103CF00024F00304A04205D0211A304600F06EFCE7
:103D00000130CFD02560DBE7BCB90020C0B900206E
:103D10002DE9F04F9DB00C4617460646039318B1A7
:103D200083690BB900F010FE7B4B9C4257D174683D
:103D3000A38918075DD52369002B5AD000234FF0C3
:103D4000010B099320238DF8293030238DF82A3078
:103D5000B846454615F8013B0BB1252B54D1B8EBBD
:103D6000070A0BD053463A462146304602F0C7FCBC
:103D7000013000F0C280099B5344099398F8003049
:103D8000002B00F0BA8000234FF0FF32049307931A
:103D90008DF853301A93CDE90523A84605225F48D4
:103DA00018F8011B02F01BFF049B78BBD90644BF27
:103DB00020228DF853201A0744BF2B228DF8532060
:103DC0002A782A2A2AD0A846079A00200A2541469E
:103DD00011F8013B303B092B69D960B324E0504B0B
:103DE0009C4201D1B468A3E74E4B9C4208BFF468E3
:103DF0009EE72146304600F061FC00289ED04FF03F
:103E0000FF301DB0BDE8F08FA846A2E7434A454603
:103E1000801A0BFA00F018430490BEE7039A111DB4
:103E20001268002A039101DB079204E0524243F03A
:103E300002030792049398F800302E2B0ED198F8C5
:103E400001302A2B38D1039B08F102081A1D1B6888
:103E5000002B0392B8BF4FF0FF330593324D03227E
:103E600098F80010284602F0BAFE40B14023401BEB
:103E700008F1010803FA00F0049B0343049398F847
:103E800000100622294808F101078DF8281002F0D9
:103E9000A6FE002837D0264B1BBB039B073323F01D
:103EA000070308330393099B4B44099350E705FB31
:103EB0000232012088468AE7002308F101080A251A
:103EC00019460593404610F8012B303A092A03D9C8
:103ED000002BC3D00591C1E705FB012101238046DA
:103EE000F0E703AB224604A930460093114B00F0E3
:103EF00023F8B0F1FF3F8146D5D1A3895B063FF59A
:103F00007EAF09987DE703AB224604A930460093B3
:103F1000084B00F051FAECE7847E01000C7F0100B1
:103F2000A47E0100647E0100127F0100167F010063
:103F3000393F0100FF6601002DE9F04F8DB00C46BE
:103F400016461F46DDF85880054600F069FD0368F7
:103F50001846049302F0F1FC002305900A93D8F868
:103F6000003094F818A00733D4F800B023F007030A
:103F700003F10802C8F80020D3E90023C4E91223A2
:103F8000D4E912894FF0FF3229F00043CDF81880B0
:103F90000793A74BDDE9060101F0ACFB70BB4FF0C6
:103FA000FF32A34BDDE9060101F086FB30BB0022A6
:103FB00000234046494601F075FB10B12D2384F8DB
:103FC00043309C4A9C4BBAF1470F8CBF90469846B1
:103FD0004FF0000903232BF00402236122600097B5
:103FE00033460BAA2146284602F02FFC013040F050
:103FF0008D804FF0FF300DB0BDE8F08F42464B464C
:104000004046494601F076FB10B18C4A8C4BDAE70A
:1040100061684BF480620AA84B1C3ED106236360A2
:1040200000232260CDF804A06168CDE9020309AB4A
:10403000284600930DF1230349EC108B02F071FB2D
:104040000AF0DF038046472B09D1099BD81C02DB0D
:104050006268934247DDAAF1020A5FFA8AFABAF16E
:10406000650F099924D80139524604F1500009918D
:1040700002F0B8FB0A9A81461318012A236102DC78
:104080002268D10701D5013323619DF82330002B2D
:10409000A5D02D2384F84330A1E7BAF1670F00F0D3
:1040A0007781BAF1470FBBD10029B9D10123B6E717
:1040B000BAF1660F19D1002963680CDD216113B9CB
:1040C0002268D20702D501330B442361099B4FF0CC
:1040D0000009A365D9E713B92268D00701D50233D7
:1040E000F3E70123F1E74FF0670ADDE90932934274
:1040F00005DB22682361D107E8D50133E5E7002B12
:10410000D4BFC3F1020301231344DEE723685A0539
:1041100007D42369424631462846B84701302BD19F
:1041200067E7BAF1650F40F2DC8000220023D4E992
:10413000120101F0ADFA002833D00123414A314683
:104140002846B84701303FF454AFDDE909239A42CD
:1041500002DB2368D8070FD531462846DDE9042362
:10416000B84701303FF445AF4FF0000804F11A0999
:104170000A9B013B434509DC23689B0700F103814F
:10418000E0680B9B9842B8BF184634E701234A46C3
:1041900031462846B84701303FF42BAF08F10108FB
:1041A000E6E7099B002B2BDC0123264A31462846F3
:1041B000B84701303FF41DAF099B23B90A9B13B9DF
:1041C0002368D907D8D531462846DDE90423B84706
:1041D00001303FF40EAF4FF0000904F11A0A099BB9
:1041E0005B424B4501DC0A9B94E701235246314672
:1041F0002846B84701303FF4FCAE09F10109EEE76B
:104200000A9AA36D9A42A8BF1A46002A914607DD72
:104210001346314642462846B84701303FF4E9AEDE
:1042200004F11A034FF0000B29EAE979069315E02F
:10423000FFFFEF7F217F01001D7F0100297F01002B
:10424000257F01002D7F01000123069A3146284673
:10425000B84701303FF4CDAE0BF1010BD4F858A0B4
:10426000AAEB09035B45EFDCDDE90923D0449A4260
:1042700015DB2368DA0712D40A9B0999A3EB0A021B
:10428000A3EB010A9245A8BF9246BAF1000F0EDCDB
:104290004FF000082AEAEA7A04F11A0919E0DDE988
:1042A000042331462846B8470130E5D1A1E65346FC
:1042B000424631462846B8470130E9D199E6012304
:1042C0004A4631462846B84701303FF492AE08F1DD
:1042D0000108DDE909239B1AA3EB0A034345EEDC41
:1042E0004AE70A9A012A01DCDB073AD50123424654
:1042F00031462846B84701303FF47BAE3146284668
:1043000008F10108DDE90423B84701303FF471AE3C
:104310000A9B002203F1FF3A0023D4E9120101F0C5
:10432000B7F9C8B95346424631462846B847013026
:104330000ED15EE60123524631462846B847013089
:104340003FF457AE08F101080A9B013B4345F1DCFD
:104350004B4604F15002DEE64FF0000804F11A0A61
:10436000F2E70123DFE701234A4631462846B847F2
:1043700001303FF43EAE08F10108E3680B9A9B1A46
:104380004345F0DCFCE64FF0000804F11909F4E7BE
:1043900000293FF48BAE00232260CDF804A0CDE9C4
:1043A000020309AB284600930DF1230349EC108B5F
:1043B00002F0B7F9804648E62DE9F04301F1430CDD
:1043C0000C46097E85B0174606466E2998460C9A1B
:1043D00000F0B38022D8632936D00AD8002900F033
:1043E000B980582900F0838004F1420584F8421016
:1043F00032E0642901D06929F6D1206813680506E6
:1044000003F104012AD51B681160002B03DA2D2269
:104410005B4284F843206F480A2239E0732900F098
:104420009D8008D86F2920D07029DDD1236843F002
:104430002003236003E0752917D07829D4D178238D
:10444000654884F8453055E0136804F14205191DAC
:104450001B68116084F8423001238CE01B6810F067
:10446000400F116018BF1BB2CFE713682568181DF5
:104470001060280601D51B6802E06806FBD51B8882
:104480006F29544814BF0A220822002184F84310DF
:104490006568002DA560C0F29580216821F00401B7
:1044A0002160002B3DD1002D40F08E806546082A0A
:1044B0000BD12368DB0708D5236962689A42DEBF07
:1044C000302305F8013C05F1FF35ACEB0503236112
:1044D000CDF800803B4603AA2146304602F0B5F9EC
:1044E00001304DD14FF0FF3005B0BDE8F0833948C1
:1044F00084F84510136821681D1D1B6815600A06A5
:104500000BD5CA0744BF41F0200121601BB92268C6
:1045100022F0200222601022B7E74D0648BF9BB26E
:10452000EFE76546B3FBF2F102FB1133C35C05F81C
:10453000013D0B460029F5D1B9E713682568181D20
:104540006169106028061B6801D5196002E06A06DF
:10455000FBD51980002365462361B9E71368191D4F
:10456000116000211D686268284602F038FB08B11E
:10457000401B606063682361002384F84330A7E731
:1045800023692A4639463046C0470130AAD02368FD
:104590009B0713D4E068039B9842B8BF1846A3E773
:1045A00001234A4639463046C04701309AD001358A
:1045B000E368039A9B1AAB42F2DCEBE7002504F1B7
:1045C0001909F5E7002BACD1037804F1420584F812
:1045D00042306CE72F7F0100407F010038B5002397
:1045E000054C05460846236001F0FAF8431C02D149
:1045F000236803B12B6038BDCCB9002007B5009308
:1046000013460A4601460348006802F0CDF903B09C
:104610005DF804FB44000020F8B50E46144605463C
:1046200018B183690BB900F08FF9214B9C422AD154
:104630006C68A369A360A3891A072ED5236963B3A5
:104640002369F6B220683746C01A6369834204DCE6
:104650002146284600F024F928BBA3680130013B1D
:10466000A36023685A1C22601E706369834204D0D1
:10467000A389DB0719D50A2E17D12146284600F059
:104680000FF990B10FE00B4B9C4201D1AC68D0E721
:10469000094B9C4208BFEC68CBE72146284600F056
:1046A0000DF80028CCD04FF0FF373846F8BD00BFDA
:1046B000847E0100A47E0100647E0100324B70B54F
:1046C0001D6806460C4625B1AB6913B9284600F0B3
:1046D0003BF92E4B9C420FD16C68B4F90C309AB266
:1046E00015072CD4D00611D40922326043F04003C0
:1046F0004FF0FF30A3813EE0254B9C4201D1AC68D6
:10470000EBE7244B9C4208BFEC68E6E7510712D563
:10471000616B41B104F14403994202D03046FFF786
:104720004FFA00236363A38923F02403A3810023AA
:10473000636023692360A38943F00803A38123698D
:104740004BB9A38903F42073B3F5007F03D021464E
:10475000304600F073F9A28912F001030CD0002357
:10476000A36063695B42A361236953B9B4F90C3058
:1047700013F08000BAD170BD920758BF6369A3607F
:10478000F2E70020F7E700BF44000020847E01002C
:10479000A47E0100647E01008A892DE9F04105466E
:1047A00010070C4658D44B68002B05DC0B6C002B13
:1047B00002DC0020BDE8F081E66A002EF9D000237B
:1047C00012F480522F68216A2B6032D0606DA38969
:1047D0005A0705D56368C01A636B0BB1236CC01A06
:1047E00000230246E66A2846216AB047431CA38993
:1047F00006D129681D2947D8284ACA40D60743D57B
:104800000022D90462602269226004D5421C01D1D1
:104810002B6803B96065616B2F600029C9D004F172
:104820004403994202D02846FFF7CAF9002060638A
:10483000C0E701232846B047411CC8D12B68002B94
:10484000C5D01D2B01D0162B01D12F60B1E7A38954
:1048500043F04003A381ADE70F69002FA9D0930770
:104860000E680F600CBF4B690023A6EB07088B6036
:10487000B8F1000F9DDD43463A46216A2846A66AF4
:10488000B047002806DCA38943F040034FF0FF3017
:10489000A3818FE70744A8EB0008E9E70100402067
:1048A00038B50B6905460C46DBB118B183690BB905
:1048B00000F04AF80C4B9C4209D16C68B4F90C30FA
:1048C0007BB121462846BDE83840FFF765BF074B5E
:1048D0009C4201D1AC68F1E7054B9C4208BFEC68F3
:1048E000ECE7002038BD00BF847E0100A47E0100FB
:1048F000647E0100002310B504468360818119465F
:104900004366C28108228361C0E90033C0E90433F1
:104910005C3001F0D5FE054B24626362044BA36258
:10492000044BE362044B236310BD00BF917201008E
:10493000B3720100EB7201000F730100014902F034
:104940000CB900BFA1480100836910B5044633BB10
:104950000365134AC0E91233124B82621B68984206
:1049600004BF0123836100F01FF86060204600F05F
:104970001BF8A060204600F017F80022E060042138
:104980006068FFF7B7FF01220921A068FFF7B2FFB7
:1049900002221221E068FFF7ADFF0123A36110BDE1
:1049A0003D490100607E0100F8B51B4B07461E68BB
:1049B000B36913B93046FFF7C7FF4836D6E901346B
:1049C000013B03D5336833B13668F7E7B4F90C50CF
:1049D0006DB16834F4E70421384602F0A8F830607D
:1049E0000028F1D10C2304463B602046F8BD0B4B58
:1049F000082265662946A56004F15C00C4E90055FB
:104A0000C4E90335C4E9055501F05AFEC4E90D5562
:104A1000C4E91255E9E700BF607E01000100FFFF15
:104A2000044B1B68186A044B002808BF1846F03076
:104A3000704700BF44000020A80000208B8973B598
:104A40009D0706460C4607D504F147032360236102
:104A50000123636102B070BD01AB6A4602F09BF8AE
:104A6000009905463046FFF7F9F848B9B4F90C301B
:104A70009A05EFD423F0030343F00203A381E3E795
:104A80000D4BB362A389206043F080032061A381B2
:104A9000009B6361019B5BB1B4F90E10304600F0DE
:104AA0009FF928B1A38923F0030343F00103A381F5
:104AB000A3891D43A581CDE73D4901002DE9F843B8
:104AC000154612F0030206460F4607D0013A214C64
:104AD000002354F8222002F0DDF80746AD1035D04F
:104AE000746A3CB91020FFF763F870620460C46018
:104AF000C0E90144D6F82480D8F808404CB940F207
:104B00007121304602F051F900230446C8F808002C
:104B100003604FF00008EB070AD5394622463046BD
:104B200002F04CF98146394630464F4602F09BF878
:104B30006D100BD0206838B922462146304602F06D
:104B40003DF92060C0F800800446E4E73846BDE83F
:104B5000F88300BFC47E01002DE9F04F9DB0804670
:104B60000C46164603938B891D060FD50B696BB94E
:104B70004021FFF773F82060206128B90C23C8F8A2
:104B800000304FF0FF30C7E04023636100234FF057
:104B9000010B099320238DF8293030238DF82A301A
:104BA00037463D4615F8013B0BB1252B3ED1B7EBFF
:104BB000060A0BD0534632462146404602F0E4FA3C
:104BC000013000F0A480099B534409933B78002BEB
:104BD00000F09D8000234FF0FF32049307938DF87F
:104BE00053301A93CDE905232F460522504817F874
:104BF000011B01F0F4FF049BD0B9D90644BF202269
:104C00008DF853201A0744BF2B228DF853202A78A1
:104C10002A2A15D02F46079A00200A25394611F86E
:104C2000013B303B092B4DD9B8B10FE02F46B8E717
:104C30003F4A3D46801A0BFA00F018430490D3E730
:104C4000039A111D1268002A039101DB079204E008
:104C5000524243F00203079204933B782E2B0CD16F
:104C60007B782A2B33D1039B02371A1D1B68002B3C
:104C70000392B8BF4FF0FF3305932E4D03223978CE
:104C8000284601F0ACFF38B14023401B013703FA3E
:104C900000F0049B034304933978062226487E1CC7
:104CA0008DF8281001F09BFF002838D0234B13BB50
:104CB000039B073323F0070308330393099B4B44FB
:104CC00009936DE705FB023201200F46A6E700239A
:104CD00001370A2519460593384610F8012B303A5A
:104CE000092A03D9002BC8D00591C6E705FB01218D
:104CF00001230746F0E703AB224604A94046009390
:104D00000F4BFFF719F9B0F1FF3F8146D6D1A389C8
:104D10005B063FF536AF09981DB0BDE8F08F03ABD9
:104D2000224604A940460093054BFFF745FBEAE7FE
:104D30000C7F0100127F0100167F0100393F010046
:104D400089710100024B0146186802F077BA00BF72
:104D50004400002038B50023064C0546084611469D
:104D6000236000F025FD431C02D1236803B12B60B2
:104D700038BD00BFCCB9002038B50546064C084602
:104D80001146002222601A4600F038FD431C02D171
:104D9000236803B12B6038BDCCB9002038B500239F
:104DA000054C05460846236000F0E2FC431C02D196
:104DB000236803B12B6038BDCCB9002038B500237F
:104DC000064C054608461146236000F0D9FC431CFA
:104DD00002D1236803B12B6038BD00BFCCB90020DD
:104DE00038B50023054C05460846236000F0D8FC82
:104DF000431C02D1236803B12B6038BDCCB900201D
:104E000038B50546064C08461146002222601A466F
:104E100000F0D6FC431C02D1236803B12B6038BDDF
:104E2000CCB9002038B50546064C0846114600228C
:104E300022601A4600F0CCFC431C02D1236803B167
:104E40002B6038BDCCB9002081F0004102E000BFEA
:104E500083F0004330B54FEA41044FEA430594EA3A
:104E6000050F08BF90EA020F1FBF54EA000C55EA75
:104E7000020C7FEA645C7FEA655C00F0E2804FEA46
:104E80005454D4EB5555B8BF6D420CDD2C4480EA28
:104E9000020281EA030382EA000083EA010180EA58
:104EA000020281EA0303362D88BF30BD11F0004FA6
:104EB0004FEA01314FF4801C4CEA113102D04042DC
:104EC00061EB410113F0004F4FEA03334CEA133317
:104ED00002D0524263EB430394EA050F00F0A7802F
:104EE000A4F10104D5F1200E0DDB02FA0EFC22FA2A
:104EF00005F2801841F1000103FA0EF2801843FA1E
:104F000005F359410EE0A5F120050EF1200E012A0E
:104F100003FA0EFC28BF4CF0020C43FA05F3C0184C
:104F200051EBE37101F0004507D54FF0000EDCF1C5
:104F3000000C7EEB00006EEB0101B1F5801F1BD36E
:104F4000B1F5001F0CD349085FEA30004FEA3C0C72
:104F500004F101044FEA445212F5800F80F09A8068
:104F6000BCF1004F08BF5FEA500C50F1000041EB6C
:104F7000045141EA050130BD5FEA4C0C404141EB70
:104F8000010111F4801FA4F10104E9D191F0000F97
:104F900004BF01460020B1FA81F308BF2033A3F11A
:104FA0000B03B3F120020CDA0C3208DD02F1140C11
:104FB000C2F10C0201FA0CF021FA02F10CE002F14C
:104FC0001402D8BFC2F1200C01FA02F120FA0CFC45
:104FD000DCBF41EA0C019040E41AA2BF01EB04518E
:104FE000294330BD6FEA04041F3C1CDA0C340EDC8C
:104FF00004F11404C4F1200220FA04F001FA02F3CF
:1050000040EA030021FA04F345EA030130BDC4F18C
:105010000C04C4F1200220FA02F001FA04F340EA81
:105020000300294630BD21FA04F0294630BD94F032
:10503000000F83F4801306BF81F480110134013D19
:105040004EE77FEA645C18BF7FEA655C29D094EA8A
:10505000050F08BF90EA020F05D054EA000C04BF08
:105060001946104630BD91EA030F1EBF00210020F3
:1050700030BD5FEA545C05D14000494128BF41F092
:10508000004130BD14F580043CBF01F5801130BDF6
:1050900001F0004545F0FE4141F470014FF0000081
:1050A00030BD7FEA645C1ABF194610467FEA655C32
:1050B0001CBF0B46024650EA013406BF52EA0335D4
:1050C00091EA030F41F4002130BD00BF90F0000FC2
:1050D00004BF0021704730B54FF4806404F13204FE
:1050E0004FF000054FF0000150E700BF90F0000FB7
:1050F00004BF0021704730B54FF4806404F13204DE
:1051000010F0004548BF40424FF000013EE700BFAD
:1051100042004FEAE2014FEA31014FEA02701FBF3D
:1051200012F07F4393F07F4F81F06051704732F06F
:105130007F4208BF704793F07F4F04BF41F40021C6
:10514000704730B54FF4607401F0004521F0004124
:105150001CE700BF50EA010208BF704730B54FF0AE
:1051600000050AE050EA010208BF704730B511F0AF
:10517000004502D5404261EB41014FF4806404F1E7
:1051800032045FEA915C3FF4D8AE4FF003025FEA6D
:10519000DC0C18BF03325FEADC0C18BF033202EBF1
:1051A000DC02C2F1200300FA03FC20FA02F001FA4B
:1051B00003FE40EA0E0021FA02F11444BDE600BFEE
:1051C00070B54FF0FF0C4CF4E06C1CEA11541DBF9D
:1051D0001CEA135594EA0C0F95EA0C0F00F0DEF868
:1051E0002C4481EA030621EA4C5123EA4C5350EA4D
:1051F000013518BF52EA033541F4801143F480139E
:1052000038D0A0FB02CE4FF00005E1FB02E506F02E
:105210000042E0FB03E54FF00006E1FB03569CF083
:10522000000F18BF4EF0010EA4F1FF04B6F5007F89
:1052300064F5407404D25FEA4E0E6D4146EB0606FB
:1052400042EAC62141EA55514FEAC52040EA5E5084
:105250004FEACE2EB4F1FD0C88BFBCF5E06F1ED82E
:10526000BEF1004F08BF5FEA500E50F1000041EB65
:10527000045170BD06F0004646EA010140EA020012
:1052800081EA0301B4EB5C04C2BFD4EB0C0541EA34
:10529000045170BD41F480114FF0000E013C00F349
:1052A000AB8014F1360FDEBF002001F0004170BD6D
:1052B000C4F10004203C35DA0C341BDC04F1140486
:1052C000C4F1200500FA05F320FA04F001FA05F212
:1052D00040EA020001F0004221F0004110EBD370DF
:1052E00021FA04F642EB06015EEA430E08BF20EA0B
:1052F000D37070BDC4F10C04C4F1200500FA04F3AE
:1053000020FA05F001FA04F240EA020001F000413F
:1053100010EBD37041F100015EEA430E08BF20EAB2
:10532000D37070BDC4F1200500FA05F24EEA020EFA
:1053300020FA04F301FA05F243EA020321FA04F029
:1053400001F0004121FA04F220EA020000EBD370E0
:105350005EEA430E08BF20EAD37070BD94F0000FE0
:105360000FD101F00046400041EB010111F4801F14
:1053700008BF013CF7D041EA060195F0000F18BFC5
:10538000704703F00046520043EB030313F4801F01
:1053900008BF013DF7D043EA0603704794EA0C0FBB
:1053A0000CEA135518BF95EA0C0F0CD050EA4106D1
:1053B00018BF52EA4306D1D181EA030101F000414E
:1053C0004FF0000070BD50EA410606BF1046194676
:1053D00052EA430619D094EA0C0F02D150EA013682
:1053E00013D195EA0C0F05D152EA03361CBF1046C3
:1053F00019460AD181EA030101F0004141F0FE4162
:1054000041F470014FF0000070BD41F0FE4141F4E5
:10541000780170BD70B54FF0FF0C4CF4E06C1CEAE5
:1054200011541DBF1CEA135594EA0C0F95EA0C0F9A
:1054300000F0A7F8A4EB050481EA030E52EA033555
:105440004FEA013100F088804FEA03334FF0805576
:1054500045EA131343EA12634FEA022245EA1115A3
:1054600045EA10654FEA00260EF000419D4208BF54
:10547000964244F1FD0404F5407402D25B084FEA01
:105480003202B61A65EB03055B084FEA32024FF4AD
:1054900080104FF4002CB6EB020E75EB030E22BF0A
:1054A000B61A754640EA0C005B084FEA3202B6EBCA
:1054B000020E75EB030E22BFB61A754640EA5C0079
:1054C0005B084FEA3202B6EB020E75EB030E22BF09
:1054D000B61A754640EA9C005B084FEA3202B6EB0A
:1054E000020E75EB030E22BFB61A754640EADC00C9
:1054F00055EA060E18D04FEA051545EA16754FEA2B
:1055000006164FEAC30343EA52734FEAC2025FEA48
:105510001C1CC0D111F4801F0BD141EA00014FF0D7
:1055200000004FF0004CB6E711F4801F04BF0143A8
:105530000020B4F1FD0C88BFBCF5E06F3FF6AFAEC4
:10554000B5EB030C04BFB6EB020C5FEA500C50F154
:10555000000041EB045170BD0EF0004E4EEA1131D7
:1055600014EB5C04C2BFD4EB0C0541EA045170BDDE
:1055700041F480114FF0000E013C90E645EA060E22
:105580008DE60CEA135594EA0C0F08BF95EA0C0F50
:105590003FF43BAF94EA0C0F0AD150EA01347FF498
:1055A00034AF95EA0C0F7FF425AF104619462CE76F
:1055B00095EA0C0F06D152EA03353FF4FDAE1046D2
:1055C000194622E750EA410618BF52EA43067FF423
:1055D000C5AE50EA41047FF40DAF52EA43057FF4B3
:1055E000EBAE12E74FF0FF3C06E000BF4FF0010CBE
:1055F00002E000BF4FF0010C4DF804CD4FEA410C22
:105600007FEA6C5C4FEA430C18BF7FEA6C5C1BD0EE
:1056100001B050EA410C0CBF52EA430C91EA030F6F
:1056200002BF90EA020F0020704710F1000F91EACC
:10563000030F58BF994208BF90422CBFD8176FEA9A
:10564000E37040F0010070474FEA410C7FEA6C5C68
:1056500002D150EA013C07D14FEA430C7FEA6C5C6F
:10566000D6D152EA033CD3D05DF8040B704700BF9B
:105670008446104662468C461946634600E000BFE9
:1056800001B5FFF7B7FF002848BF10F1000F01BDBB
:105690004DF808EDFFF7F4FF0CBF012000205DF886
:1056A00008FB00BF4DF808EDFFF7EAFF34BF01200B
:1056B00000205DF808FB00BF4DF808EDFFF7E0FFA4
:1056C00094BF012000205DF808FB00BF4DF808EDF5
:1056D000FFF7CEFF94BF012000205DF808FB00BF5C
:1056E0004DF808EDFFF7C4FF34BF012000205DF83E
:1056F00008FB00BF4FEA410C7FEA6C5C02D150EA24
:10570000013C0AD14FEA430C7FEA6C5C02D152EAB9
:10571000033C02D14FF0000070474FF0010070478A
:105720004FEA410212F5001215D211D56FF47873C9
:10573000B3EB625212D94FEAC12343F0004343EA6C
:10574000505311F0004F23FA02F018BF4042704747
:105750004FF00000704750EA013005D111F00040D1
:1057600008BF6FF0004070474FF00000704700BF67
:10577000024B58224FF0FF301A607047CCB900201E
:10578000024B58224FF0FF301A607047CCB900200E
:10579000024B58224FF0FF301A607047CCB90020FE
:1057A000024B582200201A60704700BFCCB900207D
:1057B000024B58224FF0FF301A607047CCB90020DE
:1057C000024B58224FF0FF301A607047CCB90020CE
:1057D000024B58224FF0FF301A607047CCB90020BE
:1057E000044A05491368002B08BF0B4619181846D0
:1057F00011607047C4B90020D0B90020024B582274
:105800004FF0FF301A607047CCB90020FEE700BFB0
:1058100080B485B000AFF860B96011461A460B46F7
:10582000FB711346BB71FB79002B01D0102200E005
:105830000022BB79002B01D0202300E0002313437A
:105840003A7E002A02D04FF4807200E0002242EA41
:105850000301FB68BA6802F5007243F8221000BF2A
:105860001437BD465DF8047B704780B584B000AF47
:1058700078603B1D1846FBF7D1F9F860FB685B6860
:10588000BB60BB68DA437B68012101FA03F31A406D
:10589000FB689A607B6801229A40BB681A40FB68EB
:1058A000DA6000BF1037BD4680BD80B584B000AF60
:1058B0007860084611461A460346FB700B46BB70DB
:1058C00013467B703B1D1846FBF7A6FAF860FA7882
:1058D000BB785B001A437B789B001A433B7E1B021C
:1058E00042EA03013B7F1B047A681943FB6880325C
:1058F00043F8221000BF1037BD4680BD80B584B08C
:1059000002AF78600023019300230093002301225B
:1059100001217868FFF7C9FF00BF0837BD4680BD89
:1059200080B584B002AF78600B46FB70FA78002334
:105930000193002300931346002200217868FFF7AB
:10594000B4FF00BF0837BD4680BD80B584B000AF4E
:1059500078603B1D1846FBF75FFAF8607B68012210
:1059600002FA03F31946F86800F02CF800BF10376C
:10597000BD4680BD80B584B000AF78603B1D184641
:10598000FBF74AFAF8607B68012202FA03F3194632
:10599000F86800F025F800BF1037BD4680BD80B51F
:1059A00082B000AF786039603B68002B03D1786823
:1059B000FFF7E0FF02E07868FFF7C7FF00BF083796
:1059C000BD4680BD80B483B000AF786039607B682D
:1059D0003A689A6000BF0C37BD465DF8047B70479B
:1059E00080B483B000AF786039607B683A68DA6071
:1059F00000BF0C37BD465DF8047B704780B485B0AE
:105A000000AFF8607B600B46FB721346BB72BB7A3B
:105A1000002B01D0102200E000227B6813433A7E65
:105A2000002A02D04FF4807100E00021FA7A194375
:105A3000FB6802F5C07243F8221000BF1437BD4660
:105A40005DF8047B704780B483B000AFEFF305834B
:105A50007B607B68002B08D0002383F30B88002336
:105A600083F30988022383F3148800BF0C37BD46F3
:105A70005DF8047B7046714672467346B7EE000AC5
:105A8000F7EE000AB7EE001AF7EE001AB7EE002A9A
:105A9000F7EE002AB7EE003AF7EE003AB7EE004A0A
:105AA000F7EE004AB7EE005AF7EE005AB7EE006A7A
:105AB000F7EE006AB7EE007AF7EE007A8EF3008C0C
:105AC00010B4F1EE10CA4FF66074C0F6FF740CEA21
:105AD000040CE1EE10CA10BCF446744780B586B0E1
:105AE00000AF786000233B6100237B61EFF3058307
:105AF000FB60FB68002B1FD00C20FBF7FDFD7861DD
:105B00007B69002B18D07868FBF7F6FD38613B699C
:105B1000002B0CD03A697B681A447B699A607B69D8
:105B20003A695A607B699A687B691A6004E078690F
:105B3000FBF796FE00237B617B6918461837BD464C
:105B4000BDE88040714672467346B7EE000AF7EE34
:105B5000000AB7EE001AF7EE001AB7EE002AF7EEC9
:105B6000002AB7EE003AF7EE003AB7EE004AF7EE39
:105B7000004AB7EE005AF7EE005AB7EE006AF7EEA9
:105B8000006AB7EE007AF7EE007A8EF3008C10B45C
:105B9000F1EE10CA4FF66074C0F6FF740CEA040C04
:105BA000E1EE10CA10BCF446744780B584B000AF73
:105BB0007860EFF30583FB60FB68002B11D07B68F6
:105BC000002B06D1012383F31088012383F39088EF
:105BD000FEE77B685B681846FBF742FE7868FBF7D8
:105BE0003FFE00BF1037BD46BDE88040704671469D
:105BF00072467346B7EE000AF7EE000AB7EE001AD7
:105C0000F7EE001AB7EE002AF7EE002AB7EE003AD8
:105C1000F7EE003AB7EE004AF7EE004AB7EE005A48
:105C2000F7EE005AB7EE006AF7EE006AB7EE007AB8
:105C3000F7EE007A8EF3008C10B4F1EE10CA4FF636
:105C40006074C0F6FF740CEA040CE1EE10CA10BCDC
:105C5000F446744780B483B000AF7860EFF30581F9
:105C600021B106C882F30B8881F3098800BF00BF09
:105C70000C37BD465DF8047B70467146724673462C
:105C8000B7EE000AF7EE000AB7EE001AF7EE001AB8
:105C9000B7EE002AF7EE002AB7EE003AF7EE003A28
:105CA000B7EE004AF7EE004AB7EE005AF7EE005A98
:105CB000B7EE006AF7EE006AB7EE007AF7EE007A08
:105CC0008EF3008C10B4F1EE10CA4FF66074C0F67B
:105CD000FF740CEA040CE1EE10CA10BCF4467447E1
:105CE00080B483B000AF7860EFF3058159B1EFF372
:105CF000098121ED010AB1EC010A0160002181F363
:105D00000B8881F3098800BF00BF0C37BD465DF8E2
:105D1000047B7046714672467346B7EE000AF7EE92
:105D2000000AB7EE001AF7EE001AB7EE002AF7EEF7
:105D3000002AB7EE003AF7EE003AB7EE004AF7EE67
:105D4000004AB7EE005AF7EE005AB7EE006AF7EED7
:105D5000006AB7EE007AF7EE007A8EF3008C10B48A
:105D6000F1EE10CA4FF66074C0F6FF740CEA040C32
:105D7000E1EE10CA10BCF446744780B500AF00F0E5
:105D800080F800BF80BD80B584B000AF78603B1D57
:105D90001846FBF75FFEF860FB685B68BB60BB689A
:105DA000DA437B68012101FA03F31A40FB689A6029
:105DB0007B6801229A40BB681A40FB68DA6000BF2A
:105DC0001037BD4680BD80B485B000AFF860B960C3
:105DD00011461A460B46FB711346BB71FB79002B2B
:105DE00001D0102200E00022BB79002B01D020233B
:105DF00000E0002313433A7E002A02D04FF4807261
:105E000000E0002242EA0301FB68BA6802F5007272
:105E100043F8221000BF1437BD465DF8047B70477D
:105E200008B5C820FCF7AEF9BDE808403620FCF7FD
:105E3000A9B941F20400FCF7A5B980B582B000AF62
:105E4000786001E0FFF7F5FF7B685A1E7A60002B4F
:105E5000F8D100BF0837BD4680BD80B483B000AF25
:105E600078607B68D3F8003403F00103002B14BF83
:105E700001230023DBB218460C37BD465DF8047BD6
:105E8000704780B400AF00BFBD465DF8047B70472B
:105E900080B584B000AFF860B9607A60FB687A685A
:105EA0001946B86800F0E8FB00BF1037BD4680BD5A
:105EB00080B584B000AFF860B9607A60FB687A683A
:105EC000B968184600F0C9FB0346002B0CBF01233C
:105ED0000023DBB218461037BD4680BD80B584B0C4
:105EE00000AFF860B9607A60FB707A68B968F868EA
:105EF000FFF7DEFF0346002B19D001231DE07A686F
:105F0000B968F86800F01EFB00BFFCF747F90346CC
:105F100083F00103DBB2002BF7D17A68B968F86827
:105F2000FFF7C6FF0346002B01D0012305E0FB78F5
:105F30005A1EFA70002BE2D1002318461037BD46D6
:105F400080BD80B400AF00BFBD465DF8047B7047E4
:105F500080B582B000AF786079684FF05020FCF7D0
:105F6000F5F9034618460837BD4680BD80B500AF39
:105F7000FCF7B6F980B483B000AF786039607B6815
:105F80003A68C3F8082300BF0C37BD465DF8047BB0
:105F9000704780B483B000AF78600B467B807B880D
:105FA0007A6813441B6818460C37BD465DF8047BBD
:105FB000704780B483B000AF78600B467B807B88ED
:105FC0007A68134400221A6000BF0C37BD465DF8A2
:105FD000047B704780B400AF00BFBD465DF8047B12
:105FE000704780B584B000AF7860084611461A4605
:105FF0000346FB700B46BB7013467B703B1D184677
:10600000FCF764FAF860FA78BB785B001A437B7897
:106010009B001A433B7E1B0242EA03013B7F1B04A9
:106020007A681943FB68803243F8221000BF1037AA
:10603000BD4680BD80B584B000AF78603B1D18467A
:10604000FCF744FAF8607B68012202FA03F3194670
:10605000F86800F004F800BF1037BD4680BD80B47A
:1060600083B000AF786039607B683A689A6000BF9F
:106070000C37BD465DF8047B704780B485B000AF37
:106080000346FB710023FB600023BB600FE001228D
:10609000BB6802FA03F3DAB2FB791340DBB2002BE0
:1060A00002D0FB680133FB60BB680133BB60BB6897
:1060B000072BECDDFB6803F00103002B01D101236A
:1060C00000E0002318461437BD465DF8047B704796
:1060D00080B483B000AF78607B681B7803F07F03E7
:1060E000DAB27B681A7000BF0C37BD465DF8047BDE
:1060F000704780B5A6B000AFF860B9607A60FB70F9
:106100000023C7F894307B68802B03D98023C7F81D
:10611000943002E07B68C7F894307A68D7F89430FE
:10612000D31A7B6007F11003D7F89420B96818469A
:1061300000F0A2FAFB78002B35D00023C7F890308E
:106140002BE007F11002D7F8903013441846FFF700
:10615000BFFF07F11002D7F8903013441B781846A0
:10616000FFF78BFF034683F00103DBB2002B0FD058
:1061700007F11002D7F8903013441B7863F07F03C7
:10618000D9B207F11002D7F8903013440A461A70BA
:10619000D7F890300133C7F89030D7F89030D7F85F
:1061A00094209A42CDD8FB681B6807F11002C3F80F
:1061B0004425FB681B68D7F89420C3F84825FB6882
:1061C0001B680022C3F82021FB681B6801229A602B
:1061D00000BFFB681B68D3F82031012BF9D17B6825
:1061E000002B90D100BF9837BD4680BD80B584B0EC
:1061F00000AF78603960386800F09FFBF860FA689B
:1062000039687868FCF76CFA00BF1037BD4680BD6E
:1062100080B584B000AF78607B685B7D002B22D0B6
:106220007B681B68D3F81031012B1CD17B681B7A6B
:10623000FB737B681B680022C3F810217B68DB6856
:10624000002B0CD07B689B7D002B03D0FB7B03F0E5
:106250007F03FB737B68DB68FA7B104698477B689B
:106260001B6801221A6000BF1037BD4680BD80B494
:1062700085B000AFF8607A601A460B46FB72134691
:10628000BB72FA7AFB689832796843F83210BB7AAD
:10629000002B06D0FB7AFA689833DB001344012206
:1062A0005A6000BF1437BD465DF8047B704780B468
:1062B00083B000AF7860084611461A460346FB706B
:1062C0000B46BB7013467B707B783A7C002A02D069
:1062D0004FF4807100E00021FA7819437B68A03206
:1062E00043F83210BA783B7C002B02D04FF4807117
:1062F00000E00021FB780A437968A033DB000B44FF
:106300005A6000BF0C37BD465DF8047B704780B40F
:1063100085B000AFF8607B600B46FB721346BB7222
:10632000BB7A002B01D0102200E000227B681343CF
:106330003A7E002A02D04FF4807100E00021FA7A00
:106340001943FB6802F5C07243F8221000BF1437EE
:10635000BD465DF8047B704780B485B000AFF8603F
:106360007B600B46FB721346BB72BB7A002B01D0DD
:10637000102200E000227B6813433A7E002A02D0FC
:106380004FF4807100E00021FA7A1943FB6802F5AE
:10639000E07243F8221000BF1437BD465DF8047B5D
:1063A000704780B485B000AFF860B96011461A46F6
:1063B0000B46FB711346BB71FB79002B01D01022F9
:1063C00000E00022BB79002B01D0202300E0002355
:1063D00013433A7E002A02D04FF4807200E000227C
:1063E00042EA0301FB68BA6802F5007243F8221022
:1063F00000BF1437BD465DF8047B704780B400AF22
:106400004FF050230222C3F818254FF050230122E9
:106410009A6000BFBD465DF8047B704780B500AF51
:106420001B20FCF711FA1C20FCF70EFA2A20FCF7BF
:106430000BFA0820FCF708FA0920FCF705FA0A20F5
:10644000FCF702FA0B20FCF7FFF93120FCF7FCF90E
:106450001520FCF7F9F91420FCF7F6F96FF00C00A1
:10646000FCF7F2F900BF80BD80B483B000AF786064
:106470007B68D3F8083403F00103002B14BF012319
:106480000023DBB218460C37BD465DF8047B70472D
:1064900080B483B000AF78600B46FB70FA787B68FD
:1064A000C3F8042500BF0C37BD465DF8047B704778
:1064B00080B489B000AFF860B9607A60FB6803F01F
:1064C0000303FB614FF0FF337B610023BB610EE0F0
:1064D000BA68BB691A4407F11401FB690B441278CE
:1064E0001A70FB690133FB61BB690133BB61BA6997
:1064F0007B689A42ECD37B6918462437BD465DF829
:10650000047B704780B586B000AFF860B9607A60F0
:1065100000237B610EE07B699A00FB68D0187B69E1
:106520009B00BA6813441B681946FCF729FB7B697A
:1065300001337B617A697B689A42ECD300BF1837DC
:10654000BD4680BD90B58BB000AFF860B9607A6091
:10655000FCF70CFBBB687B62FB6803F00303FB6189
:10656000FB69002B22D0FB69C3F104033B623A6A4A
:106570007B689A4201D97B683B62FA68FB69D41A4E
:106580003A6A796AF868FFF793FF0346194620468E
:10659000FCF7F6FA7A683B6AD31A7B60FA683B6AC2
:1065A0001344FB607A6A3B6A13447B627B689B08F6
:1065B000BB61BA69796AF868FFF7A4FFBB699B0001
:1065C000FA681344FB60BB699B007A6A13447B62E0
:1065D0007B6803F003037B617B69002B09D07A6938
:1065E000796AF868FFF764FF03461946F868FCF714
:1065F000C7FAFCF7B1FA00BF2C37BD4690BD2DE9B4
:10660000E04F2746A046A146A246A346A4462DED4C
:10661000108B4FF0000545EC185B45EC195A45EC22
:106620001A5A45EC1B5A45EC1C5A45EC1D5A45ECD0
:106630001E5A45EC1F5AF1EE105A4FF66076C0F61E
:10664000FF763540E1EE105A84F300882546264651
:10665000A447BDEC108BBDE8E08F30B50024A2420A
:1066600001D1002007E0035D01340D1915F8015C2C
:10667000AB42F4D0581B30BD431E0A4410B59142C2
:1066800000D110BD11F8014B03F8014FF7E7884224
:1066900001EB020310B507D8421E99420AD011F847
:1066A000014B02F8014FF8E78342F5D98118D21A5D
:1066B000D34200D110BD13F8014D01F8014DF7E7A9
:1066C00002440346934200D1704703F8011BF9E7E7
:1066D0009368013B002B936010B408DA9469A342DD
:1066E00001DB0A2903D15DF8044BFDF795BF136860
:1066F000581C1060084619705DF8044B7047F8B5D7
:1067000006460F461446D518AC4201D1002007E0DA
:106710003A4614F8011B3046FFF7DAFF431CF3D169
:10672000F8BD2DE9FF4755EC104B002D0D9F0E468F
:1067300091461946B8BF22462B4627F02007B6BF20
:1067400005F1004300231446DDF830A0BCBF1D4610
:106750002D23462F0B7004D0452F00D10136022186
:1067600000E0032103AB3246019302AB45EC104B32
:1067700000935346F9F744FC472F804602D119F0A5
:10678000010F26D0462F08EB060911D198F80030EA
:10679000302B0AD10022002320462946FEF778FF3D
:1067A00018B9C6F10106CAF80060DAF80030994459
:1067B0000022002320462946FEF76AFF38B930221E
:1067C000039B4B4505D2591C03911A70F8E7CDF88D
:1067D0000C90039B40460E9AA3EB0803136004B091
:1067E000BDE8F087F7B500290446BABF49422D231A
:1067F0002B2304F8022B0929437020DD0DF1070338
:106800000A261F465A1E91FBF6F506FB1511092DA7
:1068100001F1300103F8011C294609DC3031023B4B
:1068200002F8011CBB42224604D3101A03B0F0BD8B
:106830001346E7E713F8012B04F8012BF2E73023A6
:10684000021D19448370C170EFE72DE9F0479146AE
:106850001F468A6806460B690C46DDF82080934285
:10686000B8BF1346C9F8003091F8432012B1013384
:10687000C9F800302368990642BFD9F800300233C6
:10688000C9F80030256815F0060507D104F1190A8A
:10689000E368D9F800209B1AAB422BDC94F8433014
:1068A0002268003318BF0123920630D404F143025A
:1068B00039463046C047013023D023681A3454F893
:1068C0000E5C03F00603D9F800204FF00009042BFA
:1068D00054F8123C08BFAD1A54F80A2C14BF002516
:1068E00025EAE5759342C4BF9B1AED184D451AD1B0
:1068F000002008E00123524639463046C0470130A7
:1069000003D14FF0FF30BDE8F0870135C0E7E11853
:106910005A1C30200233224481F8430094F8451079
:1069200082F84310C2E70123224639463046C04769
:106930000130E6D009F10109D8E7034613F8012B2D
:10694000002AFBD1181A0138704770B50139044686
:1069500002B970BD234611F8015F561E03F8015BB2
:106960002DB91444A342F4D003F8015BFAE71C46A6
:106970003246EDE7F0B503787BB104462378204634
:10698000661C7BB14A1E631E12F8015F4DB113F8FD
:10699000017F3446AF42F7D0F0E70B78002B18BFE9
:1069A0000020F0BD1846FCE730B5141E05469BB02C
:1069B000184605DA8B234FF0FF302B601BB030BD3B
:1069C0004FF40273009104910246ADF80C3014BFED
:1069D00004F1FF33234669462846029305934FF698
:1069E000FF73ADF80E301E9BFEF7B6F8431CBCBF1C
:1069F0008B232B60002CE1D0009B00221A70DDE776
:106A000008B50620FEF79EF90120FEF7FFFE2DE9EE
:106A1000F74F036980460C69A342C0F28680013CAF
:106A200001F1140700F1140657F824504FEA840CC2
:106A300056F82400013506EB0C0307EB0C09019313
:106A4000B0FBF5F5A5B34FF0000A3846B646D3467D
:106A500050F8042B93B281454FEA124205FB03A381
:106A60004FEA134A9BB205FB02A2ABEB0303DEF82D
:106A700000B04FEA124A1FFA8BFB5B441FFA82FBFD
:106A8000DEF80020CBEB124202EB23429BB24FEA2E
:106A9000224B43EA02434EF8043BD9D256F80C305D
:106AA00033B9019B043B9E421A4632D3C8F81040CA
:106AB000404600F06CFA002827DB013530464FF0E5
:106AC000000C57F8041BD0F800E08BB2B9451FFA50
:106AD0008EF2ACEB030313444FEA1142C2EB1E42A9
:106AE00002EB23429BB24FEA224C43EA024340F8B6
:106AF000043BE6D256F8242006EB84032AB9043B73
:106B00009E421A460BD3C8F81040284603B0BDE891
:106B1000F08F1268043B002AC8D1013CC3E7126819
:106B2000043B002AEFD1013CEAE70020EEE770B514
:106B30004A1E68250E46554305F17401FDF78EF88F
:106B4000044640B1002105F16802C0E900160C308E
:106B5000A060FFF7B5FD204670BD2DE9F8438046E3
:106B6000894600F14804002614B93046BDE8F88390
:106B7000D4E90175013F01D52468F5E7AB89012B04
:106B800007D9B5F90E30013303D029464046C8472E
:106B900006436835EEE770B50E46B1F90E1096B0B3
:106BA000144600291D4607DA00232B60B3891A0614
:106BB00010D44FF480630EE06A46FEF7FFF8002819
:106BC000F2DB019A02F47042A2F500535A425A4194
:106BD0002A60EEE740230020236016B070BDC9B2E2
:106BE000024410B59042034601D1002303E01C7813
:106BF00001308C42F6D1184610BD7047704770B511
:106C0000456A04460E463DB91020FCF7D1FF60628C
:106C10000560C560C0E90155656AEB6883B1636AC8
:106C2000DB6853F82600B8B90121204601FA06F5C1
:106C30006A1D920000F074FA60B1C0E901650EE0CF
:106C400021220421204600F06BFA636AE860DB68C9
:106C5000002BE4D1002070BD026843F826200023F9
:106C6000C0E90333F7E770B5446A06460D463CB900
:106C70001020FCF79DFF70620460C460C0E901440D
:106C80003DB1736A6A68DB6853F82210296043F8E3
:106C9000225070BD2DE9F04101F1140C1F4606464B
:106CA0000C460D690023DCF80000013381B29D42DF
:106CB0004FEA104002FB01714FEA114789B202FB13
:106CC000007001EB00414FEA10474CF8041BEADC6E
:106CD000D7B1A368AB4212DC616830460131FFF7DF
:106CE0008EFF2269804604F10C0102320C309200C2
:106CF000FFF7C2FC214644463046FFF7B4FF04EBE1
:106D0000850301355F6125612046BDE8F081020CF5
:106D100003461204B2B90304102013F07F4F04BFDE
:106D20001B02083013F0704F04BF1B01043013F036
:106D3000404F04BF9B000230002B06DB5B0003D5F5
:106D4000013070470020E8E72020704703680146C3
:106D500013F007020BD0DA0723D4980747BF5B086C
:106D600001209B0802204CBF0B600B60704798B25B
:106D7000A8B91B0C102013F0FF0F04BF1B0A08302A
:106D80001A0704BF1B0904309A0704BF9B0802308E
:106D9000DA0702D45B0806D001300B60704710465A
:106DA000E9E7002070472020704710B50C4601210C
:106DB000FFF725FF01224461026110BD2DE9F74F65
:106DC00014460A69884623699A42BEBF0B46A0460C
:106DD0001C46D8F81070D8F80830D4F81090D8F8BD
:106DE000041007EB0906B342B8BF0131FFF707FFF4
:106DF00000F11405002205EB860E2B46734516D3D1
:106E000008F1140104F1140201EB870702EB890376
:106E10000093009B019293420CD8002E03DD5EF894
:106E2000043D002B5DD0066103B0BDE8F08F43F850
:106E3000042BE3E7B2F800B0BBF1000F23D0894682
:106E4000AC464FF0000859F8044BDCF800A0A3B2A0
:106E50004F451FFA8AFA0BFB03A34FEA144ADCF8EA
:106E6000004043444FEA14480BFB0A84E24604EB1B
:106E700013449BB24FEA144843EA04434AF8043BE4
:106E80002BD8CCF80480019B0432B3F802A0BAF1ED
:106E9000000F20D02B688946A8464FF0000BB9F8A8
:106EA00000C09BB2B8F802400AFB0C44C4465C44E4
:106EB00043EA04434CF8043B59F8043BB8F804B0E7
:106EC0001B0C4F450AFB03B303EB14434FEA134B70
:106ED00005D8C8F8043004359BE7D446B3E7E0464C
:106EE000DDE7013E99E72DE9F0470C464FEA621ACB
:106EF00007461646236949680AEB0309A36809F1A6
:106F00000105AB4232DB3846FFF779FE00238046AD
:106F100000F114011A4653452BDB2AEAEA7A04F100
:106F20001403206916F01F0201EB8A0103EB800CA9
:106F300025D0C2F1200E00201E688A4696403043BC
:106F40004AF8040B53F8040B9C4520FA0EF014D8B1
:106F5000486008B109F10205013D38462146C8F8EC
:106F60001050FFF780FE4046BDE8F08701315B001E
:106F7000C7E741F823200133CDE75146DCE7043968
:106F800053F8042B9C4541F8042FF9D8E4E7036932
:106F90000A699B1A30B50CD1920014301431841850
:106FA000114454F8045D51F8042D954203D005D3E3
:106FB0000123184630BDA042F3D3FAE74FF0FF3368
:106FC000F7E72DE9F0470D460746114614462846D7
:106FD000FFF7DDFF061E08D131463846FFF70FFEEA
:106FE0000123C0E90436BDE8F087A3BF23462C4641
:106FF00000260126A8BF1D4661683846FFF7FFFD41
:1070000005F11409C66004F11402266900F11401A7
:107010002B694FF0000E02EB860709EB830852F84C
:1070200004AB59F8045B1FFA8AF39446ACB2C84526
:107030007344A3EB04034FEA1544C4EB1A4404EB76
:1070400023449BB24FEA244E43EA044441F8044BE4
:10705000E5D8BC4504D351F8043D83B10661C2E7CD
:107060005CF8044BA2B27244131492B203EB1443C3
:1070700042EA03424FEA234E41F8042BE9E7013E7E
:10708000E9E72DE9F74359EC108BC9F30A540E4692
:1070900001211546FFF7B3FDC9F31303074634BBBF
:1070A0000193B8F1000327D002A840F8083DFFF78C
:1070B0004DFE0099F0B1019AC0F1200302FA03F3EA
:1070C000C2400B4301927B61019B002BBB6114BF4B
:1070D000022101213961C4B1A4F233440444C0F156
:1070E000350034602860384603B0BDE8F08343F4CF
:1070F0008013D5E77961E7E701A8FFF727FE019B39
:10710000012120307B613961E5E7A0F2324007EBD5
:10711000810330601869FFF7FAFDC0EB4110E1E729
:1071200038B502FB01F42146FCF798FD054618B17D
:1071300022460021FFF7C4FA284638BDF8B50746B5
:1071400014460E4621B91146BDE8F840FCF786BD4D
:1071500022B92546FCF734FD2846F8BD00F0EDF8CD
:10716000A0420FD221463846FCF778FD054600289C
:10717000F2D031462246FFF77FFA31463846FCF717
:107180001FFDE9E73546E7E72DE9F0478E688246BF
:107190000C4690469E42994637D88A8912F4906FE1
:1071A00031D02568022309696F1A656905EB450529
:1071B00095FBF3F509F101033B449D4238BF1D46A1
:1071C000530530D52946FCF749FD064650B90C2336
:1071D0004FF0FF30CAF80030A38943F04003A38189
:1071E000BDE8F0873A462169FFF746FAA38923F400
:1071F000906343F08003A38126613E446561ED1BEB
:1072000026604E46A5604E4500D94E463246414660
:107210002068FFF73CFAA36800209B1BA36023684B
:107220001E442660DCE72A46FFF788FF0646002852
:10723000E2D121695046FCF7C3FCC8E71F2938B5E5
:1072400004460D4604D9162303604FF0FF3038BDC5
:10725000426C12B152F821304BB9204600F016F8BA
:107260002A4601462046BDE83840FDF773BD012B94
:107270000AD0591C03D1162303600120E7E700243C
:10728000284642F8254098470020E0E7FEF780BAFC
:1072900010B50C46B1F90E10FDF7C4FD0028ABBFC8
:1072A000636DA3891B1823F48053ACBF6365A3816E
:1072B00010BD2DE9F0411F468B8905460C46DB05C4
:1072C000164605D502230022B1F90E10FDF798FDF0
:1072D000A3893246B4F90E10284623F48053A381C3
:1072E0003B46BDE8F041FDF747BD10B50C46B1F98E
:1072F0000E10FDF785FD431CA38915BF606523F4BF
:10730000805343F48053A38118BFA38110BDB1F90A
:107310000E10FDF743BD82B001B901A942B14BB1D6
:1073200013780B601278101C18BF012002B0704750
:107330001046FBE76FF00100F8E751F8043C181F16
:10734000002BBCBF0B58C018704749B1FF2A8DBF36
:107350008A230A700120036088BF4FF0FF30704716
:1073600008467047F8B500BFF8BC08BC9E46704799
:10737000F8B500BFF8BC08BC9E467047000000008E
:107380000080E03779C34143176E05B5B5B8934621
:10739000F5F93FE9034F384D321D30F94877825AED
:1073A0003CBF737FDD4F1575000000000000F03F0B
:1073B00000000000000024400000000000005940D0
:1073C0000000000000408F40000000000088C34023
:1073D00000000000006AF8400000000080842E4198
:1073E00000000000D01263410000000084D79741E4
:1073F0000000000065CDCD41000000205FA00242EA
:10740000000000E876483742000000A2941A6D425E
:10741000000040E59C30A2420000901EC4BCD64251
:1074200000003426F56B0C430080E03779C34143FC
:1074300000A0D8855734764300C84E676DC1AB4372
:10744000003D9160E458E143408CB5781DAF154490
:1074500050EFE2D6E41A4B4492D54D06CFF080446B
:10746000F64AE1C7022DB544B49DD9794378EA4480
:1074700028212121292048415244204641554C547D
:107480002028424F4F54292028212121290A000079
:107490000A3D3D3D20424F4F542048415244204632
:1074A00041554C5420444941474E4F535449432081
:1074B000424547494E203D3D3D0A0000417070481D
:1074C000616E646C65723A2025700A00554653520D
:1074D000203D3078253034580A000000424653528F
:1074E000203D3078253032580A0000004D4D46537B
:1074F000523D3078253032580A0000004846535239
:10750000203D3078253038580A0000003D3D3D20B0
:10751000424F4F542048415244204641554C54203C
:10752000444941474E4F5354494320454E44203D22
:107530003D3D0A0A000000000A282121212920538C
:10754000544F5050494E4720444556494345202802
:10755000212121290A00000028212121292053541A
:107560004F5050494E472044455649434520282115
:107570002121290A000000003A2D280A00000000FD
:10758000282121212920426C6F636B696E6720449A
:1075900045564943452028212121290A00000000A1
:1075A000282121212920526573657474696E672032
:1075B0004445564943452028212121290A0000003D
:1075C0000A0A00002D2D2D2D2D2D2D2D2D2D2D2D8B
:1075D0002D2D2D2D2D2D2D2D2D2D2D2D2D2D2D2DDB
:1075E0002D2D2D2D2D2D2D2D2D2D2D2D2D2D2D2DCB
:1075F0002D2D2D2D2D2D2D2D2D2D2D2D2D2D2D2DBB
:107600002D2D2D2D2D2D2D2D2D2D2D2D2D2D2D2DAA
:107610002D2D2D0A0000000032000000312E342EE6
:10762000300000006170702D626F6F742D6E726695
:10763000393136302D736563000000005374617278
:107640007465642025732076257320545A25730AA7
:1076500000000000526573657420526561736F6E9F
:107660003A202573202830782578290A0000000068
:10767000436F6D70696C65643A204A756E203235CF
:1076800020323032302031353A33313A35310A0048
:10769000446576696365206669726D7761726520FD
:1076A00056657273696F6E733A0A0000283129209B
:1076B00025730A002832292025730A00283329203F
:1076C00025730A000A426F6F74696E67206D6169E5
:1076D0006E2061707020696D6167652E2E2E0A0024
:1076E00077C295F360D2EF7F3552500F2CB6798078
:1076F000282121212920554E48414E444C45442003
:107700004952512028424F4F542920282121212914
:107710000A00000055465352203D30782530345839
:107720000A00000042465352203D3078253032583E
:107730000A0000004D4D4653523D307825303258F6
:107740000A00000048465352203D30782530385812
:107750000A0000000A28212121292053544F5050AB
:10776000494E472044455649434520282121212997
:107770000A00000028212121292053544F5050494C
:107780004E47204445564943452028212121290AB6
:10779000000000003A2D280A0000000028212121C5
:1077A00029205265736574696E67204445564943C4
:1077B000452028212121290A000000004E4D495F63
:1077C00048616E646C6572004D656D6F72794D61D4
:1077D0006E6167656D656E745F48616E646C65723D
:1077E000000000004275734661756C745F48616EFD
:1077F000646C6572000000005573616765466175D1
:107800006C745F48616E646C6572000053656375EB
:1078100072654661756C745F48616E646C65720078
:1078200044656275674D6F6E5F48616E646C65722A
:1078300000000000486172644661756C745F4861C5
:107840006E646C65720000005356435F48616E645D
:107850006C65720050656E6453565F48616E646C6F
:10786000657200005379735469636B5F48616E649D
:107870006C657200525443305F49525148616E64E6
:107880006C657200454755305F49525148616E64DE
:107890006C657200454755315F49525148616E64CD
:1078A0006C6572004950435F49525148616E646C87
:1078B000657200005350555F49525148616E646CC7
:1078C00065720000434C4F434B5F504F5745525F2A
:1078D00049525148616E646C657200004750494FCF
:1078E0005445305F49525148616E646C65720000C6
:1078F00053414144435F49525148616E646C657223
:107900000000000054494D4552305F4952514861D2
:107910006E646C657200000054494D4552315F49F8
:10792000525148616E646C657200000054494D45C7
:1079300052325F49525148616E646C6572000000BA
:107940005744545F49525148616E646C657200003F
:10795000454755325F49525148616E646C6572000B
:10796000454755335F49525148616E646C657200FA
:10797000454755345F49525148616E646C657200E9
:10798000454755355F49525148616E646C657200D8
:1079900050574D305F49525148616E646C657200BA
:1079A00050574D315F49525148616E646C657200A9
:1079B00050574D325F49525148616E646C65720098
:1079C00050574D335F49525148616E646C65720087
:1079D00050444D5F49525148616E646C65720000BD
:1079E0004932535F49525148616E646C65720000C0
:1079F0004650555F49525148616E646C6572000093
:107A00004B4D555F49525148616E646C6572000080
:107A100043525950544F43454C4C5F495251486171
:107A20006E646C65720000003E3D3D484558494E0D
:107A3000464F3D3D3E0000003C3D3D484558494EC7
:107A4000464F3D3D3C000000506F7765722D6F6ED4
:107A5000202F2042726F776E6F7574006E524553FF
:107A600045542070696E2070756C6C6564206C6F75
:107A7000770000005761746368646F6720747269EF
:107A80006767657265640000536F6674776172653D
:107A900020726573657400005265736574206672A8
:107AA0006F6D20435055206C6F636B2D7570206493
:107AB000657465637465640057616B6575702066F5
:107AC000726F6D2053797374656D204F4646206D3B
:107AD0006F646520287369676E616C2066726F6DD4
:107AE000204750494F290000656E746572696E67C2
:107AF00020646562756720696E746572666163658E
:107B0000206D6F64650000006E524553455420702F
:107B1000696E2070756C6C6564206C6F77202B200B
:107B2000536F6674776172652072657365740000C7
:107B30006F746865720000006E6F72657365745FC4
:107B40006C697665203D3D202828766F6964202A7F
:107B5000293029002F686F6D652F6B726174656E17
:107B60006B6F2F63706174682F7372632F67697412
:107B70006875622E636F6D2F6C6F6261726F2F6814
:107B8000616C2D6E7266393136302F706572697096
:107B9000682F68616C5F72657365742E6300000006
:107BA0006E6F72657365745F6C69766500000000C6
:107BB0000A0A53595354454D20495320474F494EC3
:107BC0004720464F52205245424F4F54210A000051
:107BD00046696E616C20776F7264733A2025730A70
:107BE00000000000756172742D3E696E69740000BA
:107BF0002F686F6D652F6B726174656E6B6F2F638D
:107C0000706174682F7372632F6769746875622E70
:107C1000636F6D2F6C6F6261726F2F68616C2D6E78
:107C20007266393136302F7065726970682F6861FD
:107C30006C5F756172742E630000000021226E6F0C
:107C40007420737570706F727465642075617274DE
:107C500020646174616C656E2122000021227769C5
:107C6000746820646174616C656E203D2037206FFC
:107C70006E6C79206576656E20706172697479200A
:107C8000697320706F737369626C65212200000054
:107C9000756172745F64697361626C6500000000F5
:107CA000756172745F696E69743200007561727417
:107CB0005F70757461000000FF8FFFFFFF8FFFFF93
:107CC000FE8FFFFFFE8FFFFFFD8FFFFFFC8FFFFF8B
:107CD000FC8FFFFF4661696C20746F2061637175D2
:107CE000697265206D757465780A00004661696C7B
:107CF00020746F2072656C65617365206D757465A5
:107D0000780A00004661696C20746F20696E6372A6
:107D10006561736520504D20636F756E7465720ADE
:107D2000000000004661696C20746F206465637216
:107D30006561736520504D20636F756E7465720ABE
:107D400000000000436F756C64206E6F74206C6FD0
:107D5000636B20706F7765722073617665206D7537
:107D60007465780043616E277420696E6974696177
:107D70006C697A65206D757465782C207761732045
:107D80004E554C4C0D0A000043616E277420756EF1
:107D90006C6F636B206D757465782C207761732030
:107DA0004E554C4C0D0A00002E2E2E000A000000ED
:107DB0002E2E2E0A00000000253032582000000030
:107DC0002020205F5F202020202020205F0A00004C
:107DD00020202F202F20205F5F5F207C207C5F5F92
:107DE0002020205F5F205F205F205F5F205F5F5F5C
:107DF0000A000000202F202F20202F205F205C7CF5
:107E000020275F205C202F205F60207C20275F5F81
:107E10002F205F205C200A002F202F5F5F7C20280E
:107E20005F29207C207C5F29207C20285F7C207CAF
:107E3000207C207C20285F29207C0A005C5F5F5F1B
:107E40005F2F5C5F5F5F2F7C5F2E5F5F2F205C5F2B
:107E50005F2C5F7C5F7C20205C5F5F5F2F0A0000EF
:107E600048000020000000000000000000000000AA
:107E70000000000000000000000000000000000002
:107E800000000000000000000000000000000000F2
:107E900000000000000000000000000000000000E2
:107EA00000000000000000000000000000000000D2
:107EB00000000000000000000000000000000000C2
:107EC0000000000005000000190000007D00000017
:107ED0002C2066756E6374696F6E3A20006173734F
:107EE000657274696F6E2022257322206661696C49
:107EF00065643A2066696C6520222573222C206C0B
:107F0000696E65202564257325730A00232D302BA7
:107F10002000686C4C0065666745464700494E4640
:107F200000696E66004E414E006E616E003000309A
:107F300031323334353637383941424344454600CF
:107F400030313233343536373839616263646566CF
:107F500000496E66696E697479004E614E00430097
:107F6000504F534958002E00002020202020202070
:107F700020202828282828202020202020202020D9
:107F800020202020202020202088101010101010E9
:107F90001010101010101010100404040404040435
:107FA00004040410101010101010414141414141CF
:107FB00001010101010101010101010101010101B1
:107FC00001010101101010101010424242424242C1
:107FD0000202020202020202020202020202020281
:107FE0000202020210101010200000000000000029
:107FF0000000000000000000000000000000000081
:108000000000000000000000000000000000000070
:108010000000000000000000000000000000000060
:108020000000000000000000000000000000000050
:108030000000000000000000000000000000000040
:108040000000000000000000000000000000000030
:108050000000000000000000000000000000000020
:108060000000000000000000000000000000000010
:10807000388BFF7F010000000090D0033400002007
:108080004000002038000020300000200C000020BC
:1080900000000000D136010029370100013701003E
:1080A000453701000537010030B9002024B9002010
:1080B0002CB900200000000028B900204800002052
:1080C00000000000847E0100A47E0100647E0100A7
:1080D00000000000000000000000000000000000A0
:1080E0000000000000000000000000000000000090
:1080F0000000000000000000000000000000000080
:10810000000000000000000000000000000000006F
:10811000000000000000000000000000000000005F
:10812000430000000000000000000000000000000C
:10813000000000000000000000000000000000003F
:1081400043000000000000000000000000000000EC
:10815000000000000000000000000000000000001F
:1081600043000000000000000000000000000000CC
:1081700000000000000000000000000000000000FF
:1081800043000000000000000000000000000000AC
:1081900000000000000000000000000000000000DF
:1081A000430000000000000000000000000000008C
:1081B00000000000000000000000000000000000BF
:1081C000430000000000000000000000000000006C
:1081D000000000000000000000000000000000009F
:1081E000430000000000000000000000000000004C
:1081F000000000000000000000000000000000007F
:108200004B7301001773010000000000687F01003C
:10821000667F01000B7F01000B7F01000B7F0100D7
:108220000B7F01000B7F01000B7F01000B7F010022
:108230000B7F01000B7F0100FFFFFFFFFFFFFFFF30
:10824000FFFFFFFFFFFF00000100415343494900CA
:10825000000000000000000000000000000000001E
:1082600000000000000000000000415343494900A5
:1082700000000000000000000000000000000000FE
:108280000000000000000000000000008D0B010055
:10829000690B01000769980010002000A07B104DB9
:1082A000870E49C0D15ECC5B6E34D3F5ADB40DF80A
:1082B000C56A58DA71B323365E8B2F500100200057
:1082C000EA96568ABEDA9F408B0729962E74850857
:1082D000126A0FC92B5262E833813A5E4D5E352136
:1082E000220048003044022068BC7F45A92E433458
:1082F0004EE5EF7F14B708069C2EB0A21139C2FBE1
:10830000A00EB6A2335DA92F02204DBC3B6E53C711
:1083100065A0ED42F354FC6D3311855572B5DCAFA9
:0C832000C97DF0EB3C010A2AEF4600008A
:020000040002F8
:1079D000FFFFFFFFFFFFFFFFFFFFFFFFFFFFFFFFB7
:1079E000FFFFFFFFFFFFFFFFFFFFFFFFFFFFFFFFA7
:1079F000FFFFFFFFFFFFFFFFFFFFFFFFFFFFFFFF97
:107A0000FFFFFFFFFFFFFFFFFFFFFFFFFFFFFFFF86
:107FF00077C295F360D2EF7F3552500F2CB679805F
:020000040003F7
:100000003DB8F39600000300200000005089030073
:1000100000000000000506000000000000000000D5
:10002000DEADC0DEDEADC0DEDEADC0DEDEADC0DE2C
:10003000DEADC0DEDEADC0DEDEADC0DEDEADC0DE1C
:10004000DEADC0DEDEADC0DEDEADC0DEDEADC0DE0C
:10005000DEADC0DEDEADC0DEDEADC0DEDEADC0DEFC
:1004000000FC032081D1030021E8030099E80300E8
:1004100035E8030049E803005DE8030071E80300E4
:10042000000000000000000000000000710903004F
:1004300085E8030000000000D1080300BDE80300C8
:10044000000000000000000000000000D1E80300F0
:1004500000000000E5E803000000000000000000CC
:10046000E1E40300F5E40300ED9205001F940500AC
:1004700000000000F9E803000DE9030021E9030092
:1004800035E9030049E90300000000000000000016
:100490004D310300B5DC0300000000000000000047
:1004A0005DE9030000000000000000004D3C040076
:1004B0009D3C040071E9030085E9030099E903000C
:1004C000ADE90300C1E90300D5E90300E9E9030050
:1004D000FDE903000000000011EA03000000000035
:1004E00025EA03000000000081B8040000000000BD
:1004F00039EA0300000000000000000000000000D6
:100500000000000041D703000000000000000000D0
:1005100000000000000000000000000000000000DB
:10052000000000004DEA0300000000000000000091
:1005300000000000000000000000000000000000BB
:1005400061EA03000000000000000000000000005D
:10055000000000000000000000000000000000009B
:10056000000000000000000000000000000000008B
:10057000000000000000000000000000000000007B
:10058000000000000000000000000000000000006B
:100800003E3D3D484558494E464F3D3D3E61707026
:100810002D6E7266393136302D776D6275732076A4
:10082000302E352E362B68773120545A3220284A04
:10083000756C20313420323032302031383A343740
:100840003A3536293C3D3D484558494E464F3D3D99
:100850003C00FFFFFFFFFFFFFFFFFFFFFFFFFFFF6A
:100860000B4A136818680EC80A4C216082F30B8883
:10087000022181F31488203080F30988BFF36F8F41
:10088000184700BFAFF30080AFF30080AFF30080E4
:10089000F8C90220F4C9022000BF00BF0000000018
:1008A00007480068006880F3088862B661B6BFF345
:1008B0004F8FBFF36F8F02DF00BF00BFAFF3008029
:1008C00008ED00E000BF00BF0000000000000000D5
:1008D000EFF30981234A106878B107B5DFF7B0F963
:1008E0000FBC9E465A0608D51D4B1A680C3911607C
:1008F000EFF30B8273460DC110E0194B1A681EF01E
:10090000100F08BF21ED108A2C3911600C3181E8DD
:10091000F00FEFF30B8273460C390DC172B603F082
:1009200075FF62B60E4A136819680DC982F30B8809
:100930009E460C4A106048B10AB4DFF77DF90ABC44
:100940009E465A0602D581F309887047B1E8F00F38
:100950001EF0100F08BFB1EC108A81F309887047B0
:10096000F8C90220F4C9022000BF00BF0000000047
:100970001EF0040F0CBFEFF30880EFF30980044969
:10098000084700BFAFF30080AFF30080AFF30080F3
:10099000D532030000BF00BF98B500AF0C4B012259
:1009A0009A600C4A4FF000034FF00004C2E9003493
:1009B000094A05A4D4E90034C2E9003428F005FC52
:1009C00000BF98BDAFF3008080436D380000000089
:1009D0000050014038C7012040C70120000000003E
:1009E0002DE9F04F456A97B0044606910B92129399
:1009F000DDF8808057EC106BCDE900673DB9102021
:100A000014F004FC60620560C560C0E90155636ACA
:100A1000196851B15A680123204693404A608B609F
:100A20002EF012F8636A00221A603B1EB7BF23F053
:100A30000043002301220193ACBFC8F80030C8F87E
:100A40000020AF4BDDF8048033EA080314D142F2F2
:100A50000F73129A1360009B23B9C8F31300002888
:100A600000F03E85219BDFF8ACB2002B00F0408502
:100A70000BF1030300F03ABDDDE90067002200231B
:100A80003046394613F0F2FF814668B10123129ACD
:100A90001360219B002B00F020859A4B219A03F1D3
:100AA000FF3B136000F024BDC8F30A5514AA15A932
:100AB000204647EC106B2EF0D5F90490002D7AD02B
:100AC000C7F31303B246A5F2FF35CDF84C9043F0BF
:100AD0007F5B4BF4401B00228B4B5046594613F072
:100AE000A5FB81A3D3E9002313F058FD80A3D3E92C
:100AF000002313F09DFB06460F46284613F0E4FC46
:100B00007DA3D3E9002313F049FD02460B4630468E
:100B1000394613F08DFB06460F4616F06DFD002298
:100B2000824600233046394613F0AAFF48B15046AA
:100B300013F0CAFC32463B4613F098FF08B90AF19D
:100B4000FF3ABAF1160F57D8704901EBCA01DDE937
:100B50000023D1E9000113F0B1FF00284ED00AF1C3
:100B6000FF3A00230F93149B5D1BB5F1010849BFA9
:100B7000C5F1010300234FF00008059358BF05930A
:100B8000BAF1000F3CDB0023D044CDF838A0079326
:100B9000069B092B00F28E80052BC5BF043B002568
:100BA00001250693069B023B032B00F28F80DFE8B2
:100BB00003F07D7F3171DDE914531D4405F23240AD
:100BC000202813DDC0F14000009B08FA00F805F270
:100BD000124023FA00F048EA000013F065FC0123FC
:100BE0008246A1F1F87B013D139374E7C0F1200028
:100BF000009B03FA00F0F0E70123B3E70F90B2E7A0
:100C0000059BA3EB0A030593CAF100030793002396
:100C10000E93BDE701230A930B9B002B59DD9946E8
:100C200002930022666A7260042202F11400716865
:100C3000984253D920462DF0D3FE636AB9F10E0FC6
:100C40003060D3F800B000F2E880002D00F0E580BD
:100C5000BAF1000F9DED007B8DED107B76DD0AF083
:100C60000F032A4A4FEA2A1602EBC303F00693ED5C
:100C7000007B8DED087B67D5254B06F00F0603251D
:100C8000D3E90823DDE9100113F0B2FDCDE900013D
:100C90001F4F4EE001230A930B9B534403F10109BC
:100CA00002934B46012BB8BF0123BAE70023B2E7FA
:100CB0000023F0E7012500230A9506934FF0FF3348
:100CC00000220293994612230B92AAE701230A936A
:100CD000F4E70123029399461A46F5E701315200E1
:100CE0007160A2E7AFF3008061436F63A787D23FD3
:100CF000B3C8608B288AC63FFB799F501344D33F0B
:100D00000000F07F2E8606000000F83FE005060098
:100D1000B805060013860600F10708D50135DDE9A0
:100D20000801D7E9002313F039FCCDE9080176105A
:100D30000837002EF0D1DDE90823DDE9000113F0CA
:100D400057FDCDE900011AE00225A1E700F0A080DF
:100D5000CAF100069F4BA04F022506F00F02361184
:100D600003EBC203DDE91001D3E9002313F016FC05
:100D70000023CDE90001002E7FD1002BE1D10F9B94
:100D8000002B00F087800022944BDDE9006730469D
:100D9000394613F075FE00287CD0B9F1000F79D0E8
:100DA000029B002B35DD0AF1FF3339460022304625
:100DB000089301358A4B13F0F1FB029FCDE9000146
:100DC000284613F081FBDDE9002313F0E7FB002246
:100DD000844B13F02DFA0546A1F15076002F5DD11A
:100DE0000022814BDDE9000113F020FA2A46334648
:100DF000CDE9000113F062FE002840F087822A4608
:100E000006F10043DDE9000113F03AFE002840F04E
:100E10007B82DDE91023CDE90023159B002BC0F276
:100E20004F81BAF10E0F00F34B816A4B03EBCA03FB
:100E300093ED007B0B9B002B8DED027B80F2D88025
:100E4000B9F1000F00F3D48040F05D820022664BC0
:100E50004F464E4651EC170B13F0A0FBDDE9002383
:100E600013F022FE002840F0338231230BF10105FC
:100E70000AF1010A8BF800302EE2F20705D50135A0
:100E8000D7E9002313F08AFB01237610083772E7B5
:100E9000022574E7CDF820A04F4691E74D4B03EBB8
:100EA000C70353E902010A9B002B47D002460B46B9
:100EB00000204E4913F09CFC2A465D46334613F051
:100EC000B5F9CDE90C01DDE9000116F095FB064608
:100ED00013F0FAFA024630360B46DDE9000113F052
:100EE000A5F905F8016BDDE90C23CDE9000113F04C
:100EF000C7FD002862D100203849DDE9002313F046
:100F000095F9DDE90C2313F0BBFD002840F0B78014
:100F1000A5EB0B039F427FF77CAF0022304BDDE94E
:100F20000C0113F03BFB00222D4BCDE90C01DDE958
:100F3000000113F033FBCDE90001C4E72A46334634
:100F40000BEB07055E4613F029FBCDE90C01DDE94B
:100F5000000116F051FB074613F0B6FA024630378F
:100F60000B46DDE9000113F061F906F8017BAE42A2
:100F70004FF00002CDE9000125D11C4BDDE90C0149
:100F800013F056F902460B46DDE9000113F096FD19
:100F9000002874D100201549DDE90C2313F046F92F
:100FA00002460B46DDE9000113F06AFD00283FF41C
:100FB00030AF15F8013C6A1E302B02D0DDF820A0BE
:100FC0004BE01546F5E7064B13F0E8FACDE90001D2
:100FD000BDE700BFE0050600B80506000000F03FD1
:100FE0000000244000001C40000014400000E03FCE
:100FF000DDE900675D4630463946DDE9022313F03E
:10100000F7FB16F0F9FA804613F05EFADDE90223E9
:1010100013F0C4FA0246304608F130060B46394652
:1010200013F004F905F8016BA5EB0B0602460B461D
:10103000B14538D113F0FCF806460F46DDE902232E
:1010400013F03CFDC8B930463946DDE9022313F000
:101050000DFD10B118F0010F0FD1049920462DF0AD
:10106000F3FC0023129A2B700AF101031360219BF9
:10107000002B00F03D821D603AE2CDF820A015F86B
:10108000012C6B1E392A08D19B450AD1089B0133DC
:10109000089330238BF800305B461A7801321A70BF
:1010A0008CE71D46EBE700229A4B13F077FA0022FB
:1010B000002306460F4613F0D9FC00289BD0CCE74E
:1010C0000A9A002A00F08B80069A012A6EDC139A95
:1010D000002A67D003F23343079F059D059A01213B
:1010E000204698441A4405922DF050FD0646002DE6
:1010F0000CDDB8F1000F09DD45452B46059AA8BF68
:101100004346D21AED1AA8EB03080592079BEBB1F0
:101110000A9B002B67D08FB131463A46204615F026
:1011200057FE049A0146064620462DF038FD0499E4
:10113000089020462DF088FC089B0493079BDA1B3F
:1011400004D00499204615F043FE04900121204666
:101150002DF01CFD0E9B0746002B00F0CD811A469A
:101160000146204615F034FE069B0746012B40DC65
:10117000009B002B39D1019BC3F31303002B36D105
:10118000019B23F000431B0D1B052BB1059B08F1B0
:10119000010801330593012307930E9B002B2AD1ED
:1011A000012030E0149BC3F1360395E7079B09F15A
:1011B000FF37BB42B7BF079BDF1B0797FA1ABFBFBA
:1011C0000E9B00279B180E93B9F1000FB3BF059B30
:1011D0004B46059DA3EB0905B8BF00237EE7079F9B
:1011E000059D0A9E83E7079AABE70023D4E7009B9F
:1011F000D2E7002307933B6907EB830318692DF0BF
:1012000077FCC0F12000404410F01F0047D0C0F12F
:101210002003042B3BDDC0F11C00059B0544034467
:1012200080440593059B002B05DD1A460499204652
:101230002DF04AFD0490B8F1000F05DD3946424615
:1012400020462DF041FD07460F9B53B339460498C5
:101250002DF08EFD002824DA00230A22049920466E
:101260002DF009FC0A9B0AF1FF3A0490002B00F0D4
:101270004A81002331460A2220462DF0FCFB029BC6
:101280000646002B4EDC069B022B4BDD11E0C9D03D
:101290001C33059A1A441D4498440592C2E703463C
:1012A000F6E7B9F1000F37DC069B022B34DDCDF8F1
:1012B0000890029B63B93946052220462DF0DBFBDE
:1012C0000146074604982DF053FD00283FF7CDADA9
:1012D0000B9B5D466FEA030A4FF000093946204632
:1012E0002DF0B2FB002E3FF4B8AEB9F1000F05D0DF
:1012F000B14503D0494620462DF0A6FB3146204695
:101300002DF0A2FBA9E600273E46E1E7DDF820A08C
:101310003E46AAE5000024400A9BCDF80890002B29
:1013200000F0F880002D05DD31462A4620462DF0DC
:10133000CBFC0646079B002B4CD0716820462DF055
:101340004FFB3269054606F10C0102320C30920067
:101350002CF05CFF0122294620462DF0B5FC009BB5
:10136000B1460646CDF814B003F0010307933946A1
:1013700004982DF07AFA4946054600F130080498A1
:101380002DF0F6FC32460090394620462DF00AFD3D
:10139000C368024603BB0146089004982DF0E8FCA0
:1013A000089A03461146204608932DF04DFB089BF2
:1013B000A3B9069A92B9079A82B9B8F1390F29D020
:1013C000009B002B01DD05F13108059B5D1C83F8B6
:1013D000008083E73046C2E70123E3E7009A002A52
:1013E00004DB24D1069A12BB079A02BB002BECDD6A
:1013F0000122049920462DF067FC394604902DF017
:10140000B7FC002803DCE0D118F0010FDDD0B8F103
:10141000390FD8D1059B059A5D1C3923137015F837
:10142000013C6A1E392B4ED00133137056E7059AE2
:10143000002B02F1010506DDB8F1390FEAD008F101
:101440000108059BC3E7A5EB0B03029A05F8018C85
:10145000934221D000230A22049920462DF00BFB51
:10146000B14504904FF000034FF00A024946204670
:1014700005D12DF000FB81460646059577E72DF056
:10148000FAFA3146814600230A2220462DF0F3FA6B
:101490000646F2E74FF000090122049920462DF09C
:1014A00013FC394604902DF063FC0028B7DC02D110
:1014B00018F0010FB3D115F8013C6A1E302B7FF4F0
:1014C0000DAF1546F7E7934505D131230AF1010A1F
:1014D0008BF8003002E71546A1E7DFF864B007E0BB
:1014E000219BDFF860B01BB10BF10803219A136058
:1014F000584617B0BDE8F08F069B012B7FF738AE3A
:101500000E9B07934CE6029B002B03DC069B022BF1
:101510003FF7CFAE5D46394604982DF0A6F900F1AD
:101520003008029A05F8018BA5EB0B039A42B1DD56
:1015300000230A22049920462DF09DFA0490EAE740
:101540002D8606000A86060010B5054C237833B9AF
:10155000044B13B1044800E000BF0123237010BD09
:1015600058C70120000000003486060008B5034B70
:101570001BB10349034800E000BF08BD00000000A4
:101580005CC7012034860600154B002B08BF134BA7
:101590009D46A3F5803A00218B460F461348144A16
:1015A000121A2CF057FE0F4B002B00D098470E4B11
:1015B000002B00D098470020002104000D000D48AA
:1015C000002802D00C4800E000BF13F0EDFD200021
:1015D000290001F075FC13F06FFC00BF000008004B
:1015E00000FC0320000000000000000050C30120A8
:1015F000E8EE0220000000000000000080B58EB080
:1016000002AF27F083F8F86205F03CF9B862F86A97
:1016100021F0BAFE0346B96A184611F023F9B86AF8
:1016200006F0C8FE38460C4B00930C4B0C4A0321C5
:1016300000F064F83B461946B86A05F009FA3B46E3
:10164000184621F0ADFEB96AF86A0BF07BF800BFCE
:101650003037BD4680BD00BFF8060600A80606006C
:10166000EC06060080B584B000AF27F04FF8B860F4
:1016700005F008F978600023FB73FFF7BFFFBB6834
:101680001B6810331B68FA21B8689847786805F022
:10169000B5FAB86821F078FE0346144A796818460E
:1016A00011F028FA034683F00103DBB2002B01D0CE
:1016B0000123FB730E49786806F000FF034683F0B0
:1016C0000103DBB2002B01D00123FB73FB7B002B5A
:1016D00008D008480EF004F8074A41F28831B8688B
:1016E0000BF086F800BF1037BD4680BD74C70120DF
:1016F00098C70120080706001C07060080B584B0C3
:1017000000AFF860B9607A603B60FB6800221A7035
:10171000FB68BA685A60FB687A689A60FB683A6846
:10172000DA60FB681033184621F04DFEFB681C336D
:10173000184621F048FEB969F86822F06AFE0346AF
:1017400083F00103DBB2002B07D0796809480DF064
:10175000C7FF2021084807F0A5F8FB681C33BA69C9
:101760001946F86804F036FDFB6818461037BD4688
:1017700080BD00BF2C0706005807060080B483B068
:1017800000AF7860034B18460C37BD465DF8047B0C
:10179000704700BF0025844080B584B000AF034689
:1017A000FB71084B1B68002B07D0064B186807F12C
:1017B0000C02F91D002301F0EDFF00BF1037BD46FC
:1017C00080BD00BFA8C7022080B584B000AF03462B
:1017D000FB714FF40073BB600023FB60FB79232B8C
:1017E0000BD1224B00221A60204B1B685A1C1F4948
:1017F0000A601F49FA79CA5433E01C4B1B68002B5E
:101800002FD01A4B1B68B3F5007F03D3174B002270
:101810001A6026E0FB790A2B1BD1144B1B68144A73
:101820000021D154114B1B68142B0ADD03221149EE
:101830000F482CF0DCFC0346002B02D10E4BFB6062
:1018400003E00B490D480DF04BFF084B00221A60D6
:1018500007E0064B1B685A1C04490A600449FA79E0
:10186000CA54FB6818461037BD4680BDB4C9022073
:10187000B0C7022094070600B3C7022098070600ED
:1018800090B58BB004AF0346FB711B237B611C2317
:101890003B611D23FB603D4B1B6807F10B010022E0
:1018A000184601F0EDFF0346012B0CBF0123002376
:1018B000DBB2002B00D0EEE7002303933B690293D9
:1018C0007B69019307230093012308224E214FF4E3
:1018D00096400CF019FE2E480CF060FE052021F019
:1018E00095FF052021F0A4FF1A2021F08FFF1A2078
:1018F00021F09EFFF86821F089FFF86821F098FF39
:10190000642002F0C5FB052021F0A7FF1A2021F07A
:10191000A4FFFB79012B03D11E4B53221A7002E066
:101920001C4B43221A70194B1B6807F10A0142F243
:101930001072184602F04EF90346012B0CBF01232A
:101940000023DBB2002B1BD0124B1B7818460CF087
:1019500035FE4FF4487002F09BFB0E4B1B78184687
:101960000CF02CFE0C4B1C6802F0BCFD0246002360
:10197000009300230121204603F0DEFD012300E057
:10198000002318461C37BD4690BD00BFA8C70220E3
:101990009917030040C30120ACC7022080B582B074
:1019A00002AF0C4B186841F28833009300230022E9
:1019B000032103F0C1FD642002F06AFB0CF0E4FD9A
:1019C000052021F035FF1A2021F032FF00BFBD466F
:1019D00080BD00BFACC7022080B5DAB002AF3B1DAE
:1019E000186002F07FFDC7F854013B1DD7F8542161
:1019F0001B681344C7F850313B1D1B68C7F85C31A6
:101A00004FF49673C7F84C31D7F85C31002B00F0D7
:101A10004981A74B1B6807F23B11D7F85C21184698
:101A200001F02EFF0346012B0CBF01230023DBB284
:101A3000002B00F0368197F83B311846FFF7C4FEC3
:101A4000C7F84801D7F84831002B00F02181D7F8BA
:101A500048012CF0C2FD03465B08C7F84431D7F8B3
:101A60004431B3F5967F06D9D7F8441191480DF06B
:101A700037FE002317E107F10C03D7F84821D7F808
:101A80004411184628F086FF0246D7F844319342A5
:101A900014BF01230023DBB2002B09D086480DF0D0
:101AA0001FFED7F8481185480DF01AFE0023FAE012
:101AB00007F10C03184628F09AFE0346A7F84231B6
:101AC00007F10C039B7887F8413107F10C03DB78B1
:101AD00087F8403197F84131432B0FD097F84131C7
:101AE000542B0BD097F84131532B07D097F8413145
:101AF000194673480DF0F4FD0023D4E097F8403107
:101B0000412B0BD097F84031422B07D097F840314A
:101B100019466C480DF0E4FD0023C4E097F840310D
:101B2000422B0CD197F84131432B03D1032387F883
:101B30005B3117E064480DF0D3FD0023B3E097F864
:101B40004131432B03D1022387F85B310AE097F838
:101B50004131542B03D1042387F85B3102E0012388
:101B600087F85B3197F85B31032B0FD107F10C033A
:101B70000433D7F84421D2B2043AD2B211461846FF
:101B80000FF0B0FD034687F85A310EE007F10C0361
:101B90000433D7F84421D2B2043AD2B211461846DF
:101BA0000FF038FD034687F85A3197F85A3183F021
:101BB0000103DBB2002B04D044480DF091FD00235B
:101BC00071E008200DF07AFEC7F83C01D7F83C31EF
:101BD000002B04D13E480DF083FD002363E0D7F8CD
:101BE00044010DF06BFE0246D7F83C311A60D7F87D
:101BF0003C311B68002B08D1D7F83C010DF040FEAA
:101C000034480DF06DFD00234DE0D7F84431DBB2D0
:101C1000043BDAB2D7F83C311A71D7F83C31B7F847
:101C20004221DA80D7F83C3197F85B215A71D7F816
:101C30003C31186807F10C030433D7F83C211279C2
:101C400019462CF0E3FA07F10C0304221946224846
:101C50000DF000FE97F8411197F84021D7F83C317C
:101C6000B3F906301846D7F83C311B790093034688
:101C70001A480DF035FDD7F83C311968D7F83C31DA
:101C80001B791A4616480DF0E5FDD7F83C310AE0FD
:101C900002F028FC0246D7F850319B1AC7F85C3195
:101CA000B2E600BF0023184607F5B077BD4680BDF9
:101CB000A8C70220C8070600F00706001C08060097
:101CC0002C080600440806005C080600840806008C
:101CD00098080600B0080600C8080600D8080600E4
:101CE0001809060080B582B000AF7860044B1B78FD
:101CF00018460CF063FC00BF0837BD4680BD00BF2E
:101D000040C3012080B584B000AF1B480DF0E8FC53
:101D100026F0FCFCB860B86821F036FB7860174804
:101D20000DF0DEFC0021786811F0A0FB002178683E
:101D300010F0A2FA0023FB60FB68632B11DC104B50
:101D4000D3F84034002B0CBF01230023DBB2002B5F
:101D500006D10A2002F09CF9FB680133FB60EBE737
:101D600000BF06F0F9FC4FF47A7002F091F900BF61
:101D70001037BD4680BD00BF2C0906004C09060087
:101D80000050004080B584B000AFF860B9607A6060
:101D90003B60BA683B681344B3F5803F04D340F21C
:101DA0002711074806F07EFDBB68064A13443A68CF
:101DB000796818462CF02AFA00BF1037BD4680BD5E
:101DC00068090600A8C7012080B483B000AF78601E
:101DD000034B18460C37BD465DF8047B704700BFC7
:101DE000E938050080B584B000AFF860B9607A606A
:101DF0003B60BA683B681344B3F5803F04D34FF4AB
:101E00009671074806F04EFDBB68064A13443A68CF
:101E1000194678682CF0FAF900BF1037BD4680BD2E
:101E200068090600A8C7012080B483B000AF7860BD
:101E3000034B18460C37BD465DF8047B704700BF66
:101E40000739050080B483B000AF7860034B1846B3
:101E50000C37BD465DF8047B704700BF3D39050077
:101E6000B0B59CB006AF3871397058480DF038FCE9
:101E700026F04CFC0346184621F093FC786526F0CA
:101E800045FC0346184621F07FFA386526F03EFCF3
:101E9000044607F12C0000230122012121F078FBE8
:101EA000F96A20460BF03AF84949386D10F0CAFB40
:101EB00026F02CFC024607F13003114618460BF0C1
:101EC000DFF86A4607F13C0393E8030082E8030069
:101ED00007F130030ECB386D2CF06EF84FF48033E1
:101EE000BB623C4B7B6207F144031846FFF76CFF73
:101EF0000346FB6107F148031846FFF795FF0346C9
:101F0000BB6107F14C031846FFF79CFF03463B6299
:101F10000023FB6000233B6100237B612E4BFB60B1
:101F20002E4B7B612E4B3B617D6D02AC07F10C03A8
:101F300093E8070084E807006A4607F1200393E866
:101F4000030082E8030007F118030CCBB96A2846A6
:101F500006F016F903462349184625F01DF900221C
:101F600001214FF48C7001F009FB02461E4B1A60F0
:101F70001D4B1B68002B04D14FF4A1711B4806F0C8
:101F800091FC1B4B00930023012245F2A12119482B
:101F900022F00DF80246184B1A60174B1B68002BF5
:101FA00004D140F24511114806F07CFC26F0AEFB4E
:101FB0000346002118460AF009FF06F0CDFB0F4B3F
:101FC0001B7818465837BD46B0BD00BFAC090600A7
:101FD00074C70120E1F60300811803009D19030076
:101FE000D919030098C70120A8C702206809060074
:101FF000E51C0300B8090600ACC7022080CF022010
:1020000080B584B000AF3871397006F0FBF8F86025
:102010000221F86806F008F926F078FB0346002153
:1020200018460AF0D3FE0121F86806F0FDF826F004
:102030006DFB0346002118460AF0C8FE024B1B78D0
:1020400018461037BD4680BD80CF022080B483B0D3
:1020500000AF38713970044B1B7818460C37BD46F9
:102060005DF8047B704700BF80CF022090B5ADF6CD
:102070002C0D00AF07F10C0420600C4610461946E9
:1020800007F10A0322461A8007F1080302461A8064
:10209000BB1D0A461A8040480DF022FB4FF4006336
:1020A000C7F8243807F1200107F114034FF4006248
:1020B000184628F0B9FD07F11403184629F0B0F8C6
:1020C00007F114033549184629F097F807F10C0376
:1020D00007F114021968104629F08FF807F114036C
:1020E0002F49184629F089F807F10A031A8807F1E1
:1020F00014031146184628F085FF07F114032949F7
:10210000184629F07AF807F10803B3F9002007F11F
:1021100014031146184628F075FF07F114032249ED
:10212000184629F06AF8BB1D1A8807F114031146F6
:10213000184628F067FF07F114031C49184629F0D8
:102140005CF897F83838002B01D0194A00E0194A9A
:1021500007F114031146184629F04FF807F114034C
:10216000184629F0B4F814480DF0BAFA07F1140330
:102170009A6807F120031946104807F095FA0346BC
:1021800087F823380E480DF0ABFA97F82338184635
:1021900007F62C07BD4690BDC0090600E009060001
:1021A000E8090600F0090600FC090600080A060016
:1021B000100A0600180A0600200A0600300A060067
:1021C000340A060090B5ADF6340D02AF07F10C04E9
:1021D000206007F1080001601946BB1D1A803B1DF5
:1021E0000A461A8062480DF07BFA4FF40063C7F884
:1021F000243807F1200107F114034FF40062184658
:1022000028F012FD07F11403184629F009F807F128
:1022100014035849184628F0F0FF07F1080307F1A6
:1022200014021968104628F0E8FF07F11403524918
:10223000184628F0E2FFBB1D1A8807F11403114667
:10224000184628F0DFFE07F114034C49184628F021
:10225000D4FF3B1DB3F9002007F1140311461846C3
:1022600028F0D0FE07F10C031B68002B3BD007F1D0
:1022700014034349184628F0C0FF07F10C031B68FC
:102280005B681A4607F114031146184628F0BAFE97
:1022900007F114033B49184628F0AFFF07F10C0380
:1022A0001B6803F1200107F10C031B68DA6907F1D1
:1022B0001403184628F035FF07F114033249184675
:1022C00028F09BFF07F10C031B68B3F914301A4682
:1022D00007F114031146184628F094FE07F1140381
:1022E000184628F0F4FF07F11403184628F0EFFF12
:1022F000264B9B7B002B21D0244B9968234B9B8939
:102300001A4623480DF0ECF926F000FA0346184669
:1023100021F03AF8044607F1140398681B4B9B68B8
:102320001A4A928907F120010192009303460A4656
:10233000002120460FF0A8FE012313E015480DF000
:10234000CFF907F114039A6807F12003194600201A
:1023500007F0AAF9034687F823380F480DF0C0F9B3
:1023600097F82338184607F62C07BD4690BD00BFE6
:102370004C0A0600E0090600E8090600F00906001C
:10238000640A0600700A06007C0A060074C7012071
:10239000840A0600200A0600340A060080B5ADF55E
:1023A000026D00AF012387F81F384FF40063C7F8B0
:1023B000183807F110013B1D4FF40062184628F051
:1023C00033FC26F0A3F902463B1D194610460AF0DD
:1023D0005FFAC7F81408D7F81438002B11D007F1AA
:1023E0001003D7F8142819461F4807F05DF9034673
:1023F00083F00103DBB2002B06D0002387F81F38DF
:1024000002E0002387F81F3823F089FCC7F8100882
:1024100007F110034FF400621946D7F8100804F0D2
:1024200073FCC7F81408D7F81438002B11D007F143
:102430001003D7F8142819460C4807F035F903465D
:1024400083F00103DBB2002B06D0002387F81F388E
:1024500002E0002387F81F3897F81F38184607F561
:102460000267BD4680BD00BFA80A0600B00A06008C
:1024700080B582B000AF78600D4B1B78002B0CBF8D
:1024800001230023DBB21A46094B1A70094B1A6864
:10249000074B1B78002B14BF01230023DBB2194626
:1024A000104626F062F900BF0837BD4680BD00BF68
:1024B000A8E90220B8C9022080B483B000AF7860D8
:1024C000034B18460C37BD465DF8047B704700BFD0
:1024D0005739050090B5ADF5157D02AF3B1D18705D
:1024E0003B46197005F08EFEC7F8400206F034F93D
:1024F000324B1B6803F00103002B07D126F006F9CD
:1025000002462F4B1A602D4B01221A602C4B1B6880
:10251000184620F039FFC7F83C022A480DF0E0F8D1
:102520000121D7F83C020FF0A7FE07F50B73184600
:10253000FFF7C2FF034600934FF078024FF000030D
:10254000D7F83C020FF0D6FE034687F83B321C4B0F
:102550001B680021184626F008F9194B1B6897F8EC
:102560003B221146184621F00AF9154B1A6897F8D4
:102570003B3283F00103DBB21946104626F0E1F846
:10258000C82001F085FD0E4B1B680021184626F07F
:10259000D8F80B4B1B680021184621F0F0F897F88B
:1025A0003B3283F00103DBB2002B11D006480DF063
:1025B00097F806F0D1F8054B1B7860E1BCC9022002
:1025C000B8C90220B80A0600D00A060080CF02204F
:1025D000AD480DF085F8002387F847320121D7F880
:1025E0003C0210F043FF4FF48073C7F834322AF0F6
:1025F000D0FF0346C7F83032A44B9B79002B32D072
:10260000A24B9B7B002B2ED007F596734FF4807264
:102610001946D7F83C020FF0A5FFD7F83C020FF09F
:102620006BFF03461C46D7F83C020FF02FFF034612
:102630009BB21A46920013445B009BB21AB2D7F8C1
:10264000303299B207F59670002300930B4621466D
:10265000FFF70CFD034683F00103DBB2002B02D031
:10266000012387F847322AF094FF0346002B0CBF62
:1026700001230023DBB2002B39D007F596734FF40A
:1026800080721946D7F83C020FF06CFF07F596737D
:1026900019467F480DF024F87E480DF021F8D7F850
:1026A0003C020FF029FF03461C46D7F83C020FF00E
:1026B000EDFE03469BB21A46920013445B009BB2A8
:1026C0001BB207F5967122460020FFF77BFD0346FB
:1026D00087F82F3297F82F3283F00103DBB2002BFB
:1026E00005D06D480CF0FCFF012387F847322AF033
:1026F00050FF0346002BCCBF01230023DBB2002B8D
:102700005DD007F596734FF480721946D7F83C02F6
:102710000FF028FF07F5967319465D480CF0E0FFAF
:1027200007F10C0318464FF490731A4600212BF062
:1027300091FD07F10C031946D7F8400205F022FC81
:10274000034687F82E322AF041FF04462AF021FF83
:102750000346E41A2AF03AFF03461A4621464F4838
:102760000CF0BEFF97F82E32002BC0D0D7F83C02F9
:102770000FF0C2FE03461C46D7F83C020FF086FE5F
:1027800003469BB21A46920013445B009BB21BB2F5
:1027900007F5967107F10C002246FFF713FD03467B
:1027A00087F82D3297F82D3283F00103DBB2002B2E
:1027B0009DD03B480CF094FF012387F84732334B00
:1027C0009B79002B32D0314B9B7B002B2ED007F511
:1027D00096734FF480721946D7F83C020FF0C2FE90
:1027E000D7F83C020FF088FE03461C46D7F83C029F
:1027F0000FF04CFE03469BB21A46920013445B0056
:102800009BB21AB2D7F8303299B207F5967001230D
:1028100000930B462146FFF729FC034683F0010392
:10282000DBB2002B02D0012387F84732D7F84002F1
:1028300021F044F897F84732002B18D0194B1B6849
:102840000133184A1360174B1B68194616480CF0E1
:1028500047FF144B1B68042B0CD914480CF040FFA5
:10286000104B1B68194612480BF004F902E00D4B9F
:1028700000221A60642001F00BFC0E4B1B781846F6
:1028800007F51377BD4690BDFC0A060074C701200A
:102890000C0B0600200B0600440B06006C0B060018
:1028A0008C0B0600C0C90220AC0B0600C40B06004E
:1028B000E40B060080CF022080B582B000AF3871F3
:1028C0003970FFF71FFA034B1B7818460837BD46CF
:1028D00080BD00BF80CF022080B584B000AF3871CA
:1028E00039700023FB60002006F0E0F8F860FB6818
:1028F000002B1BD0FB6819460F480CF0F1FEFB685B
:102900005B6A002B02D0FB685B6A00E00B4B194648
:102910000B480CF0E5FEF86806F0C6FFF86824F0F6
:102920003CFE002006F0C2F8F860E0E7054B1B789B
:1029300018461037BD4680BD000C0600240C06006A
:10294000280C060080CF022080B582B000AF7860EE
:102950000D4B1B78002B0CBF01230023DBB21A4662
:10296000094B1A70094B1A68074B1B78002B14BFD0
:1029700001230023DBB21946104625F0F6FE00BF06
:102980000837BD4680BD00BFA9E90220C4C90220A6
:1029900080B483B000AF7860034B18460C37BD4657
:1029A0005DF8047B704700BF6339050090B58FB0B8
:1029B00002AF3871397070480CF092FE05F022FCBD
:1029C0000346184620F084FF024607F10C0307CAAD
:1029D00083E80700FB68022098473B6942F21070C9
:1029E0009847F8627B699847FB6A002B03D16348DC
:1029F0000CF076FE0EE062480CF072FEFB6A1B687B
:102A0000002B04D0FB6A1B6818460CF039FFF86AEB
:102A10000CF036FF5B480CF063FE5B4B1B6803F069
:102A20000103002B07D125F071FE0246574B1A60B7
:102A3000554B01221A60554B1B68184620F0A4FC28
:102A4000B86253480CF04CFE0121B86A0FF014FC38
:102A500007F108031846FFF79BFF034600934FF06A
:102A600078024FF00003B86A0FF044FC034687F881
:102A70002730464B1B680021184625F076FE434B55
:102A80001B6897F827201146184620F078FE3F4B28
:102A90001A6897F8273083F00103DBB21946104615
:102AA00025F04FFEC82001F0F3FA384B1B680021D7
:102AB000184625F046FE354B1B680021184620F0CD
:102AC0005EFE97F8273083F00103DBB2002B07D0BE
:102AD00030480CF005FEFFF715F92F4B1B7847E047
:102AE0000121B86A10F0C2FC2C4B9B79002B2FD02F
:102AF00006F012FEC7E90601D7E90634234313D0D6
:102B0000D7E906010CF04CFD0346194624480CF0A9
:102B1000E7FD1E4B1B68184620F043FE0368043394
:102B20001968D7E9062388471E480CF0D9FDFFF73E
:102B300035FC0346002B03D01B480CF0D1FD07E009
:102B40001A480CF0CDFDFFF7DDF8134B1B780FE0B2
:102B50000021B86A10F08AFC0021B86A0FF08CFBE3
:102B600023F0DDF80346184604F0BEFA104B1B783C
:102B700018463437BD4690BD380C0600540C06008C
:102B8000800C06009C0C0600C8C90220C4C90220A3
:102B9000B80A0600C00C06007CCF022074C70120D2
:102BA000FC0C06001C0D06004C0D0600680D06000E
:102BB00078CF022080B582B000AF0E480CF090FDB7
:102BC00000237B604FF4FA7012F020FB03467B6019
:102BD0007B68002B03D108480CF082FD05E0074814
:102BE0000CF07EFD786812F019FB00BF0837BD4677
:102BF00080BD00BF8C0D0600BC0D0600F00D060068
:102C000090B593B002AF786025F080FDF863FB6B60
:102C10001B6808331B68F86B984749F2A8324FF0DD
:102C200000030121F86B0AF03DF801200AF048FF8B
:102C3000FFF7C0FFFEF716FDF86B0AF005F9B86361
:102C4000744A7549B86B20F054FD034687F8343058
:102C5000724A7349B86B20F04CFD034687F8303058
:102C6000704A7149B86B20F044FD034687F82C3058
:102C70006E49B86B20F055FD034687F828304FF4B5
:102C800096734FF00004CDE900344FF03C024FF052
:102C900000036749B86B20F00FFD034687F8243026
:102CA000644A6549B86B20F024FD034687F820305C
:102CB000624A6349B86B20F01CFD03463B77614ACA
:102CC0006149B86B20F015FD03463B765F49B86B50
:102CD00020F027FD03463B755D4A5E49B86B20F046
:102CE00008FD03463B7423F01AF803465A49184678
:102CF00023F0F5F903461A465849B86B20F0C4FC96
:102D000003463B7307F134031946B86B20F0ACFC63
:102D1000534A97F82C30127897F83410B86B20F09B
:102D200017FD504A97F83030127897F82C10B86B8E
:102D300020F00EFD4C4A97F82830127897F82C10A6
:102D4000B86B20F005FD97F82C3097F8242097F801
:102D50002810B86B20F0FCFC414A97F8203012781C
:102D600097F83010B86B20F0F3FC3D4A3B7C1278AA
:102D700097F82010B86B20F0EBFC394A3B7E1278B4
:102D8000397CB86B20F0E4FC354A3B7D1278397E03
:102D9000B86B20F0DDFC3B7F3A7B397DB86B20F0CF
:102DA000D7FC2F4A97F830301278397FB86B20F073
:102DB000CFFCB86B08F05CF803224FF4FA61B86BF3
:102DC00007F0F8FD00F080F928480CF089FCF86B5A
:102DD00025F052FD034687F8373097F8373019460B
:102DE00023480CF07DFC97F8373083F00103DBB209
:102DF000002B05D01F4A40F6B831F86B09F0F8FCFB
:102E0000FFF7D8FE002001F0DDF800BF4437BD46D3
:102E100090BD00BF611E0300FC0D060001200300F1
:102E2000040E0600AD2903000C0E0600140E060069
:102E3000200E0600D52403002C0E06004D200300B2
:102E4000380E0600B9280300400E0600480E0600A2
:102E5000D9280300500E0600600E06006C0E060016
:102E600080CF022078CF02207CCF0220740E060093
:102E7000980E0600B00E060080B582B000AF7860F4
:102E80007B680E4A1A6025F041FC03460121184672
:102E900025F057FC25F03AFC03460021184620F0A7
:102EA0006EFC25F033FC03460021184625F05DFC3E
:102EB000002318460837BD4680BD00BFCCC902209C
:102EC00080B582B000AF25F021FC78600F48DCF7B8
:102ED000C3FE034683F00103DBB2002B04D040F2B3
:102EE0002F310B4805F0DEFC08490A480CF0F8FBCE
:102EF000094803F08DF84FF4FA620849786809F040
:102F00001FFB002318460837BD4680BD755E0300D1
:102F100068090600CC0E0600792E0300012C030080
:102F200080B483B000AF0346FB7197F90730002BE4
:102F30000BDBFB7903F01F02074997F907305B09A8
:102F4000012000FA02F241F8232000BF0C37BD46F1
:102F50005DF8047B704700BF00E100E080B483B0FF
:102F600000AF0346FB7197F90730002B0CDBFB79B0
:102F700003F01F02074997F907305B09012000FAA7
:102F800002F2603341F8232000BF0C37BD465DF8E4
:102F9000047B704700E100E080B483B000AF0346DB
:102FA0003960FB7197F90730002B0ADB3B68DAB216
:102FB0000C4997F907305201D2B20B4483F8002331
:102FC0000AE03B68DAB20849FB7903F00F03043BDF
:102FD0005201D2B20B441A7600BF0C37BD465DF8E1
:102FE000047B704700E100E000ED00E080B582B0B6
:102FF00000AF184B00221A60174B00221A602021E4
:10300000164820F003FD0121144820F0C3FC0821DC
:10301000124820F00AFD0021104820F006FD022190
:103020000E4820F014FD07211420FFF7B5FF0123FF
:103030007B607B681B010A4A03F0100313611420B4
:10304000FFF78CFF1420FFF76BFF00BF0837BD466A
:1030500080BD00BF10E000E018E000E0004001404B
:1030600000ED00E080B582B000AF00237B60094B2B
:103070001B68B3F1FF3F04D04FF4C071064805F060
:1030800011FC72B600BF7B68002BFCD000BF083774
:10309000BD4680BD7CC00120F00E060080B500AFAB
:1030A000DCF7D2FD064B1B68054A43F4700313603E
:1030B000044B1B68034A43F04043136000BF80BDCC
:1030C00088ED00E034EF00E080B400AF064B4FF035
:1030D00080521A60BFF34F8FBFF36F8F00BFBD46A2
:1030E0005DF8047B704700BF04ED00E080B400AFE2
:1030F00072B6074B1B680133054A1360BFF34F8F4D
:10310000BFF36F8F00BFBD465DF8047B704700BF03
:103110007CC0012080B500AF0A4B1B68002B04D196
:103120004FF40671084805F0BDFB064B1B68013BD8
:10313000044A1360034B1B68002B00D162B600BF2A
:1031400080BD00BF7CC00120F00E060080B584B0B9
:1031500000AF4FF4A0711E4820F03AFC0023FB6042
:1031600020F099FC78601A4820F043FC38604FF456
:103170008071174820F02CFC01F0B4F902463B683E
:103180009B1A23F07F43BB60BB68012B0DD901F074
:10319000A1FE0346022B08D00123BB6005E001F02D
:1031A0007FFA0246FB681343FB60BB685A1EBA6095
:1031B000002BF4D1FB68002B03D0064B4FF080525C
:1031C0001A60786820F06DFC00BF1037BD4680BDE6
:1031D0000040014004ED00E080B588B000AF7860A9
:1031E0007B68394A934201D9374B7B6072B6BFF393
:1031F0004F8FBFF36F8F354820F0FBFBF86101F074
:10320000F5FC0346002B55D0FA697B68134423F084
:103210007F43BB6101212D4820F0CBFBBA6900211F
:103220002A4820F0A4FB4FF4A071284820F0D0FBDE
:103230004FF48031254820F0ADFBBFF34F8FBFF333
:103240006F8F7B687B617B69002B0DD0BFF34F8F45
:1032500020BFBFF36F8F1E4BD3F800211C4BD3F858
:1032600004311343002BF1D04FF48031174820F084
:10327000A0FB4FF4A071154820F0AAFB4FF4807119
:10328000124820F0A5FB0121104820F083FB0F48D5
:1032900020F0AFFB38613A69FB69D31A23F07F4312
:1032A000FB601420FFF75AFEFB68002B02D0F86881
:1032B00001F0D4F962B6BFF34F8FBFF36F8F00BF39
:1032C0002037BD4680BD00BFFDFFFF00004001402C
:1032D00000E100E080B586B000AF78607B689B6954
:1032E0007B617B69023B1B78FB74FB7C012B1BD051
:1032F000022B21D0002B28D17B681B68FB60F8686B
:10330000DCF782FC0246154B1A60144B1B68002B3D
:1033100004D140F20731124805F0C4FA0F4B1B6884
:103320001846DCF789FC15E07B681B68FB60FB68CE
:103330001846DCF78DFC0DE0DCF762FCDCF774FC72
:10334000FFF7ACFEFDF78CFA04E040F2423104488E
:1033500005F0A8FA00BF1837BD4680BDF4C90220A9
:10336000F00E060080B485B000AFF860B9607A60F6
:103370003B60FB68043BFB60FB684FF080721A60A7
:10338000FB68043BFB607A68FB681A60FB68043BDF
:10339000FB603B4AFB681A60FB68043BFB60FB6810
:1033A0004FF012321A60FB68043BFB60FB684FF081
:1033B00003321A60FB68043BFB60FB684FF002328B
:1033C0001A60FB68043BFB60FB684FF001321A6037
:1033D000FB68043BFB603A68FB681A60FB68043BCF
:1033E000FB60FB684FF011321A60FB68043BFB6026
:1033F000FB684FF010321A60FB68043BFB60FB680F
:103400004FF009321A60FB68043BFB60FB684FF029
:1034100008321A60FB68043BFB60FB684FF0073220
:103420001A60FB68043BFB60FB684FF006321A60D1
:10343000FB68043BFB60FB684FF005321A60FB68D9
:10344000043BFB60FB684FF004321A60FB68043BEE
:10345000FB60FB686FF043021A60FB68043BFB6093
:10346000BA68FB681A60FB68043BFB60FB680022DB
:103470001A60FB6818461437BD465DF8047B704738
:103480006530030080B500AF0C4B1B680B4A43F45A
:103490007F031360094B1B68084A43F07F431360A6
:1034A000FFF7A4FD064B00221A60FDF7F9F901F0C1
:1034B000ADF9FFF7D7FD0023184680BD20ED00E0F1
:1034C0007CC0012080B584B000AF786039607B6833
:1034D000FB60FB68002B04D140F20311264805F085
:1034E000E1F9FFF703FEFB681A68FB68DB6BF9681C
:1034F000096C01FB03F31A44FB689A60FB68002225
:103500009A63FB681A68FB685A60FB681A68FB6874
:10351000DB6B013BF968096C01FB03F31A44FB68A0
:10352000DA60FB68FF2283F84420FB68FF2283F8FF
:1035300045203B68002B0ED1FB681B69002B14D083
:10354000FB681033184601F03DFA0346002B0CD0FF
:10355000FFF7BAFD09E0FB681033184620F05AFD6A
:10356000FB682433184620F055FDFFF7D3FD0123F7
:1035700018461037BD4680BD5C0F060080B58AB086
:1035800002AFF860B9601346FB71FB68002B04D1F1
:103590004FF4BB71144805F085F9BB68002B02D1CC
:1035A0000023FB6104E0FB68BA6802FB03F3FB61E4
:1035B000FB695033184620F0F7FDB861BB69002B5A
:1035C0000DD0BB697B617B6950337B61FA79BB6944
:1035D000009313467A69B968F86820F070FABB69FD
:1035E00018462037BD4680BD5C0F060080B58AB006
:1035F00000AFF860B9607A603B6000237B62FB68D3
:103600003B623B6A002B04D140F2F121604805F097
:1036100049F9BB68002B03D13B6A1B6C002B01D11D
:10362000012300E00023002B04D140F2F22158488E
:1036300005F038F93B68022B03D13B6ADB6B012BA9
:1036400001D1012300E00023002B04D140F2F3213B
:103650004F4805F027F901F03DFC0346002B02D14D
:103660007B68002B01D1012300E00023002B04D153
:1036700040F2F621464805F015F9FFF737FD3B6AA1
:103680009A6B3B6ADB6B9A4202D33B68022B1DD1DB
:103690003A68B968386A20F07FFAF8613B6A5B6A79
:1036A000002B0AD03B6A2433184601F08BF90346FD
:1036B000002B07D0FFF708FD04E0FB69002B01D0C9
:1036C000FFF702FDFFF726FD01235CE07B68002B7E
:1036D00003D1FFF71FFD002355E07B6A002B06D1C5
:1036E00007F11403184601F0CFF901237B62FFF7BD
:1036F00011FD00F01FFEFFF7F9FC3B6A93F8443020
:103700005BB2B3F1FF3F03D13B6A002283F8442050
:103710003B6A93F845305BB2B3F1FF3F03D13B6A9C
:10372000002283F84520FFF7F5FC3A1D07F114034A
:103730001146184601F0BEF90346002B1DD1386A28
:1037400020F022FB0346002B11D03B6A10337A682D
:103750001146184601F0EEF8386A20F0ADFA00F094
:103760002FFE0346002B88D1FFF7AEFC85E7386AB1
:1037700020F0A2FA00F024FE7FE7386A20F09CFADD
:1037800000F01EFE002318462837BD4680BD00BF4E
:103790005C0F060080B588B000AFF860B9607A6051
:1037A0003B60FB68BB61BB69002B04D140F2C331B5
:1037B000324805F077F8BB68002B03D1BB691B6C5E
:1037C000002B01D1012300E00023002B04D14FF492
:1037D00071712A4805F066F83B68022B03D1BB697A
:1037E000DB6B012B01D1012300E00023002B04D16E
:1037F00040F2C531214805F055F820F04CF97861C8
:10380000BB699A6BBB69DB6B9A4202D33B68022BA4
:103810002AD1BB6993F84530FB743A68B968B86936
:1038200020F0BAF997F91330B3F1FF3F12D1BB6919
:103830005B6A002B15D0BB692433184601F0C2F82F
:103840000346002B0DD07B68002B0AD07B68012239
:103850001A6006E0FB7C0133DBB25AB2BB6983F825
:1038600045200123FB6101E00023FB61786920F022
:1038700018F9FB6918462037BD4680BD5C0F06006D
:1038800080B58AB000AFF860B9607A6000237B62CF
:10389000FB683B623B6A002B04D14FF4A06158489F
:1038A00005F000F8BB68002B03D13B6A1B6C002BB2
:1038B00001D1012300E00023002B04D140F2045188
:1038C0004F4804F0EFFF01F005FB0346002B02D147
:1038D0007B68002B01D1012300E00023002B04D1E1
:1038E00040F20951464804F0DDFFFFF7FFFB3B6A59
:1038F0009B6BFB61FB69002B19D0B968386A20F01B
:10390000B5F9FB695A1E3B6A9A633B6A1B69002B37
:1039100009D03B6A1033184601F054F80346002BD7
:1039200001D0FFF7D1FBFFF7F5FB012363E07B68D4
:10393000002B03D1FFF7EEFB00235CE07B6A002B3A
:1039400006D107F11403184601F09EF801237B62AB
:10395000FFF7E0FB00F0EEFCFFF7C8FB3B6A93F8D3
:1039600044305BB2B3F1FF3F03D13B6A002283F8DE
:1039700044203B6A93F845305BB2B3F1FF3F03D17B
:103980003B6A002283F84520FFF7C4FB3A1D07F18C
:1039900014031146184601F08DF80346002B1DD183
:1039A000386A20F0DBF90346002B11D03B6A243340
:1039B0007A681146184600F0BDFF386A20F07CF99D
:1039C00000F0FEFC0346002B8FD1FFF77DFB8CE758
:1039D000386A20F071F900F0F3FC86E7386A20F0CD
:1039E0006BF900F0EDFC386A20F0B8F90346002BC3
:1039F0003FF47BAF002318462837BD4680BD00BF8B
:103A00005C0F060080B58AB000AF78603960002393
:103A10007B627B68FB6100233B62FB69002B04D166
:103A200040F291516A4804F03DFFFB691B6C002B8A
:103A300004D040F29551664804F034FF01F04AFA90
:103A40000346002B02D13B68002B01D1012300E08B
:103A50000023002B04D140F29A515D4804F022FF6C
:103A6000FFF744FBFB699B6BBB61BB69002B1ED05E
:103A7000BB695A1EFB699A63FB691B68002B04D162
:103A800001F08AFB0246FB699A60FB691B69002B07
:103A900009D0FB691033184600F094FF0346002B51
:103AA00001D0FFF711FBFFF735FB01238BE03B68EB
:103AB000002B0BD13B6A002B04D040F2E15144486B
:103AC00004F0F0FEFFF726FB00237CE07B6A002B6E
:103AD00006D107F10C03184600F0D6FF01237B62E4
:103AE000FFF718FB00F026FCFFF700FBFB6993F8DB
:103AF00044305BB2B3F1FF3F03D1FB69002283F88E
:103B00004420FB6993F845305BB2B3F1FF3F03D12A
:103B1000FB69002283F84520FFF7FCFA3A4607F1DB
:103B20000C031146184600F0C5FF0346002B2CD1AC
:103B3000F86920F013F90346002B20D0FB691B68BD
:103B4000002B09D1FFF7D2FAFB699B68184601F0F8
:103B5000DFF93862FFF7DEFAFB6924333A68114671
:103B6000184600F0E7FEF86920F0A6F800F028FCFF
:103B70000346002B7FF474AFFFF7A6FA70E7F869ED
:103B800020F09AF800F01CFC6AE7F86920F094F83D
:103B900000F016FCF86920F0E1F80346002B3FF432
:103BA0005FAF3B6A002B0DD0FFF7A0FAF8691FF05A
:103BB000DBFF7861FB699B687969184601F074FA4C
:103BC000FFF7A8FA002318462837BD4680BD00BF7E
:103BD0005C0F060080B58AB000AFF860B9607A600B
:103BE00000237B62FB683B623B6A002B04D14FF4ED
:103BF000CD61594804F056FEBB68002B03D13B6AE7
:103C00001B6C002B01D1012300E00023002B04D109
:103C100040F26C61504804F045FE01F05BF9034648
:103C2000002B02D17B68002B01D1012300E000238F
:103C3000002B04D140F27161474804F033FEFFF7D6
:103C400055FA3B6A9B6BFB61FB69002B1BD03B6AFF
:103C5000DB68BB61B968386A20F008F83B6ABA696A
:103C6000DA603B6A5B6A002B09D03B6A2433184652
:103C700000F0A8FE0346002B01D0FFF725FAFFF75E
:103C800049FA012363E07B68002B03D1FFF742FA76
:103C900000235CE07B6A002B06D107F11003184675
:103CA00000F0F2FE01237B62FFF734FA00F042FBE2
:103CB000FFF71CFA3B6A93F844305BB2B3F1FF3F65
:103CC00003D13B6A002283F844203B6A93F84530D5
:103CD0005BB2B3F1FF3F03D13B6A002283F845207A
:103CE000FFF718FA3A1D07F110031146184600F0C5
:103CF000E1FE0346002B1DD1386A20F02FF8034661
:103D0000002B11D03B6A24337A681146184600F024
:103D100011FE386A1FF0D0FF00F052FB0346002B63
:103D20008DD1FFF7D1F98AE7386A1FF0C5FF00F09F
:103D300047FB84E7386A1FF0BFFF00F041FB386A99
:103D400020F00CF80346002B3FF479AF002318460F
:103D50002837BD4680BD00BF5C0F060080B584B02B
:103D600000AF78607B68FB60FB68002B04D140F2F9
:103D7000B771054804F096FDF86820F023FA00BFFB
:103D80001037BD4680BD00BF5C0F060080B586B011
:103D900000AFF860B9607A603B60BB6A186B7B6803
:103DA0009B001A46A5212AF055FABB6A1A6B7B685C
:103DB00003F18043013B9B0013443B613B6923F0CB
:103DC00007033B613B6903F00703002B04D040F27B
:103DD0006131444804F066FDBB68002B1FD000230E
:103DE0007B6112E0BA687B6913441978BA6A7B690F
:103DF000134434330A461A70BA687B6913441B783B
:103E0000002B06D07B6901337B617B690B2BE9D9E1
:103E100000E000BFBB6A002283F83F2003E0BB6ADA
:103E2000002283F834203B6A052B01D905233B622D
:103E3000BB6A3A6ADA62BB6A3A6A9A64BB6A00226F
:103E4000DA64BB6A0433184620F004F9BB6A1833FD
:103E5000184620F0FFF8BB6ABA6A1A613B6AC3F1E0
:103E60000602BB6A9A61BB6ABA6A5A6200237B6126
:103E700008E0BB6A7A691432002143F822107B699A
:103E800001337B617B69002BF3D0BB6A0022C3F84E
:103E9000B420BB6A002283F8B820BB6A5433602286
:103EA000002118462AF0D6F9BB6A0F4A9A65BB6A08
:103EB0000E4ADA65BB6A0E4A1A66BB6A196B3B6822
:103EC000FA683869FFF74EFA0246BB6A1A607B6AE5
:103ED000002B02D07B6ABA6A1A6000BF1837BD4651
:103EE00080BD00BFA00F06003C6406005C640600B5
:103EF0001C64060080B582B000AF7860FFF7F6F86A
:103F00002A4B1B680133294A1360294B1B68002B7D
:103F100009D1274A7B681360244B1B68012B10D101
:103F200000F0D6FE0DE0234B1B68002B09D1204B7F
:103F30001B68DA6A7B68DB6A9A4202D81C4A7B6893
:103F400013601D4B1B6801331B4A13601A4B1A6820
:103F50007B681A647B68DA6A184B1B689A4203D93B
:103F60007B68DB6A154A13607B68DA6A13469B003C
:103F700013449B00124A1A447B68043319461046C6
:103F800020F075F8FFF7C6F80A4B1B68002B08D025
:103F9000074B1B68DA6A7B68DB6A9A4201D2FFF73B
:103FA00093F800BF0837BD4680BD00BFE8CA0220B5
:103FB000F8C90220F4CA022004CB0220F0CA022071
:103FC000FCC9022080B584B000AF7860FFF78EF89E
:103FD0007B68002B02D1264B1B6800E07B68FB60EE
:103FE000FB680433184620F09FF8FB689B6A002B9F
:103FF00004D0FB681833184620F096F81D4B1B6858
:1040000001331C4A13601A4B1B68FA689A420BD1A1
:10401000FB6804331946184820F029F8174B1B6831
:104020000133164A136009E0154B1B68013B144A23
:104030001360F8681FF0A3FF00F01CFFFFF76AF899
:10404000104B1B68002B0FD0094B1B68FA689A4273
:104050000AD10D4B1B68002B04D040F2D2410B4813
:1040600004F020FCFFF730F800BF1037BD4680BDDC
:10407000F8C9022004CB0220B8CA0220CCCA022010
:10408000E8CA0220F4CA022010CB0220A00F0600CA
:1040900080B584B000AF78600023FB607B68002BA4
:1040A00011D00D4B1B68002B04D040F23C510B4843
:1040B00004F0F8FB00F03EF90021786801F082F985
:1040C00000F07EF9F860FB68002B01D1FEF7FCFFE1
:1040D00000BF1037BD4680BD10CB0220A00F0600E8
:1040E00080B588B000AF78607B68BB61BB69002B8E
:1040F00004D14FF4AD61254804F0D4FB244B1B6878
:10410000BA699A4202D10023FB773AE0FEF7EEFF4C
:10411000BB695B697B611F4B1B683B611E4B1B6866
:10412000FB60FEF7F7FF7A693B699A4203D07A6930
:10413000FB689A4202D10223FB7722E07B69174A8F
:10414000934212D1BB699B6A002B0BD1BB6993F8D8
:10415000B830DBB2012B02D10223FB7711E003233D
:10416000FB770EE00223FB770BE07B690C4A93425E
:1041700002D07B69002B02D10423FB7701E00123ED
:10418000FB77FB7F18462037BD4680BDA00F060099
:10419000F8C902209CCA0220A0CA0220D0CA02206C
:1041A000B8CA022080B584B000AF78600023FB60FD
:1041B0007B68BB607B68002B04D140F20E710C4819
:1041C00004F070FBBB685B690A4A93420AD1BB6882
:1041D0009B6A094A934205D0BB689B6A002B01D1B8
:1041E0000123FB60FB6818461037BD4680BD00BF49
:1041F000A00F0600D0CA0220A4CA022080B584B055
:1042000000AF78607B68FB607B68002B04D14FF4C3
:10421000E7611F4804F046FB1E4B1B68FA689A4290
:1042200032D0FB68002B2FD0FEF760FFF868FFF755
:10423000B9FF0346002B25D0FB68043318461FF056
:1042400073FFFB68DA6A144B1B689A4203D9FB6858
:10425000DB6A114A1360FB68DA6A13469B00134459
:104260009B000E4A1A44FB680433194610461FF09F
:10427000FEFEFB68DA6A074B1B68DB6A9A4201D3D1
:10428000FEF722FFFEF746FF00BF1037BD4680BD98
:10429000A00F0600F8C90220F0CA0220FCC90220C3
:1042A00080B584B002AF1A4B019300230093002322
:1042B0008022184918481FF0B3FD78607B68012BF5
:1042C00002D101F0D3F878607B68012B12D172B66D
:1042D000124B1B685433124A1360124B4FF0FF32DB
:1042E0001A60114B01221A60104B00221A60FFF76E
:1042F000C9F808E07B68B3F1FF3F04D14FF40261D5
:104300000B4804F0CFFA00BF0837BD4680BD00BFA0
:104310000CCB0220E40F06007D4B0300F8C90220FD
:104320004CC1012008CB0220F4CA0220ECCA0220B2
:10433000A00F060080B400AF044B1B680133034A92
:10434000136000BFBD465DF8047B704710CB0220B0
:1043500080B483B000AF00233B60144B1B68002B7C
:1043600001D001233B60124B1B68DB6A002B02D09B
:1043700000237B6012E00F4B1B68012B02D9002346
:104380007B600BE03B68002B02D000237B6005E0E4
:10439000094B1A68094B1B68D31A7B607B68184667
:1043A0000C37BD465DF8047B704700BFF0CA0220A1
:1043B000F8C90220FCC9022008CB0220ECCA022066
:1043C00080B584B000AF0023FB600023BB603C4B92
:1043D0001B68002B04D140F685013A4804F062FACC
:1043E000FEF784FE364B1B68013B354A1360344BA5
:1043F0001B68002B5CD1344B1B68002B58D02FE07E
:10440000324BDB68DB68FB60FB68183318461FF033
:104410008BFEFB68043318461FF086FEFB68DA6AE1
:104420002B4B1B689A4203D9FB68DB6A284A13604E
:10443000FB68DA6A13469B0013449B00254A1A4422
:10444000FB680433194610461FF011FEFB68DA6A58
:10445000214B1B68DB6A9A4202D3204B01221A606F
:104460001A4B1B68002BCBD1FB68002B01D000F04E
:1044700001FD1B4B1B687B607B68002B10D000F09C
:104480000FF90346002B02D0144B01221A607B68FF
:10449000013B7B607B68002BF1D1114B00221A603D
:1044A0000E4B1B68002B03D00123BB60FEF70CFEF4
:1044B000FEF730FEBB6818461037BD4680BD00BF12
:1044C00010CB0220A00F0600E8CA0220A4CA0220D6
:1044D000F0CA0220FCC90220F8C90220FCCA02204E
:1044E000F8CA022080B483B000AF054B1B687B6024
:1044F0007B6818460C37BD465DF8047B704700BFEB
:10450000ECCA022080B483B000AF00237B60054B6F
:104510001B683B603B6818460C37BD465DF8047B62
:10452000704700BFECCA022080B400AF034B1B6889
:104530001846BD465DF8047B704700BFE8CA0220FC
:1045400080B586B000AFF860B9607A6000237B6107
:1045500006233B61FFF7EEFE3A4B1B68BA689A42AE
:1045600068D33B69013B3B617A691346DB00134426
:104570009B001A46FB6898183A6913469B0013443F
:104580009B00314A1344012219461FF08AFC02465F
:104590007B6913447B613B69002BE2D17A69134646
:1045A000DB0013449B001A46FB689818274B1B68D6
:1045B000022219461FF075FC02467B6913447B6199
:1045C0007A691346DB0013449B001A46FB6898186F
:1045D0001F4B1B68022219461FF063FC02467B69D1
:1045E00013447B617A691346DB0013449B001A462F
:1045F000FB6813440422174918461FF052FC024678
:104600007B6913447B617A691346DB0013449B008A
:104610001A46FB68134403220F4918461FF041FC59
:1046200002467B6913447B617B68002B02D07B6868
:1046300000221A60FFF7C4FE7B6918461837BD4692
:1046400080BD00BFE8CA0220FCC902209CCA02202B
:10465000A0CA0220B8CA0220D0CA022080B582B007
:1046600000AF78600B4B1A687B681A440A4B1B68D2
:104670009A4204D940F61521084804F013F9054B75
:104680001A687B681344034A136000BF0837BD46AD
:1046900080BD00BFECCA022008CB0220A00F06009C
:1046A00080B586B000AF00237B614C4B1B68002BAC
:1046B00040F083804A4B1B6801333B61484A3B69A9
:1046C00013603B69002B1AD1464B1B681B68002BFB
:1046D00004D040F67F21444804F0E4F8414B1B68C5
:1046E000FB60424B1B683F4A1360404AFB68136003
:1046F0003F4B1B6801333E4A136000F0BBFB3D4B50
:104700001B683A699A4249D3364B1B681B68002BD9
:1047100004D1384B4FF0FF321A603FE0314B1B6839
:10472000DB68DB68BB60BB685B687B603A697B68A1
:104730009A4203D22F4A7B6813602FE0BB68043390
:1047400018461FF0F1FCBB689B6A002B04D0BB68C5
:10475000183318461FF0E8FCBB68DA6A264B1B6862
:104760009A4203D9BB68DB6A234A1360BB68DA6AE2
:1047700013469B0013449B00204A1A44BB68043331
:10478000194610461FF073FCBB68DA6A1C4B1B68A5
:10479000DB6A9A42B8D301237B61B5E7184B1B68EB
:1047A000DA6A164913469B0013449B000B441B68AE
:1047B000012B07D901237B6104E0124B1B680133F5
:1047C000104A1360104B1B68002B01D001237B6142
:1047D0007B6918461837BD4680BD00BF10CB02204C
:1047E000ECCA02209CCA0220A00F0600A0CA022028
:1047F00000CB022008CB0220F0CA0220FCC9022014
:10480000F8C90220F8CA0220FCCA022080B584B090
:1048100000AF404B1B68002B03D03F4B01221A60B6
:1048200073E03D4B00221A603C4B1B681B6BBB6066
:104830004FF0A5337B60BB681B687A689A4211D140
:10484000BB6804331B687A689A420BD1BB68083393
:104850001B687A689A4205D1BB680C331B687A687A
:104860009A4208D02D4B1A682C4B1B6834331946DA
:10487000104603F0CBFF294B1B68294A1268C3F886
:10488000BC20284B1B68FB600AE0FB68002B04D1AE
:1048900040F6B731244804F005F8FB68013BFB60A3
:1048A0002249FA6813469B0013449B000B441B6883
:1048B000002BEAD0FA6813469B0013449B001B4A66
:1048C00013443B603B685B685A683B685A603B68CE
:1048D0005A683B6808339A4204D13B685B685A685F
:1048E0003B685A603B685B68DB680C4A13600D4AA2
:1048F000FB681360094B1B68D3F8BC30084A13608F
:10490000064B1B6854330A4A136000BF1037BD467C
:1049100080BD00BF10CB0220FCCA0220F8C90220D3
:10492000E4CA0220F0CA0220A00F0600FCC902203F
:104930004CC1012080B582B000AF786039607B68DF
:10494000002B04D140F6CE31084803F0ABFF084BF2
:104950001B681833194678681FF0ADFB01213868D1
:1049600000F030FD00BF0837BD4680BDA00F060037
:10497000F8C9022080B584B000AFF860B9607A60F1
:10498000FB68002B04D140F6F9310C4803F08AFF94
:104990000B4B1B6818331946F8681FF068FB7B68DF
:1049A000002B02D04FF0FF33BB607968B86800F08D
:1049B00009FD00BF1037BD4680BD00BFA00F060037
:1049C000F8C9022080B584B000AF78607B68DB68EE
:1049D000DB68BB60BB68002B04D140F6294123484B
:1049E00003F060FFBB68183318461FF09DFB204B97
:1049F0001B68002B1FD1BB68043318461FF094FBC3
:104A0000BB68DA6A1B4B1B689A4203D9BB68DB6A36
:104A1000184A1360BB68DA6A13469B0013449B0074
:104A2000154A1A44BB680433194610461FF01FFB91
:104A300000F020FA05E0BB68183319460F481FF054
:104A400016FBBB68DA6A0E4B1B68DB6A9A4205D913
:104A50000123FB600B4B01221A6001E00023FB6085
:104A6000FB6818461037BD4680BD00BFA00F06008A
:104A700010CB0220F0CA0220FCC90220A4CA0220E6
:104A8000F8C90220FCCA022080B483B000AF78606D
:104A9000064B1A687B681A60054B1A687B685A6077
:104AA00000BF0C37BD465DF8047B704700CB022089
:104AB000ECCA022080B586B000AF786039607B68B0
:104AC000002B04D140F69441234803F0EBFE3B68F1
:104AD000002B04D140F695411F4803F0E3FEFEF79A
:104AE00005FB1E4B1B683B617B685B683A69D31A08
:104AF000FB603B681B68B3F1FF3F02D100237B6181
:104B000023E07B681A68164B1B689A4207D07B68C3
:104B10005B683A699A4202D301237B6115E03B68E6
:104B20001B68FA689A420BD23B681A68FB68D21A73
:104B30003B681A607868FFF7A7FF00237B6104E0F9
:104B40003B6800221A6001237B61FEF7E3FA7B6970
:104B500018461837BD4680BDA00F0600ECCA0220DB
:104B600000CB022080B400AF034B01221A6000BFCB
:104B7000BD465DF8047B7047FCCA022080B584B056
:104B800000AF78604FF480601EF08FFF00F0E0F817
:104B9000124B1B68012B01D9FEF796FAFFF7D8FBE1
:104BA000F860FB68012BF1D9FFF7C4FB0C4B1A68C6
:104BB0000C4B1B689A4204D240F65C510A4803F041
:104BC00071FEFFF7C5FBF860FB68012B02D9F8689E
:104BD000FEF702FBFFF7F4FBD8E700BFFCC9022099
:104BE00008CB0220ECCA0220A00F060080B483B0DC
:104BF00000AF01233B600123FB710F4B1B68002BAF
:104C000002D00023FB7110E00C4B1B68002B02D07C
:104C10000023FB7109E00A4B1A680A4B19683B68CC
:104C2000CB1A9A4201D10223FB71FB7918460C374B
:104C3000BD465DF8047B7047A4CA0220FCCA02206E
:104C4000D0CA0220E8CA022080B487B000AFF86062
:104C5000B9607A60BB68002B0DDCFB68002B02D1C9
:104C6000084B1B6800E0FB687B617B69BA68143203
:104C7000796843F8221000BF1C37BD465DF8047BFD
:104C8000704700BFF8C9022080B485B000AF7860DB
:104C900039600023FB603B68002B0EDC7B68002B37
:104CA00002D10A4B1B6800E07B68BB60BB683A68B6
:104CB000143253F82230FB6001E00023FB60FB68F4
:104CC00018461437BD465DF8047B7047F8C90220CA
:104CD00080B582B000AF00237B600CE07A68134699
:104CE0009B0013449B00124A134418461FF092F98C
:104CF0007B6801337B607B68052BEFD90D481FF083
:104D000089F90D481FF086F90C481FF083F90C480B
:104D10001FF080F90B481FF07DF90B4B054A1A6014
:104D20000A4B054A1A6000BF0837BD4680BD00BF68
:104D3000FCC9022074CA022088CA0220A4CA022028
:104D4000B8CA0220D0CA02209CCA0220A0CA0220EF
:104D500080B582B000AF19E0FEF7C8F90F4BDB68F1
:104D6000DB687B607B68043318461FF0DDF90C4B71
:104D70001B68013B0A4A13600A4B1B68013B094A46
:104D80001360FEF7C7F978681FF0F9F8054B1B6848
:104D9000002BE1D100BF0837BD4680BDB8CA022054
:104DA000E8CA0220CCCA022080B586B000AFF86005
:104DB000B9607A60FB70FB68002B02D12C4B1B683A
:104DC00000E0FB687B61BB687A691A607B6903F16C
:104DD0003402BB685A607B69DA6ABB681A617B6916
:104DE0001A6BBB68DA617B691A6CBB689A607B6975
:104DF0009A6CBB685A61BB6800229A61FB78052BEC
:104E00001AD01B4B1B687A699A4203D1BB680022F7
:104E10001A7318E0BB68FA781A73FB78032B12D167
:104E2000FFF788FA7B699B6A002B02D0BB680222DD
:104E30001A73FFF7C5FA06E07869FFF751F90346E0
:104E40001A46BB681A737B68002B09D07B691B6B01
:104E500018461FF078F803461A46BB681A8402E029
:104E6000BB6800221A8400BF1837BD4680BD00BF52
:104E7000F8C9022080B483B000AF0C4B1B681B68DC
:104E8000002B04D10A4B4FF0FF321A6008E0074BA9
:104E90001B68DB68DB687B607B685B68044A1360C7
:104EA00000BF0C37BD465DF8047B70479CCA0220EA
:104EB00008CB022080B483B000AF054B1B687B6039
:104EC0007B6818460C37BD465DF8047B704700BF11
:104ED000F8C9022080B483B000AF0B4B1B68002BD5
:104EE00002D101237B6008E0084B1B68002B02D134
:104EF00002237B6001E000237B607B6818460C374F
:104F0000BD465DF8047B7047F4CA022010CB022036
:104F100080B584B000AF78607B68BB600023FB6025
:104F20007B68002B51D0BB68DA6A2A4B1B68DB6AAE
:104F30009A4241D2BB689B69002B06DB254B1B685C
:104F4000DB6AC3F10602BB689A61BB685969BB683A
:104F5000DA6A13469B0013449B001F4A134499428C
:104F600022D1BB68043318461FF0DEF8194B1B68CA
:104F7000DA6ABB68DA62BB68DA6A184B1B689A4265
:104F800003D9BB68DB6A154A1360BB68DA6A13464B
:104F90009B0013449B00104A1A44BB680433194613
:104FA00010461FF064F804E00A4B1B68DA6ABB681D
:104FB000DA620123FB6008E0BB689A6C054B1B6852
:104FC000DB6A9A4201D20123FB60FB681846103766
:104FD000BD4680BDF8C90220FCC90220F0CA0220EB
:104FE00080B584B000AF78607B68BB600023FB6055
:104FF0007B68002B4AD0284B1B68BA689A4204D0C1
:1050000040F6D171254803F04DFCBB68DB6C002BEA
:1050100004D140F6D271214803F044FCBB68DB6C3C
:105020005A1EBB68DA64BB68DA6ABB689B6C9A423A
:105030002CD0BB68DB6C002B28D1BB68043318462E
:105040001FF072F8BB689A6CBB68DA62BB68DB6AF7
:10505000C3F10602BB689A61BB68DA6A104B1B6831
:105060009A4203D9BB68DB6A0D4A1360BB68DA6AEF
:1050700013469B0013449B000A4A1A44BB6804333E
:10508000194610461EF0F3FF0123FB60FB6818462B
:105090001037BD4680BD00BFF8C90220A00F060032
:1050A000F0CA0220FCC9022080B586B000AF78604B
:1050B00039607B683B610123FB607B68002B5ED01D
:1050C0003B69DB6C002B04D14FF481512E4803F077
:1050D000E9FB3B699B6C3A689A4202D93B687B6169
:1050E00002E03B699B6C7B613B69DB6A7A699A42AF
:1050F00045D03B69DB6CFA689A4240D1234B1B6870
:105100003A699A4204D141F23B011F4803F0CAFBBD
:105110003B69DB6ABB603B697A69DA623B699B6920
:10512000002B04DB7B69C3F106023B699A613B6992
:105130005969BA6813469B0013449B00144A1344F0
:1051400099421CD13B69043318461EF0EDFF3B69C0
:10515000DA6A104B1B689A4203D93B69DB6A0D4A35
:1051600013603B69DA6A13469B0013449B00084AAC
:105170001A443B690433194610461EF078FF00BFFD
:105180001837BD4680BD00BFA00F0600F8C9022039
:10519000FCC90220F0CA022080B400AF074B1B6894
:1051A000002B04D0054B1B68DA6C0132DA64034B28
:1051B0001B681846BD465DF8047B7047F8C902209D
:1051C00080B586B000AFF860B9607A603B60FDF7EB
:1051D0008DFF264B1B6893F8B830DBB2022B16D03C
:1051E000224B1B68D3F8B410FA68D2430A40C3F8C4
:1051F000B4201E4B1B68012283F8B8203B68002BAB
:1052000005D00121386800F0DDF8FDF75DFFFDF7FE
:1052100081FFFDF76BFF7B68002B05D0134B1B68EC
:10522000D3F8B4207B681A60104B1B6893F8B83031
:10523000DBB2022B02D000237B610AE00B4B1B6820
:10524000D3F8B410BA68D2430A40C3F8B42001239B
:105250007B61064B1B68002283F8B820FDF75AFFDC
:105260007B6918461837BD4680BD00BFF8C90220CB
:1052700080B588B000AFF860B9603B601346FB7141
:105280000123FB61FB68002B04D141F270214948E6
:1052900003F008FBFB68BB61FDF728FF3B68002BB0
:1052A00004D0BB69D3F8B4203B681A60BB6993F89B
:1052B000B830FB75BB69022283F8B820FB79042B58
:1052C0002DD801A252F823F037530300DD5203001A
:1052D000EF520300FF52030009530300BB69D3F8E8
:1052E000B420BB681A43BB69C3F8B42026E0BB698D
:1052F000D3F8B4305A1CBB69C3F8B4201EE0BB69B4
:10530000BA68C3F8B42019E0FB7D022B04D0BB6956
:10531000BA68C3F8B42011E00023FB610EE0BB695A
:10532000D3F8B430B3F1FF3F07D041F2A1212148B7
:1053300003F0B8FA01E000BF00E000BFFB7D012BE5
:1053400030D1BB69043318461EF0EEFEBB69DA6A41
:10535000194B1B689A4203D9BB69DB6A164A136072
:10536000BB69DA6A13469B0013449B00134A1A4434
:10537000BB690433194610461EF079FEBB699B6A6F
:10538000002B04D041F2B0210A4803F08BFAFFF75A
:1053900071FDBB69DA6A0A4B1B68DB6A9A4201D964
:1053A000FDF792FEFDF7B6FEFB6918462037BD46B5
:1053B00080BD00BFA00F0600F0CA0220FCC9022079
:1053C000F8C9022080B584B000AF78603960214B05
:1053D0001B68FB60204B1B68043318461EF0A4FEBC
:1053E0007B68B3F1FF3F0AD13B68002B07D01A4B13
:1053F0001B680433194619481EF039FE26E0FA6886
:105400007B681344BB60144B1B68BA685A60BA6867
:10541000FB689A4209D2124B1A680F4B1B6804337F
:10542000194610461EF047FE10E00E4B1A680A4B54
:105430001B680433194610461EF03DFE0A4B1B68DC
:10544000BA689A4202D2084ABB68136000BF10379C
:10545000BD4680BDECCA0220F8C90220D0CA022095
:10546000A0CA02209CCA022008CB022080B584B0CA
:1054700002AF00237B6000F0F1FA0E4B1B68002B9B
:105480000AD00D4B019303230093002380220B4984
:105490000B481EF0C5FC78607B68002B04D140F2FD
:1054A0001311084803F0FEF97B6818460837BD461B
:1054B00080BD00BF44CB022048CB0220FC0F060079
:1054C000F13F05000410060080B584B000AFF8601D
:1054D000B9607A603B60BB68002B04D140F2651173
:1054E000144803F0DFF9FB69002B1ED000F0B6FA78
:1054F000FB69FA681A60FB69BA689A61FB693A68E5
:10550000DA61FB69BA691A62FB69043318461EF056
:10551000A1FD7B68002B08D0FB6993F8283043F08D
:105520000403DAB2FB6983F8282000BF1037BD46B8
:1055300080BD00BF0410060080B58AB000AFF860DF
:10554000B9607A603B6000237B62FB68002B04D16A
:105550004FF4C1711B4803F0A5F91B4B1B68002BCE
:105560002AD0BB687B617B68BB61FB68FB61BB6861
:10557000052B18DCFFF7AEFC0346022B09D1124BBA
:10558000186807F1140100233A6BFEF72FF87862D0
:1055900012E00D4B186807F1140100230022FEF7FA
:1055A00025F8786208E0084B186807F11401002319
:1055B0003A68FEF7EFF878627B6A18462837BD46EE
:1055C00080BD00BF0410060044CB022080B586B029
:1055D00002AF78603960204B1B68DB68DB68FB60DA
:1055E000FB68043318461EF09FFDFB6893F82830D3
:1055F00003F00403002B1DD0FB689A697B68D11867
:105600007B683A68F86800F0B5F80346002B1AD0BA
:105610000023009300237A680021F868FFF78CFFCD
:10562000B860BB68002B0ED14FF4FC710B4803F03F
:1056300039F908E0FB6893F8283023F00103DAB267
:10564000FB6883F82820FB681B6AF868984700BF4E
:105650001037BD4680BD00BF3CCB022004100600C1
:1056600080B584B000AF78603960FEF763FE07F163
:105670000803184600F05EF8F860BB68002B2AD1DA
:105680003B68002B0AD17A68FB689A4206D8FEF77D
:1056900097FEF9687868FFF799FF1EE03B68002BDA
:1056A00008D0104B1B681B68002B01D1012300E0C0
:1056B00000233B600C4B18687A68FB68D31A3A6881
:1056C00019461EF079FBFEF77BFE0346002B04D142
:1056D000FDF7FAFC01E0FEF773FE00BF1037BD4690
:1056E00080BD00BF40CB022044CB022080B485B0F7
:1056F00000AF78600E4B1B681B68002B01D10122A4
:1057000000E000227B681A607B681B68002B05D1D3
:10571000074B1B68DB681B68FB6001E00023FB6034
:10572000FB6818461437BD465DF8047B704700BF20
:105730003CCB022080B584B000AF7860FEF7D2FE8B
:10574000F8600B4B1B68FA689A4205D200F026F904
:105750007B6801221A6002E07B6800221A60044A1A
:10576000FB681360FB6818461037BD4680BD00BF5C
:105770004CCB022080B586B000AFF860B9607A608B
:105780003B6000237B61FB68BA685A60FB68FA687B
:105790001A61BA687B689A4212D87A683B68D21A52
:1057A000FB689B699A4202D301237B611BE0104B8B
:1057B0001A68FB680433194610461EF07CFC12E0A0
:1057C0007A683B689A4206D2BA683B689A4202D32A
:1057D00001237B6107E0074B1A68FB680433194615
:1057E00010461EF068FC7B6918461837BD4680BD20
:1057F00040CB02203CCB022080B58CB002AFB9E098
:10580000BB68002B13DA07F1080304337B627B6A61
:10581000002B04D14FF436715E4803F043F87B6AE5
:105820001B687A6A50687A6A926811469847BB6822
:10583000002BC0F29E803B693B623B6A5B69002B98
:1058400004D03B6A043318461EF06EFC3B1D18461C
:10585000FFF770FFF861BB68092B00F28B8001A293
:1058600052F823F08D5803008D5803008D58030023
:10587000F75803000B590300495903008D580300E2
:105880008D580300F75803000B5903003B6A93F847
:10589000283043F00103DAB23B6A83F82820FA6823
:1058A0003B6A9B69D118FB68FA69386AFFF762FFA7
:1058B0000346002B5ED03B6A1B6A386A98473B6AF6
:1058C00093F8283003F00403002B53D0FA683B6AA6
:1058D0009B691A440023009300230021386AFFF7D4
:1058E0002BFEB861BB69002B44D140F2133129482B
:1058F00002F0D8FF3EE03B6A93F8283023F0010322
:10590000DAB23B6A83F8282034E03B6A93F8283007
:1059100043F00103DAB23B6A83F82820FA683B6A55
:105920009A613B6A9B69002B04D140F22B311948E4
:1059300002F0B8FF3B6A9A69FB69D118FB69FA6902
:10594000386AFFF717FF15E03B6A93F8283003F039
:105950000203002B03D1386A1EF034FC0AE03B6AD4
:1059600093F8283023F00103DAB23B6A83F8282049
:1059700000E000BF084B1B6807F108010022184631
:10598000FDF77EFF0346002B7FF43AAF00BF2837B8
:10599000BD4680BD0410060044CB022080B588B00F
:1059A00002AF42E02A4B1B68DB681B683B61284B57
:1059B0001B68DB68DB68FB60FB68043318461EF07D
:1059C000B3FBFB681B6AF8689847FB6893F82830BC
:1059D00003F00403002B28D0FB689B693A69134449
:1059E000BB60BA683B699A420ED9FB68BA685A60D4
:1059F000FB68FA681A61164B1A68FB68043319468B
:105A000010461EF058FB10E00023009300233A6973
:105A10000021F868FFF790FD78607B68002B04D1C7
:105A20004FF461710B4802F03DFF094B1B681B6886
:105A3000002BB7D1064B1B687B61074B1B68044AE0
:105A40001360054A7B69136000BF1837BD4680BDEF
:105A50003CCB02200410060040CB022080B500AFF2
:105A6000FDF744FB0D4B1B68002B13D10C481EF0B7
:105A7000D1FA0C481EF0CEFA0B4B094A1A600B4BB8
:105A8000084A1A60002210210520FDF777FD024622
:105A9000024B1A60FDF73EFB00BF80BD44CB0220E5
:105AA00014CB022028CB02203CCB022040CB02208A
:105AB00080B584B000AF78603960FEF73BFC154BD1
:105AC0001A683B681344144A934207D97B680C2236
:105AD0001A60FEF775FC4FF0FF3317E00D4B1B68A3
:105AE000FB600C4B1A683B6813440A4A13600B4B6B
:105AF0001A683B68D31A094A1360094B1A683B6855
:105B00001344074A1360FEF75BFCFB681846103726
:105B1000BD4680BD84C00120E8AE032080C00120C6
:105B200050CB022080B582B000AF78601DF09EFFA0
:105B30000346002B03D0B221044802F0B3FEFEF767
:105B4000F9FB00BF0837BD4680BD00BF4810060006
:105B500080B58AB000AF3B4618460FF0FDFD3B6AAA
:105B6000034A1268134418462837BD4680BD00BF5B
:105B700080C00120F0B5ADF2CC4D06AF07F10C03AB
:105B800018600023C7F8A8340023A7F8A63407F14B
:105B90000C0364228249186828F039FD07F10C03D0
:105BA0001B6800221A70FEF7BFFC0346C7F89C343E
:105BB000D7F89C3419467B4809F0F2FD7A4809F081
:105BC000EFFD07F1140207F1180320211846FEF734
:105BD000B7FC0346C7F89C340023C7F89834C2E0EA
:105BE000D7F8982407F118011346DB0013449B00F3
:105BF0000B440C331B78042B3AD801A252F823F043
:105C00001D5C0300155C0300595C0300615C03002C
:105C1000695C0300722387F8AF342DE0522387F8C4
:105C2000AF34D7F8982407F118011346DB0013446A
:105C30009B000B4404331B68C7F8A834D7F898249A
:105C400007F118011346DB0013449B000B4420337B
:105C50001B88A7F8A6340FE0422387F8AF340BE087
:105C6000532387F8AF3407E0442387F8AF3403E0C9
:105C70003F2387F8AF3400BF0023C7F8A03407F1F3
:105C800014031B68642B15D9D7F8982407F1180161
:105C90001346DB0013449B000B4418331A6807F1CA
:105CA00014031B684149A1FB03135B09B2FBF3F327
:105CB000C7F8A034D7F8982407F118011346DB0081
:105CC00013449B000B4404331D6897F8AF64D7F866
:105CD000982407F118011346DB0013449B000B4482
:105CE00010331B68BB60D7F8982407F118011346DE
:105CF000DB0013449B000B4420331B887B60D7F8E8
:105D0000982407F118011346DB0013449B000B4451
:105D100008331968D7F8982407F118001346DB00F8
:105D200013449B00034418331868D7F8982407F1EC
:105D300018041346DB0013449B0023441C331B68E8
:105D40000493D7F8A0340393029001917A680092EB
:105D5000BB6832462946164809F022FDD7F8983428
:105D60000133C7F89834D7F89824D7F89C349A426E
:105D7000FFF436AFD7F8A834002B0BD0B7F8A63411
:105D800007F10C000093D7F8A8340A4A6421006890
:105D900010F0E0FA00BF07F2B447BD46F0BD00BF07
:105DA000A8100600B4100600C01006001F85EB51B5
:105DB000F81006002C11060090B583B000AF786093
:105DC0007868FFF7D7FEFFF7C3FE04461EF005FA1A
:105DD00003461A4621460B4809F0E2FC0A4B1B8891
:105DE0001946094B9B881846074B1B881A46064BD9
:105DF0009B88D31A0246054809F0D2FC00BF0C3735
:105E0000BD4690BD3411060080EB022054110600FF
:105E100080B500AF154B0A221A60144B0B225A6052
:105E2000124B4FF0FF329A60104B4FF0FF32DA60A6
:105E30000E4B00221A610D4B00221A750B4B0E22DD
:105E40005A750A4B4FF0EB729A61084B07221A778A
:105E5000074B00221A71064807F082FA0022034914
:105E6000034807F017FA00BF80BD00BF88C00120BB
:105E7000A8C00120F0B5A1B004AF002387F86F30AF
:105E80000023BB663B1D64220021184628F0E2F97E
:105E900007F036FE03461C4607F03EFE03461D464D
:105EA00007F046FE03461E4607F04EFE03460093EB
:105EB00033462A462146464823F023FAFFF7A8FF37
:105EC000444809F06DFC444809F06AFC424809F076
:105ED00067FC414809F064FC404809F061FC404817
:105EE00009F05EFC07F00CFE034619463D4809F038
:105EF00057FC07F011FE034619463B4809F050FCD9
:105F000007F016FE03461946384809F049FC07F029
:105F10001BFE03461946364809F042FC354809F095
:105F20003FFC354809F03CFC3B1D1846FFF744FF99
:105F3000324B1B68002B0BD0314809F031FC2F4B42
:105F40001B6807F1680210469847034687F86F30D0
:105F50002C4809F025FCBB6E002B18D107F0D0FDB2
:105F600003461C4607F0D8FD03461D4607F0E0FD3A
:105F700003461E4607F0E8FD02463B1D01930092D2
:105F800033462A462146204823F0BBF919E007F0A2
:105F9000B7FD03461C4607F0BFFD03461D4607F04C
:105FA000C7FD03461E4607F0CFFD0246BB6E0293B7
:105FB0003B1D0193009233462A462146134823F0A5
:105FC000A0F997F86F3018467437BD46F0BD00BF92
:105FD00078110600CC110600D0110600F011060061
:105FE0001C12060034120600441206005412060069
:105FF00064120600741206007812060054CB0220C8
:1060000090120600A4120600CC1206001813060017
:1060100080B483B000AF7860044A7B68136000BF2F
:106020000C37BD465DF8047B704700BF54CB02209F
:1060300080B584B000AF78607B681B78002B0DD0F2
:106040007B6899687B681B78002B01D0544B00E07B
:10605000544B1A46544809F043FB0CE07B6899689E
:106060007B681B78002B01D04D4B00E04D4B1A464E
:106070004E4809F035FB7B685B68022B08D17868D5
:106080001EF052FA03461946494809F029FB70E010
:106090007B685B68032B08D178681EF06DFA0346B5
:1060A0001946444809F01CFB63E07B685B68042BDD
:1060B0002AD10023FB607B68103318461EF07BFA60
:1060C0000246FB68934234BF01230023DBB2002B5E
:1060D0000FD07B681033F96818461EF07CFA03462F
:1060E0001B781946344809F0FBFAFB680133FB6062
:1060F000E1E77B68103318461EF05DFA0346194647
:106100002E4809F0EDFA34E07B685B68012B0DD175
:1061100078681EF0CDF90346002B01D0284B00E033
:10612000284B1946234809F0DBFA22E00023BB6024
:106130007B68103318461EF03EFA0246BB68934255
:1061400034BF01230023DBB2002B0FD07B68103358
:10615000B96818461EF03FFA03461B7819461648E0
:1061600009F0BEFABB680133BB60E1E7164809F0ED
:10617000B7FA7B68DB681B78002B06D07B68DB688E
:106180001946124809F0ACFA05E07B68DB6819464D
:106190000F4809F0A5FA00BF1037BD4680BD00BF0B
:1061A0006C130600701306007413060080130600BB
:1061B0008C130600981306009C130600A413060017
:1061C000AC130600B4130600BC130600D01306007F
:1061D000D813060090B589B000AFF860B9607A6056
:1061E000FB685B68032B2BD0786828F0F6F9034630
:1061F00007F110007A68F96800F0FEF807F1100363
:1062000018461EF0F7F90346002B01D0002411E0D8
:1062100007F1100318461EF008FA044607F11003B0
:1062200018461EF012FA03461A462146B8681EF0B8
:106230001DFA012407F1100318461DF0D1F821E0E2
:10624000786828F0CAF9F861FB6901331946B86823
:106250001EF01BFA034683F00103DBB2002B04D0CF
:106260000B4809F03DFA00240CE0FB6901337A6821
:1062700013441A467968B8681EF033FAB8681EF0FD
:106280003FFA0124234618462437BD4690BD00BF7F
:10629000DC130600B0B582B000AF78607B6803F114
:1062A00010047B68103318461EF085F90346194622
:1062B00020461EF0EAF9034683F00103DBB2002B0F
:1062C00001D0002329E07B681C3318461EF092F9A8
:1062D0000346002B07D07B689B681946114809F0DC
:1062E000FFF9002319E07B6803F110047B681C337D
:1062F00018461EF09AF905467B681C3318461EF0B6
:10630000A4F903461A46294620461EF0AFF97B68D9
:10631000103318461EF0F4F9012318460837BD461D
:10632000B0BD00BFFC13060080B582B000AF78603E
:1063300039607B685B68022B09D07B6899687B6851
:106340005B681A46084809F0CBF9002307E07B6830
:1063500010333A68194678681DF0AEFF03461846B8
:106360000837BD4680BD00BF2414060080B582B04A
:1063700000AF78600B46FB707B685B68012B09D02F
:106380007B6899687B685B681A46084809F0A8F939
:10639000002307E07B681033FA78194678681DF00F
:1063A000C4FF034618460837BD4680BD601406008A
:1063B00080B584B000AFF860B9607A60FB685B6854
:1063C000042B09D0FB689968FB685B681A4609488A
:1063D00009F086F9002308E0FB6803F110017B68EF
:1063E000BA68F8681DF0F2FF034618461037BD463C
:1063F00080BD00BF9814060080B594B000AFF8606F
:10640000B9607A603B60F8681CF0DDFF07F11C039F
:1064100020220021184627F01DFF1F23FB643A6845
:10642000FB6C9A4201D23B68FB6407F11C03FA6CD7
:106430007968184627F0EAFEBB685B68042B00F217
:10644000AD8001A252F823F08D6503005D64030066
:10645000E5640300116503001F6503003A685249B3
:10646000786828F0C2F80346002B07D03A684F49F5
:10647000786828F0BAF80346002B05D10122F968A4
:10648000B8681DF052FF88E03A684949786828F0FA
:10649000ACF80346002B07D03A684649786828F0E4
:1064A000A4F80346002B05D10022F968B8681DF056
:1064B0003CFF72E00023BB6107F1180107F11C03E8
:1064C0000022184610F000F8F863FB6B002B14BF95
:1064D00001230023DBB21A46F968B8681DF025FFD6
:1064E00000BF5AE000237B6107F1140107F11C0390
:1064F000002218460FF0E8FF38647A6907F11C03A0
:106500009A4245D03A6CF968B8681DF0D5FE46E06D
:106510003B687A68F968B8681DF0A1FE3DE03B6809
:1065200003F00103002B35D13B685B081946F8687E
:106530001EF0ABF8034683F00103DBB2002B2BD136
:106540003B685B081946F8681EF010F90023BB642D
:106550003B685B08BA6C9A4218D2BB6C5B007A68E5
:1065600013440221184624F0E7F978647B6C002B71
:106570000BDBB96CF8681EF02EF803467A6CD2B2C9
:106580001A70BB6C0133BB64E2E700BF00BF04E0DC
:1065900000BF02E000BF00E000BF00BF00BFF8681E
:1065A0005037BD4680BD00BFAC130600D4140600B2
:1065B000B4130600DC140600B0B584B000AF7860F8
:1065C000396078681EF0A0FB02463B6893428CBF9E
:1065D00001230023DBB2002B02D0284809F00EFB78
:1065E00078681EF0A2FB02463B6893428CBF0123F1
:1065F0000023DBB2002B3DD078681DF0DCFFF86093
:106600007B681B6818461EF0A0FB04467B685B682D
:1066100018461EF09AFB03462246396878681EF039
:10662000A3FBB8607B681C687B685D687B68184664
:106630001CF013FF03461A46294620461CF023FF90
:1066400078687B6819687B689B681A467B681B685A
:10665000D31A1A461CF046FF7B68BA681A60BA68FB
:10666000FB681A447B685A607B681A683B681A4466
:106670007B689A6000BF1037BD46B0BDE4140600C9
:10668000B0B586B000AF786039603B68002B6AD047
:106690007B689B681A467B685B68D31A1A463B681E
:1066A00093420FD87B685C687B6818461CF0D5FE67
:1066B00003461A46396820461EF0CDFC02467B6828
:1066C0005A6050E02A4A396878681EF0E3FC786125
:1066D00078681DF070FF38617B68796918461EF094
:1066E00021FDF860FB68BB607B681C687B685D68A7
:1066F0007B6818461CF0B1FE0346FA68294620461E
:106700001EF024FDB8607B6818461CF0A6FE034608
:106710001A463968B8681EF09EFCB8607B681C6831
:106720007B685D687B6818461CF097FE03461A4636
:10673000294620461CF0A7FE78687B6819687B68AC
:106740009B681A467B681B68D31A1A461CF0CAFE5F
:106750007B68FA681A607B68BA685A60FA687B6975
:106760001A447B689A6000BF1837BD46B0BD00BFB1
:10677000F4140600B0B58AB000AFF860B9607A6072
:106780003F4A0121F8681EF085FC7862F8681DF028
:106790004CFF03467B6107F1140207F10803114621
:1067A00018461EF02BFF03463B62FB68796A1846C9
:1067B0001EF0B8FCF861FB69BB61FC68FA693B6AD2
:1067C000D51878681EF005F903461A462946204672
:1067D0001EF09CFB0023BB61FB681C6807F10803EB
:1067E00018461EF020FF03461D68FB6818461CF083
:1067F00034FE0346FA69294620461EF0A7FCB8611C
:10680000BB690133BB6107F1080318461EF00BFF9B
:1068100003461C68FB685D68FB6818461CF01DFE9B
:106820000346BA69294620461EF090FCB861FB6811
:106830001C68FB685D68FB6818461CF00EFE03468A
:106840001A46294620461CF01EFEF868FB681968A7
:10685000FB689B681A46FB681B68D31A1A461CF033
:1068600041FEFB68FA691A60FB68BA695A60FA6906
:106870007B6A1A44FB689A6000BF2837BD46B0BDEA
:106880001015060080B500AF094B1B6803F001032B
:10689000002B0AD1074800F013F8054B01221A60BB
:1068A000054A0649034827F046FC024B184680BDBE
:1068B00090CB022058CB022078C001202D5D05002E
:1068C00080B582B000AF78607B6800221A707B6868
:1068D000043300221A605A609A60DA601A617B6899
:1068E000183318461FF022FC7B68243318461FF02B
:1068F00045FC7B6800221A637B6800225A637B6830
:10690000094A5A617B6804338021184624F006FE48
:10691000064B074A0749786800F020F97B6818465B
:106920000837BD4680BD00BF94CB0220535D0500F3
:106930002C1506003815060080B586B000AF7860CB
:10694000396040F2011200212B4827F083FC4FF4FC
:1069500080723968284827F059FC2749274808F0F1
:10696000BFFE274924480FF073FD786124490020B9
:106970000FF06EFD3861796978681FF04AFAF860A7
:10698000FB68002B13D1796978681FF099FAB86019
:10699000BB68002B0BD0BB681B681946194808F070
:1069A0009FFEBB689B6838699847012320E0FB681D
:1069B000002B05D17969144808F092FE002317E0F6
:1069C0003A69796978681FF0D0FA0346002B0AD03B
:1069D0000E4808F085FE0E4808F082FE786800F048
:1069E0000DF9012304E039690A4808F079FE002313
:1069F00018461837BD4680BD14CC02203C15060051
:106A000044150600481506006015060084150600AA
:106A1000981506009C15060080B584B000AF78601C
:106A20007B6804334FF480720849184609F044F833
:106A3000F860FB68002B04DD04497868FFF77CFFF1
:106A400000E000BF1037BD4680BD00BF18CD02205A
:106A500090B591B000AF786039607B681833FB6304
:106A6000F86B1FF0B3FB0346BB63F86B1FF0BEFB74
:106A700003467B6307F1340207F1380311461846D9
:106A80001FF0C5FB0346002B2FD007F13803184633
:106A90001FF0E6FB024607F10C03114618461FF0F3
:106AA00066F907F10C0318461DF0C1FB044638686F
:106AB0001DF0BDFB03461946204624F036F8034678
:106AC000002B07D038681DF0B2FB0346194620485A
:106AD00008F006FE07F10C0318461CF061FC07F1F4
:106AE000380318461FF0ABFBC4E77B6803F11804BA
:106AF0007B681833184600F03FFB03460133194604
:106B0000204600F04FFB7B681833184600F0BEFBB0
:106B100004467B681833184600F02EFB0346013309
:106B20009C4234BF01230023DBB2002B06D009486E
:106B300008F0D6FD7721084801F0B4FE7B681833D1
:106B4000396818461FF0A3FB00BF4437BD4690BD0F
:106B5000B8150600EC1506000C16060090B589B0B5
:106B600000AFF860B9607A603B60B86827F035FD27
:106B70000346172B03D982211E4801F093FEBB6800
:106B80007B617B68BB613B68FB61FB6803F12404AC
:106B9000FB682433184600F08FFB03460133194687
:106BA000204600F09FFBFB682433184600F00EFCE3
:106BB0000446FB682433184600F07EFB034601338D
:106BC0009C4234BF01230023DBB2002B06D00A48CD
:106BD00008F086FD8C21074801F064FEFB68243331
:106BE00007F11402114618461FF082FB00BF24373C
:106BF000BD4690BD0C1606004816060080B586B04E
:106C000000AF7860384808F06BFD384808F068FD40
:106C10007B68183318461FF0A4FB034683F001037A
:106C2000DBB2002B2AD07B681833184600F0A4FA98
:106C3000034619462E4808F053FD00237B617B680C
:106C40001833184600F098FA02467B69934234BF25
:106C500001230023DBB2002B0DD07B681833796948
:106C600018461FF06BFBF860F868FFF7E1F97B69E5
:106C700001337B61E3E71F4808F032FD7B68243372
:106C8000184600F019FB034619461B4808F028FD7A
:106C900000233B617B682433184600F00DFB02465D
:106CA0003B69934234BF01230023DBB2002B0DD09C
:106CB0007B682433396918461FF06EFBB860B868EA
:106CC00001F0E4F83B6901333B61E3E70B4808F06E
:106CD00007FD0B4808F004FD0A4808F001FD00BF5D
:106CE0001837BD4680BD00BF64160600701606004A
:106CF00098160600AC160600E81606009815060061
:106D0000F81606001417060090B58DB000AFF860B5
:106D1000B9607A6007F11C0300221A605A609A6019
:106D200007F11C037A68B968184623F07DFF07F164
:106D30001C03184624F074FA0023FB62FB68183326
:106D4000184600F019FA0246FB6A934234BF012349
:106D50000023DBB2002B00F0AC80FB681833F96A2B
:106D600018461FF0EBFAB862BB6A1B78002B40F0A4
:106D70009580B86A1DF05BFA024607F11C031146C4
:106D8000184624F03AFAB86A1DF05DFA0346042B5F
:106D900000F28B8001A252F823F000BF936E030033
:106DA000B16D0300E16D03000F6E03003D6E030043
:106DB000B86A1DF07DFB03461A4607F11C03114615
:106DC000184624F064F90346002B0CBF012300236E
:106DD000DBB2002B64D0C2213B4801F063FD5FE0D1
:106DE000B86A1DF0A1FB024607F11C0311461846C4
:106DF00024F008F90346002B0CBF01230023DBB26B
:106E0000002B4FD0C621304801F04CFD4AE0B86A53
:106E10001DF0B2FB024607F11C031146184624F090
:106E2000ECF90346002B0CBF01230023DBB2002B3F
:106E30003AD0CA21244801F035FD35E007F11003AE
:106E4000B96A18461DF059FB07F1100318461FF0E8
:106E5000C9FA044607F1100318461DF0ACFB0246C0
:106E600007F11C032146184624F06CF90346002B59
:106E70000CBF01230023DBB2002B03D0CF2112482B
:106E800001F010FD00BF07F1100318461CF0A8FA2E
:106E90000BE0D3210C4801F005FD06E000BF04E043
:106EA00000BF02E000BF00E000BFFB6A0133FB62ED
:106EB00044E707F11C03184624F009FA7B6A1846D8
:106EC0003437BD4690BD00BF0C16060080B598B0A3
:106ED00000AFF860B9607A6007F1440300221A60DD
:106EE0005A609A6007F144037A68B968184623F03B
:106EF0009BFE0023FB6500233B6500233B640023CE
:106F0000BB6507F14403F96D184624F0BAFA03464D
:106F1000002B0DD007F14403F96D184624F09EF9BB
:106F20000246FB6D1344FB6540F2E7333B640BE024
:106F300007F1400207F14403F96D184624F0A3F964
:106F40000246FB6D1344FB6500237B653B6C7A6D49
:106F50009A4280F0C18007F14403F96D184624F08D
:106F6000D4F90346002B40F0B68007F1280207F160
:106F700044001823F96D24F0F6F80246FB6D134423
:106F8000FB6507F14403F96D184624F0F5F9034653
:106F9000002B1CD000237B6207F1240207F144037D
:106FA000F96D184623F0D5FF0246FB6D1344FB65CF
:106FB0007A6A07F128031946F8681FF00AF80346B1
:106FC000002B00F08480BB6D0133BB657FE007F1CF
:106FD0004403F96D184624F07DFA0346002B1DD0BA
:106FE000002387F8233007F1230207F14403F96DEA
:106FF000184624F023F80246FB6D1344FB6597F80E
:10700000232007F128031946F8681EF0FBFF03460A
:10701000002B5CD0BB6D0133BB6558E007F1440326
:10702000F96D184624F0EFF90346002B1BD007F149
:10703000180307F11C0207F14400F96D24F0B8F8B9
:107040003865FA6D3B6D1344FB65FA69BB6907F15E
:107050002801F8681EF0A2FF0346002B37D0BB6D55
:107060000133BB6533E007F14403F96D184624F0A2
:10707000ABF90346002B20D000237B6100233B614A
:1070800007F1100307F1140207F14400F96D24F031
:1070900023F83865FA6D3B6D1344FB657A693B69EB
:1070A000DBB207F12801F8681EF0D0FF0346002B81
:1070B0000DD0BB6D0133BB6509E07A6CFB6D1344E9
:1070C0001B7803F0E0031946064808F009FB7B6DC6
:1070D00001337B653AE700BFBB6D18466037BD469C
:1070E00080BD00BF3C17060080B582B000AF78605D
:1070F00078681EF008FE0346002B0AD0074808F007
:10710000EFFA0021786800F017FB002178681EF084
:10711000EBFD00BF0837BD4680BD00BF5C17060011
:1071200080B588B002AFF860B9607A603B60B9683A
:10713000F8681EF0BDFF78613B8C7A699A4208DBE3
:10714000BB8C7A699A4204DC7B699AB23B681A80EC
:107150000BE07B6801221A703A8CB98C7B69009332
:107160000B46B968034808F0BBFA00BF1837BD46A4
:1071700080BD00BF7417060080B483B000AF786094
:107180007B685B681A467B681B68D31ADB10044A6D
:1071900002FB03F318460C37BD465DF8047B7047CD
:1071A000CDCCCCCCB0B584B000AF78603960786815
:1071B0001FF0BCF902463B6893428CBF01230023B9
:1071C000DBB2002B02D02F4808F018FD786800F0E1
:1071D0005DF802463B6893428CBF01230023DBB27B
:1071E000002B4AD07868FFF7C7FFF8607B681B6800
:1071F00018461FF0ACF904467B685B6818461FF020
:10720000A6F903462246396878681FF0AFF9B860DE
:107210007B681C687B685D687B6818461FF0FEF819
:1072200003461A46294620461FF00EF978687B6807
:1072300019687B689B681A467B681B68D31ADB1049
:10724000114A02FB03F31A461FF0ACF97B68BA68D7
:107250001A60FA6813469B001344DB001A46BB68A9
:107260001A447B685A607B6819683A6813469B0029
:107270001344DB00CA187B689A6000BF1037BD4614
:10728000B0BD00BFC0170600CDCCCCCC80B483B05D
:1072900000AF78607B689B681A467B681B68D31ACE
:1072A000DB10044A02FB03F318460C37BD465DF8B9
:1072B000047B7047CDCCCCCC80B483B000AF786079
:1072C0007B685B681A467B681B68D31A9B10044A6C
:1072D00002FB03F318460C37BD465DF8047B70478C
:1072E000ABAAAAAAB0B584B000AF7860396078685C
:1072F0001FF07EF902463B6893428CBF01230023B6
:10730000DBB2002B02D02F4808F078FC786800F040
:107310005DF802463B6893428CBF01230023DBB239
:10732000002B4AD07868FFF7C7FFF8607B681B68BE
:1073300018461FF06EF904467B685B6818461FF01C
:1073400068F903462246396878681FF071F9B86019
:107350007B681C687B685D687B6818461FF09BF83B
:1073600003461A46294620461FF0ABF878687B682A
:1073700019687B689B681A467B681B68D31A9B1048
:10738000114A02FB03F31A461FF06EF97B68BA68D4
:107390001A60FA6813465B0013449B001A46BB68E8
:1073A0001A447B685A607B6819683A6813465B0028
:1073B00013449B00CA187B689A6000BF1037BD4613
:1073C000B0BD00BFC0170600ABAAAAAA80B483B0A4
:1073D00000AF78607B689B681A467B681B68D31A8D
:1073E0009B10044A02FB03F318460C37BD465DF8B8
:1073F000047B7047ABAAAAAA80B582B000AF7860C0
:107400007B6819687B689B681A467B681B68D31A7F
:10741000DB10064A02FB03F31A4678681FF0C2F835
:107420007B6818460837BD4680BD00BFCDCCCCCCAC
:1074300080B582B000AF78607B6819687B689B6814
:107440001A467B681B68D31A9B10064A02FB03F39B
:107450001A4678681FF008F97B6818460837BD4659
:1074600080BD00BFABAAAAAAB0B58AB000AFF860D1
:10747000B9607A60464A0121F8681FF07BFA7862A9
:10748000F8681EF0A3FE03467B6107F1140207F1C2
:1074900008031146184600F017F903463B62FB68E3
:1074A000796A18461FF0EDF9F861FB69BB61FC6869
:1074B0003A6A13469B001344DB001A46FB699D1889
:1074C00078681EF0D9FE03461A46294620461FF06A
:1074D0007CF80023BB61FB681C6807F108031846B1
:1074E0001FF019F803461D68FB6818461EF096FF4A
:1074F0000346FA69294620461FF084FAB861BB6941
:107500002833BB6107F1080318461FF004F803464F
:107510001C68FB685D68FB6818461EF07FFF034629
:10752000BA69294620461FF06DFAB861FB681C68ED
:10753000FB685D68FB6818461EF070FF03461A463C
:10754000294620461EF080FFF868FB681968FB6832
:107550009B681A46FB681B68D31ADB100D4A02FBB6
:1075600003F31A461FF01EF8FB68FA691A60FB68FD
:10757000BA695A607A6A13469B001344DB001A46C4
:10758000FB691A44FB689A6000BF2837BD46B0BD4E
:10759000D0170600CDCCCCCCB0B58AB000AFF86027
:1075A000B9607A60464A0121F8681FF0F4FA7862FF
:1075B000F8681FF038FB03467B6107F1140207F1FE
:1075C00008031146184600F09BF803463B62FB682F
:1075D000796A18461FF056FAF861FB69BB61FC68CE
:1075E0003A6A13465B0013449B001A46FB699D18D8
:1075F00078681EF072FE03461A46294620461FF0A0
:1076000046F80023BB61FB681C6807F108031846B5
:107610001FF019FB03461D68FB6818461EF03BFF70
:107620000346FA69294620461FF018FBB861BB697A
:107630000C33BB6107F1080318461FF004FB034637
:107640001C68FB685D68FB6818461EF024FF034653
:10765000BA69294620461FF001FBB861FB681C6827
:10766000FB685D68FB6818461EF015FF03461A4666
:10767000294620461EF025FFF868FB681968FB685C
:107680009B681A46FB681B68D31A9B100D4A02FBC5
:1076900003F31A461EF0E8FFFB68FA691A60FB68FC
:1076A000BA695A607A6A13465B0013449B001A4613
:1076B000FB691A44FB689A6000BF2837BD46B0BD1D
:1076C000D0170600ABAAAAAA90B583B000AF786025
:1076D000396078681EF01FFF03461B681C46386837
:1076E0001EF019FF03461B68E31ADB10034A02FB76
:1076F00003F318460C37BD4690BD00BFCDCCCCCCB3
:1077000090B583B000AF7860396078681FF09BFA5D
:1077100003461B681C4638681FF095FA03461B6831
:10772000E31A9B10034A02FB03F318460C37BD46CD
:1077300090BD00BFABAAAAAA80B588B000AF7860A0
:107740000B46FB704FF4FA63BB61B86908F0B6F8FA
:1077500078617B69002B06D12F4807F0C1FF2221F9
:107760002E4801F09FF8BA690021786926F072FD71
:10777000BA6979697868FFF7C7FA0346FB60FB7856
:10778000002B0BD0FB681946254807F0A9FF254BB5
:107790005A68244B9B681344FB6107E0FB68194659
:1077A000214807F09DFF1F4B5B68FB611F4BDB68A7
:1077B000002B06D01D4BDB68FA6808321146F869C9
:1077C000984700233B61194B5B683969FA6988184F
:1077D0000422144998473B6904333B61134B5B68AF
:1077E0003969FA69881807F10C01042298473B6946
:1077F00004333B610D4B5B683969FA698818FA6894
:10780000796998470A4807F06BFF786908F038F8FB
:1078100000BF2037BD4680BDEC170600F4170600F8
:107820003C1806002CCE02205C1806001CCE02205C
:107830007818060080B584B000AF78600C4B1B68E8
:107840000C4A51680B4A9268881807F10C0104220F
:1078500098470346002B06D0064B1A68FB689A42ED
:1078600001D1012300E0002318461037BD4680BD3A
:107870001CCE02202CCE022080B582B000AF0023A7
:107880007B600D4B5B680D4A51680C4A9268881802
:10789000391D042298470346002B04D0084807F0FE
:1078A0001FFF012303E0074807F01AFF00231846D3
:1078B0000837BD4680BD00BF1CCE02202CCE022062
:1078C000881806009C18060080B588B000AFF860E4
:1078D000B9601346FB710023BB61274B5B68FB61FA
:1078E000FB79002B04D0244B9B68FA691344FB619D
:1078F00000237B61214B1B68B969FA69881807F17D
:10790000140104229847BB690433BB611A4B1A68FF
:107910007B699A4208D07969174B1B681A46184848
:1079200007F0DEFE002323E0144B1B68B969FA69F7
:10793000881807F1100104229847BB690433BB6122
:107940003B6919460F4807F0CBFE3B69BA689A427B
:1079500001D200230CE0094B1B68B969FA69881849
:107960003A69F9689847BA693B691344BB613B6956
:1079700018462037BD4680BD2CCE02201CCE0220EA
:10798000BC180600D818060080B58AB000AF786031
:107990004FF4FA633B620023FB614FF4FA63BB616F
:1079A000B86907F08BFF78617B69002B06D13A48F4
:1079B00007F096FE7F21394800F074FFBA69002174
:1079C000786926F047FC0022B9697869FFF77CFFE7
:1079D00038613B69002B07D1F86907F051FF7869DE
:1079E00007F04EFF002352E0386A07F067FFF861A6
:1079F000FB69002B06D1284807F072FE8E2127482C
:107A000000F050FF3A6A0021F86926F023FC3A6A38
:107A1000F9697868FFF778F9F860FB68002B07D1FF
:107A2000F86907F02DFF786907F02AFF00232EE0A0
:107A30003A69FB689A4207D0F86907F021FF786934
:107A400007F01EFF002322E000237B627A6A3B6975
:107A50009A4215D2FA697B6A13441A7879697B6A6B
:107A60000B441B789A4207D0F86907F009FF786940
:107A700007F006FF00230AE07B6A01337B62E5E73B
:107A8000F86907F0FDFE786907F0FAFE0123184651
:107A90002837BD4680BD00BFEC170600F41706006E
:107AA00080B586B000AF78604FF4FA633B61386907
:107AB00007F004FFF860FB68002B04D1264807F0AC
:107AC0000FFE002343E03A690021F86826F0C2FB6C
:107AD00000237B617868FFF7ADFE0346002B1CD0C6
:107AE0001E4807F0FDFD01223969F868FFF7ECFE3A
:107AF00078611B4807F0F4FDFFF7BEFE7B69002BA1
:107B000004D0012178681EF0EFF806E0154807F070
:107B1000E7FD002178681EF0E7F87B69002B05D1AE
:107B200000223969F868FFF7CFFE78617B69002B86
:107B300004D1F86807F0A4FE002308E07A69F96828
:107B40007868FFF7C3F9F86807F09AFE0123184632
:107B50001837BD4680BD00BFEC170600F4180600BC
:107B6000181906003019060080B584B000AF78609F
:107B7000FEF788FEF8603B4807F0B2FDFCF7B2FC68
:107B80000246394B1A60394B1B68002B1CD0374B0F
:107B90001B6803F56A436033334A1268934213D972
:107BA000334B1B7883F00103DBB2002B05D0314847
:107BB00007F096FD304807F093FD2D4B01221A7017
:107BC000F868FEF729FF1AE0294B1B78002B10D02C
:107BD0000021F868FFF7B0FD284807F081FD28482C
:107BE00007F07EFD274B9B68002B02D0254B9B683E
:107BF00098471F4B00221A701C4B00221A6041F25A
:107C00008833214A4FF0FF310020FDF7D9FAB860E0
:107C1000FCF768FC0246144B1A60BB68002B06D1C7
:107C2000134B1B78002B02D0F868FEF7F5FE164BBD
:107C30001B6803F00103002B03D00B4B1B680B4A9E
:107C40001360114B1B6803F00203002B96D0074B07
:107C500000221A600B4B9B68002B8FD0094B9B684E
:107C600098478BE75C19060040CE02203CCE0220EC
:107C7000AAE902207419060098190600BC1906002A
:107C8000D01906001CCE022038CE022080B582B06A
:107C900000AF78600A4807F023FDFEF7F3FD0346C6
:107CA00018461EF090F8074807F01AFDFEF7EAFDA7
:107CB00003461846FEF7A2FF00BF0837BD4680BD49
:107CC000F41906000C1A060080B584B000AF786085
:107CD000FEF7D8FDF8600021F868FFF72DFDF86881
:107CE000FEF78CFF054B1868002301220221FDF7E7
:107CF000BFFA00BF1037BD4680BD00BF18CE0220BE
:107D000090B589B002AF3C4684E80F007B68002B39
:107D100004D140F229114B4800F0C4FD3B68002B10
:107D200004D14FF49571474800F0BCFD464B1C460A
:107D30003B460FCB84E80F00444B07F1280207CAEB
:107D400083E80700414B9B68002B03D13F4B4FF466
:107D500080629A603D4B1B68002B04D140F23511C4
:107D6000384800F09FFD394B1B68B3F1FF3F04D149
:107D700040F23711334800F095FDFEF783FD78613E
:107D8000334B344A34497869FEF7E8FE334B344AC2
:107D900034497869FEF7E2FE334B344A3449786956
:107DA000FEF7DCFE7869FFF77BFE034683F00103F4
:107DB000DBB2002B0ED02F4807F092FC78691EF042
:107DC00002F8002178691DF08FFFFFF755FD2A4862
:107DD00007F086FC78691DF096FF034683F00103E7
:107DE000DBB2002B12D07869FFF7CEFD034683F09B
:107DF0000103DBB2002B09D0204807F071FCFEF72D
:107E000041FD034600211846FFF796FC1C4B0193E9
:107E1000012300930023FA221A491B481CF000F8A2
:107E20000346002B0CBF01230023DBB2002B04D040
:107E30004FF4A871034800F035FD00BF1C37BD4664
:107E400090BD00BFF41706001CCE02202CCE0220ED
:107E5000F7700500241A0600301A06008D7C030016
:107E6000381A0600541A0600C97C03005C1A060082
:107E7000741A06007C1A06000C1A0600A01A0600E6
:107E800018CE0220B81A0600697B030080B582B0C4
:107E900000AF78607B681B6819460E4807F020FC2D
:107EA0007B685B68002B0BD07B685B681B78002BC2
:107EB00006D07B685B681946074807F011FC05E0AF
:107EC0007B685B681946054807F00AFC00BF083765
:107ED000BD4680BDC41A0600CC1A0600D41A06009E
:107EE00080B588B000AF7860396007F10C030022DC
:107EF0001A605A609A6007F10C030021184625F0B9
:107F000009FBF861FB69002B05DAF9691A4807F0EB
:107F1000E7FB00232CE007F10C031946386809F051
:107F2000BFF80346FB76FB7E83F00103DBB2002B38
:107F300003D13B68DB69002B09D1F9690F4807F0D1
:107F4000CFFBFB69184609F02DFB002310E0FB690D
:107F5000184609F027FB034683F00103DBB2002B30
:107F600005D0F969064807F0BBFB002300E00123B8
:107F700018462037BD4680BDD81A0600001B0600F3
:107F8000381B060080B584B000AF786039600023EC
:107F9000FB7339687868FFF7A3FF0346BB73BB7BAD
:107FA00083F00103DBB2002B0CD0FB7B0133FB73AE
:107FB000FB7B0F2BEDD908F089FE3121044800F03E
:107FC00071FCE6E7BB7B18461037BD4680BD00BF9D
:107FD000641B060090B58FB000AF786039607B6895
:107FE0005A697B685B691B681B6810469847C7E93C
:107FF0000A0107F108031C220021184626F02AF97D
:108000003B68B3F90630BB833B685B79184609F0DF
:10801000CDFB034687F82130D7E90A34012B74F1F0
:10802000000301DBBB6AFB603B681B79184607F065
:1080300045FC7862002387F837307B6A002B4CD0F0
:108040003B6819683B681B791A46786A26F0DEF8A7
:108050003B685B79184609F0CFFB034687F822306E
:1080600097F82230412B02D0422B0AD013E03B6814
:108070001B791946786A25F0D9F8034687F8373016
:1080800010E03B681B791946786A25F005F903462C
:1080900087F8373006E0134807F022FB786A07F0CC
:1080A000EFFB1BE07B68183397F83720796A184696
:1080B00008F024F80346002B08D097F8371007F192
:1080C00008020023786A09F077F802E0064807F012
:1080D00007FB786A07F0D4FB00E000BF3C37BD46E1
:1080E00090BD00BFA81B0600C81B060082B080B56B
:1080F00086B002AFF860B9607A60FB61FB681A462F
:108100000023136053609360D360FB6800221A74ED
:10811000FB68BA685A61FB681833282200211846A8
:1081200026F098F8FB68183318461EF0F6FFFB6837
:10813000403307F12C0207CA83E807000E4B1B7877
:1081400083F00103DBB2002B03D068210B4800F061
:10815000A9FB094B00221A70BB6A009307F11C03AC
:108160000ECB786808F0D2FDFB6818461037BD4684
:10817000BDE8804002B0704741C30120641B060087
:1081800082B090B589B006AF7860396007F1180108
:1081900081E80C00164B1B6803F00103002B1BD178
:1081A00003AC07F1280393E8070084E807006C4656
:1081B00007F11C0393E8070084E80700BB693A68ED
:1081C00079680C48FFF792FF094B01221A600A4AAE
:1081D0000A49084825F0AFFF094B064A1A60054BCB
:1081E00018460C37BD46BDE8904002B0704700BF4E
:1081F00094CE022048CE022078C001207D71050077
:1082000044CE022080B500AF054B1B68002B03D184
:108210007521044800F046FB014B1B68184680BDE1
:1082200044CE0220641B06002DE990488CB000AFBC
:1082300078600B46FB707B681B7C83F00103DBB22C
:10824000002B03D07A21534800F02CFB7B685A693D
:108250007B685B691B681B6810469847C7E9060185
:108260004FF000034FF00004C7E90A344A4B7B6229
:108270002D2387F82330FB78022B0CD17B681B88D9
:108280009BB24FF00004C7E90A34444B7B6263237E
:1082900087F823300EE0FB78012B0BD17B685B88DD
:1082A0009BB24FF00004C7E90A343D4B7B62732355
:1082B00087F82330D7E90A34234307D197F82330CE
:1082C0001A46796A374807F00BFA5FE07B681B6C47
:1082D000FA7810469847D7E90A0107F083F9034670
:1082E0001A46796A304807F0FBF9D7E90612D7E950
:1082F0000A3413EB010B44EB020CC7E904BC7B68A6
:108300005A697B685B691B681B6810469847C7E918
:108310000601D7E90612D7E90434994272EB040347
:10832000B4BF01230023DBB2002B28D0D7E904120D
:10833000D7E90634C91A62EB04028B4694465846C4
:10834000614607F04FF903461A46796A174807F065
:10835000C7F97B685B6C4FF47A709847F860FB68EC
:10836000002BCCD0F9687868FFF734FEFB681B68F7
:10837000184607F085FAF86807F082FABFE77B68CD
:108380009B6C9847796A0A4807F0AAF93037BD46CE
:10839000BDE89088641B0600E81B0600EC1B060085
:1083A000F41B0600F81B0600341C0600701C0600B7
:1083B0009C1C060080B5B6B002AF786007F10800DB
:1083C0004FF496730093324B324A022100F0C0F80A
:1083D00007F1080319467868FEF73AFB07F108032E
:1083E00018461AF0DDFF07F13000002300932A4BF6
:1083F0002A4A022100F0ACF807F1300319467868E8
:10840000FEF726FB07F1300318461AF0C9FF07F103
:108410005800234B0093234B234A0321F9F76EF9AD
:1084200007F1580319467868FEF712FB07F1580365
:1084300018461AF0B5FF07F18000194B00931B4B4B
:108440001B4A0321F9F75AF907F1800319467868A6
:10845000FEF7FEFA07F1800318461AF0A1FF07F1B4
:10846000A8000F4B0093134B134A0321F9F746F969
:1084700007F1A80319467868FEF7EAFA07F1A8039E
:1084800018461AF08DFF00BFD037BD4680BD00BF33
:10849000C01C0600001D06000C1D06004C1D060039
:1084A000A81D0600581D0600A01D0600AC1D0600F4
:1084B000FC1D0600081E0600601E060080B586B082
:1084C00002AF786039600023FB73396807F10F024F
:1084D00048F6A0430193002300930B4617497868A0
:1084E000FEF71EFE3B68991C07F10F0248F6A043F9
:1084F0000193002300930B4611497868FEF710FEA4
:10850000104978681DF0EBFD02463B685A600E4941
:1085100078681DF0E4FD02463B689A600B49786874
:108520001DF0DDFD02463B68DA60FB7B83F0010352
:10853000DBB218461037BD4680BD00BF001D0600E7
:108540004C1D0600A01D0600FC1D0600601E060056
:1085500080B584B000AFF860B9607A603B60FB68BA
:1085600000221A70FB68BA685A60FB687A689A60E1
:10857000FB683A68DA60FB68103318461AF023FF8C
:10858000FB681C3318461AF01EFFB969F8681BF027
:1085900081FF034683F00103DBB2002B07D079682B
:1085A000094807F09DF82021084800F07BF9FB6896
:1085B0001C33BA691946F8681BF0A7FEFB68184619
:1085C0001037BD4680BD00BF6C1E0600981E060019
:1085D000F0B58FB006AFFBF7A7FF03463B613B69E1
:1085E0001946594807F07CF83A691346DB001344F2
:1085F0009B00184607F062F97861544807F070F85C
:108600007B69002B00F09C803B6907F1080219464A
:108610007869FBF795FF03463B610023FB6087E029
:10862000FA681346DB0013449B001A467B69134427
:108630001B7B042B1BD801A252F823F057860300A2
:10864000518603005D86030063860300698603008C
:108650007223FB770EE05223FB770BE04223FB777C
:1086600008E05323FB7705E04423FB7702E03F2338
:10867000FB7700BF0023BB61BB68642B10D9FA688D
:108680001346DB0013449B001A467B6913449A6926
:10869000BB682F49A1FB03135B09B2FBF3F3BB617A
:1086A000FA681346DB0013449B001A467B691344A7
:1086B0005C68FD7FFA681346DB0013449B001A4692
:1086C0007B6913441E69FA681346DB0013449B0060
:1086D0001A467B6913441B8C7B60FA681346DB00E7
:1086E00013449B001A467B6913449968FA68134641
:1086F000DB0013449B001A467B6913449869FA68AF
:108700001346DB0013449B001A467B691344DB6964
:108710000493BB690393029001917B6800933346F5
:108720002A4621460B4806F0DBFFFB680133FB605D
:10873000FA683B699A42FFF473AF786907F0A0F8D2
:1087400000BF2437BD46F0BDD41E0600E01E060063
:108750001F85EB51181F060098B500AF154806F0AD
:10876000BFFFFFF735FFFDF7F3F904461BF035FDBA
:1087700003461A462146104806F0B2FF0F4B1B88ED
:1087800019460E4B9B8818460C4B1B881A460B4B00
:108790009B88D31A02460A4806F0A2FF094B1B68C1
:1087A000002B02D0074B1B689847074806F098FF3C
:1087B00000BF98BD4C1F0600581F060080EB02202A
:1087C000781F060098CE02209C1F060080B483B05C
:1087D00000AF7860044A7B68136000BF0C37BD4669
:1087E0005DF8047B704700BF9CCE022080B483B04C
:1087F00000AF7860044A7B68136000BF0C37BD4649
:108800005DF8047B704700BFA0CE022080B586B023
:1088100002AF786039601D4B1B78DBB283F0010337
:10882000DBB2002B07D01A4B1B78DBB2002B02D037
:108830001EF0ABFEFEE7164B01221A7064220021E7
:10884000144825F007FD7B6800933B68124A6421B9
:1088500010480DF07FFD114B1B68002B02D00F4B11
:108860001B6898470B4806F09BFF1EF08EFE074BD7
:1088700001221A700023FB6002E0FB680133FB60F9
:10888000FB68074A9342F8DDECE700BFABE9022042
:10889000ACE90220A4CE0220582006009CCE022083
:1088A000FEFF0F0080B588B002AF78603960374BAB
:1088B0001B78DBB283F00103DBB2002B11D0344B09
:1088C0001B78DBB2002B0CD000237B6102E07B69BC
:1088D00001337B617B692F4A9342F8DD1EF055FE20
:1088E000FEE72B4B01221A70642200212A4825F052
:1088F000B1FC7B6800933B68284A642126480DF050
:1089000029FD274B1B68002B03D0254B1B682248F1
:10891000984700233B6114E01F4806F041FF2148BF
:1089200006F03EFF1EF031FE0023FB6002E0FB6814
:108930000133FB60FB681C4A9342F8D93B69013361
:108940003B613B690F2BE7DD1EF01FFE174B1B68D9
:10895000002B02D0154B1B6898470F4806F020FFEC
:10896000104806F01DFF124806F01AFF1EF00DFE1B
:10897000064B01221A700023BB6002E0BB68013382
:10898000BB60BB68084A9342F8D9E6E7ADE902202C
:10899000AEE90220FEFFFF00A4CE022080200600E8
:1089A000A0CE022090200600FEFF0F009CCE0220E9
:1089B000AC20060080B586B000AFB9607A603B603D
:1089C0000346FB731C2006F079FF78617B69002B5E
:1089D00004D1214806F084FE002338E07B69FA7B4D
:1089E0001A707B69BA685A607B693A685A613B6859
:1089F000002B1CD07B68002B19D0386806F05EFF76
:108A000002467B699A617B699B69002B07D1786973
:108A100006F036FF104806F063FE002317E07B697E
:108A20009B693A687968184625F0F0FB02E07B699B
:108A300000229A61094B1B680133084A1360074BF7
:108A40001B681A467969064806F04AFE7B69184693
:108A50001837BD4680BD00BFD020060074CF02206D
:108A6000EC20060080B582B000AF78607B68002BF8
:108A700013D00C4B1B68013B0A4A1360094B1B685F
:108A80001A467968084806F02BFE7B689B691846F1
:108A900006F0F6FE786806F0F3FE00BF0837BD4624
:108AA00080BD00BF74CF02200C21060080B584B0C9
:108AB00000AF7860084B1B6807F10C017A68184614
:108AC000FAF7DEFE0346012B01D1FB6800E000232C
:108AD00018461037BD4680BD4CCF022080B5AAB0E5
:108AE00000AFF860B9607A603B60FB68002B03D18F
:108AF0005B215D48FFF7D6FEBB68002B03D15C21EC
:108B00005948FFF7CFFE07F198033A68796818468D
:108B100022F08AF80023C7F8A430FB6800221A70FC
:108B200007F198030021184622F08CFC0346002B25
:108B300000F0958007F198030021184622F0A1FC6F
:108B40000346002B01D000238AE007F1940207F1CD
:108B500098030021184622F096FB0246D7F8A4306D
:108B60001344C7F8A43073E007F19803D7F8A410B2
:108B7000184622F048FC034683F00103DBB2002BC9
:108B80001AD007F19803D7F8A410184600F056F948
:108B90000246D7F8A4301344C7F8A43007F198036D
:108BA000D7F8A410184600F049F90246D7F8A430C7
:108BB0001344C7F8A4304BE007F1100207F1980006
:108BC0008023D7F8A41022F0CEFA0246D7F8A430BA
:108BD0001344C7F8A43007F110031946D7F8B000C2
:108BE00025F0D4FC0346002B25D107F19803D7F8D4
:108BF000A410184622F007FC0346002B19D0BB68CE
:108C0000013BFA68134400221A70BB68013B07F16C
:108C10009800FA68D7F8A41022F0A5FA0246D7F80F
:108C2000A4301344C7F8A430F86825F0D6FC0346F6
:108C300016E0002314E007F19803D7F8A4101846B3
:108C400000F0FCF80246D7F8A4301344C7F8A4306B
:108C5000D7F894305A1EC7F89420002B84D10023F3
:108C60001846A837BD4680BD2C210600B0B582B09D
:108C700000AF78603960364A7B6814461D460FCDD8
:108C80000FC40FCD0FC42B682360002201210120E7
:108C9000FAF774FC02462F4B1A602E4B1B68002B10
:108CA00003D18A212C48FFF7FDFD00220821012075
:108CB000FAF764FC0246294B1A60284B1B68002B0C
:108CC00003D18C212448FFF7EDFD0022042101206F
:108CD000FAF754FC0246224B1A60214B1B68002B0A
:108CE00003D18E211C48FFF7DDFD002204210A205C
:108CF000FAF744FC02461B4B1A601A4B1B68002B08
:108D000003D190211448FFF7CDFD1422002116480D
:108D100025F0A0FA3B68002B07D0134A3B681446A5
:108D20001D460FCD0FC42B682360092200210F4878
:108D300025F090FA092200210D4825F08BFA09222E
:108D400000210C4825F086FA00BF0837BD46B0BDAB
:108D500008CF022040CF02202C21060044CF022061
:108D600048CF02204CCF02202CCF022050CF02202F
:108D70005CCF022068CF022080B588B000AFF860D9
:108D8000B9607A603B6007F11403BA68F968184665
:108D900021F04AFF07F11403184622F041FA07F1C7
:108DA00014032149184622F028FA204B5A6807F18B
:108DB00014031146184622F020FA07F114031C4947
:108DC000184622F01AFA194B1B68984703461A46B0
:108DD00007F114031146184622F014F97B68002BA2
:108DE0000BD007F114031349184622F006FA07F1D5
:108DF00014037968184622F000FA07F114030E49AB
:108E0000184622F0FAF907F11403BA6A39681846CD
:108E100022F0E8F807F11403184622F058FAFB692B
:108E200018462037BD4680BD6421060008CF0220C9
:108E3000682106006C2106007021060080B588B00C
:108E400000AF786039603968786822F095FA034697
:108E5000002B08D007F110031A463968786822F011
:108E600078F8034658E03968786822F0CCFA03466F
:108E7000002B09D007F1140307F11802396878684C
:108E800022F096F9034647E03968786822F0DAFA6A
:108E90000346002B34D03968786822F0F2FA034692
:108EA000002B02D01E4806F01BFC0023FB6107F1DB
:108EB0000C031A463968786822F0E5F90246FB6926
:108EC0001344FB6115E03A68FB691344194678685E
:108ED000FFF7B4FF0246FB691344FB613A68FB6984
:108EE000134419467868FFF7A9FF0246FB6913444B
:108EF000FB61FB685A1EFA60002BE4D1FB690BE0B2
:108F00007B681A683B6813441B7803F0E00319463A
:108F1000044806F0E5FB002318462037BD4680BD17
:108F2000742106008421060080B58EB000AF786001
:108F3000396000237B6307F120033A68796818469B
:108F400021F072FE07F12003796B184622F07AFABD
:108F50000346002B00F0AC8007F12003796B184624
:108F600022F08FFA0346002B02D0544806F0B8FBDB
:108F700007F11C0207F12003796B184622F083F9F0
:108F800002467B6B13447B632C2006F097FC38630E
:108F90003B6B00221A703B6B00225A623B6B002233
:108FA0009A6268E007F10C0207F120001023796B48
:108FB00022F0D9F802467B6B13447B6307F10C0364
:108FC00019463F4825F0E2FA0346002B14D107F179
:108FD0002003796B184622F016FA0346002B4AD07C
:108FE0003A6B07F120002023796B22F0BCF802468F
:108FF0007B6B13447B633EE007F10C031946314859
:1090000025F0C4FA0346002B2BD107F12003796B1E
:109010001846FFF713FFF8623B6B5B6A002B15D114
:10902000F86A06F04BFC02463B6B5A623B6B5B6A8C
:10903000002B0BD03B6B586A3A6A7B6B1344FA6A7D
:10904000194625F0E3F83B6BFA6A9A6207F12003B0
:10905000796B1846FFF7F2FE02467B6B13447B6385
:1090600009E007F12003796B1846FFF7E7FE024697
:109070007B6B13447B6307F12003796B184622F066
:10908000C2F90346002B04D0FB695A1EFA61002B7B
:1090900088D13B6B1B78002B08D13B6B5B6A002BA4
:1090A00004D1386B06F0ECFB002302E03B6B00E0E0
:1090B000002318463837BD4680BD00BF9C210600FE
:1090C0006C2106007021060080B584B000AF786086
:1090D0001C4806F005FB7B68002B2AD07B68DB6907
:1090E000002B26D07B681B89002B22D07B68DA6995
:1090F0007B681B8919461046FFF716FF0346FB6085
:10910000FB68002B19D0104806F0EAFA0F4B1868DC
:1091100007F10C0100230022FAF768FA0346012B3D
:109120000BD00B4806F0DCFAFB6818461EF035FA47
:1091300003E0084806F0D4FA00E000BF00BF103793
:10914000BD4680BDB4210600D02106004CCF0220D0
:10915000F02106002022060090B587B002AF7860AB
:1091600039601D4806F0BCFA7B68002B0ED11B4805
:1091700006F0B6FA0023FB73194B186807F10F01CC
:1091800000230022FAF732FA002321E0154A7C6816
:109190006B46111D03C9186004331970136804F17C
:1091A0000C0207CA26F04DFA0346002B0FD00E48DA
:1091B00006F096FA0123BB737868FFF785FF084B2A
:1091C000186807F10E0100230022FAF70FFA0023B6
:1091D00018461437BD4690BD382206004C220600C2
:1091E00040CF022050CF02206022060090B587B009
:1091F00002AF78603960314806F072FA4FF0000330
:109200004FF00004C7E902347B68002B0CD12C48D6
:1092100006F066FA2B4B186807F1080100230022BC
:10922000FAF7E4F9002345E0274A7C686B46111DF4
:1092300003C9186004331970136804F10C0207CADB
:1092400026F0FFF90346002B30D0204806F048FAFC
:109250007B681B8919461E4806F042FA7B68D9696B
:109260007B681B891A461B4806F0F4FA7B681B8949
:10927000052B0FD17B68DB69184621F0A4FA034661
:109280000C46C7E90234D7E902341946124806F001
:1092900027FA02E0114806F023FA0A4B186807F192
:1092A000080100230022FAF7A1F902E00C4806F0B9
:1092B00017FA002318461437BD4690BD70220600E9
:1092C0004C22060044CF02205CCF02206022060020
:1092D0008C220600A0220600A8220600B422060066
:1092E000C822060080B582B000AF78600B4B1868CA
:1092F000391D00230022FAF779F90346012B08D023
:109300007B681946064806F0EBF97B681846FFF7BC
:10931000A9FB00BF0837BD4680BD00BF48CF022073
:10932000DC22060090B5ADB002AF786039607E48AF
:1093300006F0D6F90023C7F89C307B68002B07D1D4
:109340007A4806F0CDF90020FFF7CCFF0023E6E0D5
:10935000774A7C686B46111D03C918600433197085
:10936000136804F10C0207CA26F06BF9034683F078
:109370000103DBB2002B04D06E4806F0B1F90023E4
:10938000CDE06B4B00221A706B4806F0A9F97B68A0
:109390001B891946694806F0A3F97B685B79002BA5
:1093A00004D1674806F09CF90023B8E07B685B793C
:1093B000842B0DD10023002200210120FFF7FAFAAF
:1093C000C7F89400D7F89400FFF78CFF0023A6E0BD
:1093D0007B685B79452B40F09A804FF0FF33C7F8EC
:1093E00090304FF0FF33C7F88C304FF0FF33C7F8A1
:1093F00088307B689B69C7F8A43045E0D7F8A43073
:109400009B880F2B3BD17F23C7F8A030D7F8A4301F
:10941000DB887F2B04D8D7F8A430DB88C7F8A030CE
:10942000D7F8A430996807F10803D7F8A0201846A8
:1094300024F0ECFE07F10802D7F8A0301344002214
:109440001A7007F1080319463E4806F049F907F17A
:10945000900207F108033C4918460CF0CFFF07F1D2
:109460008C0207F10803394918460CF0C7FF07F1D1
:10947000880207F10803364918460CF0BFFFD7F8F9
:10948000A4301B68C7F8A430D7F8A430002BB5D19E
:10949000D7F89030B3F1FF3F09D0D7F88C30B3F153
:1094A000FF3F04D0D7F88830B3F1FF3F08D12948F7
:1094B00006F016F9D7F89C00FFF714FF00232EE002
:1094C000D7F890107B68DA697B681B890020FFF76A
:1094D00071FAC7F89800D7F88C20D7F898309A60BE
:1094E000D7F88820D7F89830DA60D7F88C20D7F8EA
:1094F00088309A422CBF01230023DAB2D7F8983083
:109500001A74D7F89800FFF7EDFE002307E0124B1E
:109510001868002300220021FAF768F80023184693
:10952000AC37BD4690BD00BF0C2306004C220600A0
:1095300068CF0220C8220600602206008C220600A6
:10954000242306005023060060230600682306003B
:10955000702306007823060048CF0220F0B5ADF551
:10956000865D81B006AF07F128041C3C206007F13E
:109570000800016007F1080104390A6007F10802D8
:10958000083A136007F10803043B07F1080107F1EB
:10959000A800083807F10802083A126800921B6810
:1095A0000A684FF48051FFF7E7FB07F5855303F195
:1095B0000403186007F12803083B374A1C4613468A
:1095C0000FCB07C4238007F12803143B184610F083
:1095D0001FFA10F00BFA03469C4607F5855303F17A
:1095E00004031B689DB207F5855303F104031B6850
:1095F0009EB207F1A804083C07F12802143A02AB16
:1096000007CA03C31A7001960095234662460221D9
:1096100000200FF09BFE07F58553186007F5855372
:109620001B68002B23D007F585531B6803F1180234
:1096300007F12803083B1946104626F0E2FE07F121
:109640002803153B3C221A7007F12802153A012322
:109650000C2107F58550006826F036FB0F4B996802
:109660000F4B104A07F5855000680EF035F907F1E9
:1096700028031C3B1A6807F12803143B03CB106036
:1096800051601B78137207F128031C3B186807F51B
:1096900085570C37BD46F0BDA023060008CF022039
:1096A0005991030014CF022090B58BB000AFF86140
:1096B000B9617A61144B1B6800211846F9F702FF63
:1096C000124C38467B69BA69F969FFF747FF2346B0
:1096D0003A461068516803C3127A1A700A4B1B6825
:1096E00007F127010A4A1846FAF7CAF80346012B80
:1096F00002D197F8273003E0064805F0F1FF002378
:1097000018462C37BD4690BD40CF022050CF0220D6
:10971000A0860100B023060090B58FB006AF234CA1
:109720003B46184610F074F923463A4610685168D3
:1097300003C3127A1A7010F059F903461C461B4AEB
:1097400002AB07CA03C31A700023019300230093DE
:1097500000232246012100200FF0F8FDF861FB698B
:1097600018331349184626F04CFE124B9968124BD9
:10977000124AF8690EF0B0F8114B1B6807F110019E
:10978000104A1846FAF77CF80346012B02D1D7E9B4
:10979000043406E00C4805F0A3FF4FF000034FF03F
:1097A0000004184621462437BD4690BD5CCF0220F8
:1097B000D023060008CF0220ED91030014CF022031
:1097C00044CF0220A0860100B023060090B5AFB0C0
:1097D00006AF786139612B4C3B46184610F018F9FA
:1097E00023463A461068516803C3127A1A7010F083
:1097F000FDF803461C46234A02AB07CA03C31A708E
:10980000002301930023009300232246012100201E
:109810000FF09CFDC7F89C001B4B5B6807F11C0018
:1098200001933B6900937B69184A80210CF092FDFB
:10983000D7F89C30183307F11C021146184626F061
:10984000E0FD114B9968124B124AD7F89C000EF0BC
:1098500043F8114B1B6807F11801104A1846FAF734
:109860000FF80346012B04D10D4805F039FFBB6901
:1098700003E00C4805F034FF00231846A437BD462A
:1098800090BD00BF68CF022008CF0220D42306007D
:109890002593030014CF022048CF0220A0860100A8
:1098A000E8230600B023060080B582B000AF7860E0
:1098B0007B6819461E4824F069FE0346002B05D13B
:1098C00079681C4800F0EEF903462DE07B681946E4
:1098D000194824F05BFE0346002B04D1786800F0A1
:1098E00015FB034620E07B681946144824F04EFE21
:1098F0000346002B05D179680E4800F041FB034672
:1099000012E07B6819460E4824F040FE0346002B07
:1099100004D1084800F064FB034605E07B68194663
:10992000084805F0DDFE002318460837BD4680BD17
:10993000002406002CCF0220042406000C2406007C
:10994000142406001C24060090B58FB004AFF86004
:10995000B9601346FB71BB68002B03D10E216B4825
:10996000FEF7A0FFB9686A4805F0BAFE0323FB774B
:10997000002387F827303C23BB8300233B62AFE002
:10998000396AB868FFF722FFB861B969614805F024
:10999000A7FEBB69002B33D13A6AB9685E4805F06F
:1099A0009FFE97F82730013387F8273097F8272054
:1099B000FB7F9A4219D897F82710FA7FBB8B57483C
:1099C00005F08EFEBB8B564A02FB03F31A46554B3D
:1099D000A3FB02239B091846FAF75AFB524805F0ED
:1099E0007FFE3B6A013B3B6277E03B6A0093BB68CA
:1099F0004E4A4FF480714E480CF0ACFC002380E0DE
:109A0000BB691B78012B0FD1B9684A4805F068FE85
:109A1000BB68494A4FF4807145480CF09BFCB8691B
:109A2000FFF720F800236CE0BB691B78002B54D1B2
:109A3000002387F82730BB69D868BB695B69BA69BE
:109A40005268B969097C02910192009303463A6A0F
:109A5000B9683A4805F044FEFB68DC68BB695868A1
:109A6000BB699969BB695A69FB79A0470346FB75D5
:109A7000B869FEF7F7FFFB7D83F00103DBB2002B33
:109A80001ED0BB69DA68BB695B68009313463A6A0B
:109A9000B9682B4805F024FEBB69DB68BA695268D7
:109AA000029201933B6A0093BB68264A4FF480718F
:109AB0001F480CF04FFCB869FEF7D4FF002320E0EC
:109AC000BB691B7C002B08D0BB69DB683A6AB968AC
:109AD0001D4805F005FE012313E03B6A01333B629C
:109AE0003B6AB3F57A6FFFF44BAFB968174805F0DE
:109AF000F7FDBB68164A4FF480710D480CF02AFC44
:109B0000002318462C37BD4690BD00BF44240600F4
:109B1000842406009C240600B0240600D4240600F9
:109B200040420F00D34D6210F42406000C250600BD
:109B3000D8E902202C2506005425060070250600D1
:109B4000A4250600D42506000426060018260600D3
